:020000040000FA
:1000000090DB0020390300005D0300005F03000067
:100010006103000063030000650300006703000044
:100020006703000067030000670300006703000028
:1000300067030000670300003B300000EF32000060
:10004000DF8D0000E98D0000F38D0000FD8D0000C4
:10005000078E0000118E00001B8E0000258E000010
:100060002F8E0000398E0000438E00004D8E000060
:10007000578E0000618E00006B8E0000758E0000B0
:100080007F8E0000898E0000938E00009D8E000000
:10009000A78E0000B18E0000BB8E0000C58E000050
:1000A000CF8E0000D98E0000E38E0000ED8E0000A0
:1000B000F78E0000018F00000B8F0000158F0000ED
:1000C0001F8F0000298F0000338F00003D8F00003C
:1000D000478F0000518F00005B8F0000658F00008C
:1000E0006F8F0000798F0000838F00008D8F0000DC
:1000F000978F0000A18F0000AB8F0000B58F00002C
:10010000BF8F0000C98F0000D38F0000DD8F00007B
:10011000E78F0000F18F0000FB8F000005900000CA
:100120000F90000019900000239000002D90000017
:1001300037900000419000004B9000005590000067
:100140005F90000069900000739000007D900000B7
:1001500087900000919000009B900000A590000007
:10016000AF900000B9900000C3900000CD90000057
:10017000D7900000E1900000EB900000F5900000A7
:10018000FF90000009910000139100001D910000F4
:1001900027910000319100003B9100004591000043
:1001A0004F910000619100006B910000759100007B
:1001B0007F91000089910000939100009D910000C3
:1001C000A7910000B1910000BB910000C591000013
:1001D000CF910000D9910000E3910000ED91000063
:1001E000F7910000019200000B92000015920000B0
:1001F0001F92000029920000339200003D920000FF
:1002000000F002F800F071F80AA090E8000C8244B7
:100210008344AAF10107DA4501D100F066F8AFF294
:10022000090EBAE80F0013F0010F18BFFB1A43F0D4
:100230000103184750760100707601000A444FF020
:10024000000C10F8013B13F0070408BF10F8014B35
:100250001D1108BF10F8015B641E05D010F8016B7A
:10026000641E01F8016BF9D113F0080F1EBF10F8DE
:10027000014BAD1C0C1B09D16D1E58BF01F801CB01
:10028000FAD505E014F8016B01F8016B6D1EF9D584
:100290009142D6D370470000002300240025002699
:1002A000103A28BF78C1FBD8520728BF30C148BFD9
:1002B0000B607047642915F07B86732916F08D82D8
:1002C000002070471FB516F053FB9DE8030016F0A1
:1002D000C5F916F0A7F904000020002116F032FB42
:1002E000401C60601FBD10B510BD16F0A1FA11468C
:1002F000FFF7E8FF15F097FC16F0BFFA03B4FFF71D
:10030000F2FF03BC16F0F0FAEFF3108072B67047FC
:10031000EFF310807047EFF3108062B6704730BF84
:10032000704780F311887047EFF311807047000029
:100330000138FDD170470000DFF83C00016841F44E
:1003400070010160BFF34F8FDFF83000016821F0CA
:1003500040410160BFF36F8F09480047FEE7FEE7A9
:10036000FEE7FEE7FEE7FEE7FEE700000548064978
:10037000064A074B7047000088ED00E034EF00E0CC
:1003800001020000909B002090DB002090CB002019
:1003900090CB002010B50246F64B1B68F64C23406C
:1003A000F64CA34209D1F64B9A4202D101F11E0349
:1003B00001E001F14003184611E0EE4B1B68EE4CE2
:1003C0002340F04CA34209D1ED4B9A4202D101F1F6
:1003D0001E0301E001F13E03184600E0002010BDBD
:1003E0002DE9F04105460E46144631462846FFF7F2
:1003F000D1FF07462146384601F0E0F9384601F0C2
:1004000039FABDE8F08170B504460D46294620460C
:10041000FFF7C0FF0646304601F068FA304601F0AB
:10042000E7F970BD826801238B409A438260704770
:1004300001228A40C260826801238B401A43826095
:10044000704730B5034632B1DC684FF001158D407E
:1004500004EA05000FE05C6801258D4045F4803515
:1004600004EA050000F480342CB140F470204FF40D
:1004700080348C40A04330BD01228A40C260704766
:10048000026801238B401A4302607047026801230F
:100490008B409A430260704770B5144689004569E5
:1004A0000F268E40B54304F00F068E40354345615C
:1004B000056A0F268E40B54303F003068E40354390
:1004C000056204F00F02062A0CD3092A0AD8951FE8
:1004D000EA00C56930269640B54304F030069640E0
:1004E0003543C56170BD70B50C4665014035284483
:1004F000920005680F269640B54303F00F0696401C
:100500003543056085690F269640B543C3F303263E
:1005100096403543856146680F25954026EA0505D6
:10052000C3F30316964035434560C6690F259540D1
:1005300026EA0505C3F3035696403543C56103F427
:10054000702575B141690F259540A943C3F3024554
:10055000954029434161056901269640354305616F
:1005600004E0056901269640B543056170BD024669
:10057000106901238B401840704701228A400261B4
:1005800070470246906901238B4018407047012252
:100590008A408261704710B503464C0140342344C1
:1005A000002002E09C6810C2401CDC6804F48074E7
:1005B0000CB90828F6D310BD10B50A0C120401F0CE
:1005C0000F040123A3401A43836A1A43826210BDB9
:1005D000F0B503460024520801E0641C5208002ACA
:1005E000FBD1674DAB4201D1002000E0012000EBC0
:1005F0004006654F3E447454F0BD70B5604DA8424E
:1006000001D1002400E001244D014035284404EBD1
:1006100044055D4E35446E5C0425B5406A4304EBE9
:100620004405594E35446E5C012505FA06F124E077
:1006300005680F269640B54303F00F0696403543F4
:10064000056085690F269640B543C3F3032696409F
:100650003543856146680F25954026EA0505C3F3B5
:100660000316964035434560012904D046680625A7
:100670009540AE434660121D491E0029D8D170BD79
:10068000F0B514463E4FB84201D1002200E00122ED
:100690004F014037384419E0002602EB4207DFF8EB
:1006A000E8C0674417F801C0012707FA0CF502E01B
:1006B00087683E446D1E002DFAD102EB4207DFF839
:1006C000C8C067447F5C26FA07F780C41F1EA3F1E9
:1006D0000103E1D1F0BD0022490801E0521C4908A4
:1006E0000029FBD10263704700F5606343F82120C5
:1006F000704730B542EA034500F5646444F8215080
:1007000030BD70B5044600202AB101F11005012664
:1007100006FA05F5284313B101258D402843C4F896
:10072000000D70BD82684FF480338B409A43826025
:10073000704782684FF480338B401A438260704761
:100740000146486B70474163704782688A43826004
:10075000704782680A4382607047024609B1D068D8
:1007600005E0506800F480330BB140F4702070470E
:10077000C160704700E00F400000FF7000000510EE
:100780000080034000000A1000000020826B22F06D
:1007900003020A43826370470146886B00F003003E
:1007A0007047416270470146486A704702684FF4DB
:1007B00080738B401A430260704702684FF4807365
:1007C0008B409A430260704701460868C0F30040BE
:1007D000704710B5C1F30313C0F8C43F531E0C4655
:1007E00063F31F14C0F8C84F10BD0246084B1868C9
:1007F00019B1C0F305135B1C0B6020F47C70044B33
:100800001B1F1B6803F00F0340EA03107047000032
:10081000C88F034070B50446E10901208840C543F4
:100820000A20FFF785FD0320D34908600A20FFF75F
:100830007FFDD248C0F8C0520A20FFF779FD0020A2
:10084000CD4908600A20FFF773FD70BD10B50A207E
:10085000FFF76EFD0320C84908600A20FFF768FD16
:100860000020C649C1F8C0020A20FFF761FD002040
:10087000C14908600A20FFF75BFD10BD00BFC048FA
:10088000806900F001000028F9D1704710B50220FE
:10089000FFF74EFDFFF7F2FFB948C46904F00C0002
:1008A00008B1022010BDB74801F0D7FA0220FFF7C7
:1008B0003FFDFFF7E3FFB248C46904F00C0008B144
:1008C0000220EFE70020EDE7AD4800680004800B50
:1008D0007047AB480068C0F30A40704710B58B09F9
:1008E000A74C6360C1F38303A36092080DE0A44B9F
:1008F0005B690360001D521E3AB1A14B9B6823B98E
:100900009F4B5B685B1C9E4C6360002AEFD110BD5F
:100910002DE9F04107460E46144600BF9848856908
:1009200005F001000028F9D1B00995494860C6F3E7
:1009300083008860A40838E0934800689349084021
:100940009349884206D19048006880B210B9304679
:10095000FFF760FF8A49386848610A20FFF7E8FC22
:1009600000BF8748856905F001000028F9D105F02E
:10097000100078B18448006884490840844988425E
:1009800005D18148006880B208B9FFF75FFF2846AB
:10099000BDE8F0813F1D641E3CB17948806820B9F4
:1009A00077484068401C76494860002CC4D176489E
:1009B0000068764908407649884205D17248006847
:1009C00080B208B9FFF742FF6D488069E0E770B573
:1009D00005460C466C4800686C4908406C498842E2
:1009E00006D16948006880B210B92046FFF712FFAF
:1009F000A00963494860C4F38300886008464561E4
:100A0000806970BD10B56048006860490840604961
:100A1000884205D15C48006880B208B9FFF716FF2C
:100A20005C48574980310860FFF728FF554801F0BE
:100A300014FA0220FFF77CFCFFF720FF5048806982
:100A400010BD01464E484160006B704702464C485D
:100A50004260016300BF4A48806900F0010000283D
:100A6000F9D147488069704710B503464448436050
:100A7000434C34340BE008682060091D241D521ECD
:100A800000BF3F48806900F001000028F9D1002A2A
:100A9000F1D13B48806910BD0146394841604FF0B3
:100AA000FF30374A10621046006A704710B503469F
:100AB000334843604FF0FF30314C2062501E01EB51
:100AC000800104E051F804092D4C2062521E002AD6
:100AD000F8D12B48006A10BD01218140284A1165D8
:100AE00070472749096C41F00101254A11642249E8
:100AF000FC39096941F004011F4AFC3A1161704751
:100B00001D49FC39096921F004011B4AFC3A1161B5
:100B10001B49096C21F00101194A11647047014613
:100B200049B11548FC38406900F0040008B10420C0
:100B300070470020FCE71248806900F0010008B10E
:100B40000020F5E70420F3E710B5044604200A4925
:100B5000FC3948610C4800680C4908400C4988423F
:100B600005D10948006880B208B9FFF76FFE10BDD3
:100B70000348806970470000FCD00F4000E00A4045
:100B800000F00A40005800F000E00F400000FF7045
:100B90000000051001007BE330B50246F74B182436
:100BA000F7480068F74D2840F74DA84201D1F74BB0
:100BB0001B24002108E053F83100904203D103EBDD
:100BC000C100406830BD491CA142F4D30020F9E7C0
:100BD00002F001031BB1D0F800340B4302E0D0F85F
:100BE00000348B43C0F8003402F002031BB1D0F88C
:100BF00020340B4302E0D0F820348B43C0F820347B
:100C0000704730B5024601208840C1B2D2F80034A6
:100C1000D2F8204403EA010008B1012000E00020DE
:100C200004EA01050DB1022500E00025284330BD8E
:100C300002F001031BB1D0F808340B4302E0D0F8F6
:100C400008348B43C0F8083402F002031BB1D0F81B
:100C500004340B4302E0D0F804348B43C0F804346E
:100C600002F004031BB1D0F80C340B4302E0D0F8BF
:100C70000C348B43C0F80C3402F4803323B1D0F829
:100C8000383543F0010303E0D0F8383523F0010391
:100C9000C0F838357047F0B5024601208840C1B22F
:100CA000D2F80834D2F80444D2F80C64D2F838559B
:100CB00003EA010008B1012000E0002004EA010776
:100CC0000FB1022700E00027384306EA01070FB101
:100CD000042700E00027384305F0010717B14FF45F
:100CE000803700E000273843F0BDF0B5A44D2D68F3
:100CF000A44E3540A64EB5421AD0002416E0012578
:100D0000A5400D4085B1D0F8C45F67000326BE4002
:100D1000B543C0F8C45FD0F8C45F6700C2F34116A2
:100D2000BE403543C0F8C45F651CECB2082CE6DB5E
:100D300002F001051DB1D0F800550D4302E0D0F8D6
:100D400000558D43C0F8005502F002051DB1D0F8E2
:100D500004550D4302E0D0F804558D43C0F8045506
:100D600002F004051DB1D0F808550D4302E0D0F89B
:100D700008558D43C0F8085502F008051DB1D0F89C
:100D800018550D4302E0D0F818558D43C0F818559A
:100D90007B4D2D687B4E35407D4EB5420BD002F029
:100DA00010051DB1D0F83C550D4302E0D0F83C557C
:100DB0008D43C0F83C5503F001051DB1D0F80C552A
:100DC0000D4302E0D0F80C558D43C0F80C5503F0EC
:100DD00002051DB1D0F810550D4302E0D0F81055B2
:100DE0008D43C0F8105503F004051DB1D0F814551B
:100DF0000D4302E0D0F814558D43C0F8145503F0AC
:100E000008051DB1D0F81C550D4302E0D0F81C5563
:100E10008D43C0F81C555A4D2D685A4E35405C4ED6
:100E2000B54217D003F400751DB1D0F844550D43F9
:100E300002E0D0F844558D43C0F8445503F44075A2
:100E40001DB1D0F840550D4302E0D0F840558D4318
:100E5000C0F840551BB9D0F828550D4302E0D0F832
:100E600028558D43C0F82855F0BDF0B514461D46F1
:100E700001268E40F1B2D0F800650E400EB1012679
:100E800000E000263246D0F804650E400EB102267E
:100E900000E000263243D0F808650E400EB104266B
:100EA00000E000263243D0F818650E400EB1082647
:100EB00000E000263243324E3668324F3E40344F17
:100EC000BE420FD0D0F83C650E400EB1102600E0B7
:100ED00000263243D0F8C46F4F00FE4006F00306F0
:100EE00042EA46122260D0F80C650E400EB101268F
:100EF00000E000263346D0F810650E400EB1022601
:100F000000E000263343D0F814650E400EB10426ED
:100F100000E000263343D0F81C650E400EB10826D1
:100F200000E000263343164E3668164F3E40184FF9
:100F3000BE420CD0D0F840650E4046B1D0F84465B2
:100F40000E400EB1FE1401E04FF4807633432B6067
:100F5000F0BDD0F810240A43C0F810247047D0F830
:100F600010248A43C0F810247047024611B1D2F809
:100F700018047047D2F81404FBE700007C690100F4
:100F800000E00F400000FF7000000A103C6A010002
:100F900000000510C0F81C14704770B504460D46DB
:100FA0002046FFF7F9FD06462946304600F006FCCC
:100FB000304600F05FFC70BD70B504462046FFF778
:100FC000EBFD0546284600F091FC284600F010FC99
:100FD00070BD2DE9F04107460C4615463846FFF72F
:100FE000DBFD06463019294600F0E8FB301900F019
:100FF00041FCBDE8F08170B506460C463046FFF76F
:10100000CBFD0546281900F071FC281900F0F0FB13
:1010100070BD0246002000EB81001058704700238D
:1010200003EB8103C250704730B504460D460022E1
:1010300029462046FFF7CCFD002301222946204601
:10104000FFF753FE30BD30B504460D460222294657
:101050002046FFF7BDFD0823662229462046FFF7FC
:1010600044FE30BD30B504460D46002229462046D8
:10107000FFF7AEFD0023012229462046FFF735FE8B
:1010800030BD30B504460D46022229462046FFF702
:101090009FFD0823012229462046FFF726FE30BD8A
:1010A00030B504460D46022229462046FFF790FD42
:1010B0000823012229462046FFF717FE30BD30B530
:1010C00004460D46022229462046FFF781FD0823EB
:1010D000662229462046FFF708FE30BD30B504469B
:1010E0000D46022229462046FFF772FD082366229C
:1010F00029462046FFF7F9FD30BD30B504460D46C0
:10110000022229462046FFF763FD0823662229466E
:101110002046FFF7EAFD30BD30B504460D460022FB
:1011200029462046FFF754FD082301222946204680
:10113000FFF7DBFD30BD30B504460D460823012224
:1011400029462046FFF7D1FD012229462046FFF718
:101150003FFD30BD30B504460D4609230122294626
:101160002046FFF7C2FD012229462046FFF730FD49
:1011700030BD30B504460D46022229462046FFF711
:1011800027FD0823012229462046FFF7AEFD30BD8A
:1011900030B504460D46022229462046FFF718FDC9
:1011A0000923012229462046FFF79FFD30BD30B5B7
:1011B00004460D46022229462046FFF709FD082372
:1011C000012229462046FFF790FD30BD30B5044688
:1011D0000D46022229462046FFF7FAFC0823662224
:1011E00029462046FFF781FD30BD30B504460D4647
:1011F000022229462046FFF7EBFC0823012229465C
:101200002046FFF772FD30BD30B504460D46022280
:1012100029462046FFF7DCFC082301222946204608
:10122000FFF763FD30BD30B504460D460222294666
:101230002046FFF7CDFC0A23012229462046FFF76E
:1012400054FD30BD30B504460D46022229462046E5
:10125000FFF7BEFC0823012229462046FFF745FD83
:1012600030BD30B504460D46022229462046FFF720
:10127000AFFC0823012229462046FFF736FD30BD8A
:1012800030B504460D46022229462046FFF7A0FC51
:101290000823012229462046FFF727FD30BD30B53F
:1012A00004460D46022229462046FFF791FC0823FA
:1012B000012229462046FFF718FD30BD30B504460F
:1012C0000D46002229462046FFF782FC002301221A
:1012D00029462046FFF709FD30BD30B504460D46CE
:1012E000022229462046FFF773FC082301222946E3
:1012F0002046FFF7FAFC30BD30B504460D4600220B
:1013000029462046FFF764FC4FF402730122294668
:101310002046FFF7EAFC30BD30B504460D460022FA
:1013200029462046FFF754FC4FF4847301222946D6
:101330002046FFF7DAFC30BD0146D1F8480570477A
:1013400010B50146C1F307401F4BDB6E01248440FA
:10135000234033B1012303EB40031C4C54F823001A
:1013600003E04300194C54F82300C1F30722D0F8DE
:101370002C350F249440A34301F00F0494402343E1
:10138000C0F82C3510BDD0F834250A43C0F83425F8
:101390007047D0F834258A43C0F834257047D0F818
:1013A00030250A43C0F830257047D0F830258A43ED
:1013B000C0F830257047064AC0F82025D0F824250B
:1013C0000A43C0F82425704700E00F40146B010069
:1013D0004B434F4C30B50246E64B0624E6480068C6
:1013E000E64D2840E64DA84201D1E64B0A240021F3
:1013F00008E053F83100904203D103EBC10040688C
:1014000030BD491CA142F4DB0020F9E7016A41F03C
:1014100010010162704770B503460C461646184627
:10142000FFF7F4FF012E01D1D74A00E0D74A14207C
:1014300000FB0240401E02EB82018900B0FBF1F08C
:10144000451EDD60D3F8C00F00F0010048B1D04860
:101450002044401ECE49B0FBF1F0451E45F080000F
:10146000D86070BD016A41F0200101620121C0F81D
:101470000418704700B502460B461046FFF7F2FF0E
:10148000C2F8003800BD11B1012908D102E0C0F84E
:10149000002804E042F08003C0F81C3800BF00BF01
:1014A0007047016A21F01001016270470021C0F805
:1014B0000418016A21F020010162704770B50446EA
:1014C0000D462046FFF786FF06462946304600F0C7
:1014D00075F9304600F0CEF970BD70B5044620466F
:1014E000FFF778FF0546284600F000FA284600F08E
:1014F0007FF970BD01210161704702690A430261F1
:101500007047D0F80C1841F00101C0F80C18704772
:10151000D0F80C280A43C0F80C287047002101615C
:10152000704702698A4302617047D0F80C1821F0B5
:101530000101C0F80C187047D0F80C288A43C0F895
:101540000C287047024629B1906908B10120704704
:101550000020FCE7506908B10120F8E70020F6E719
:10156000024609B1906970475069FCE7024631B103
:10157000D2F8140808B1012070470020FCE7D2F827
:10158000100808B10120F7E70020F5E7024611B185
:10159000D2F814087047D2F81008FBE70121C161A6
:1015A00081617047C16170470121C0F81818704708
:1015B000C0F81818704742EA4103036070470146BB
:1015C000C86A70470146486800F0010008B1012070
:1015D00070470020FCE70146486800F0400008B171
:1015E000012070470020FCE74160704702465168C7
:1015F00001F0010008B10020704701F0120010B1A5
:1016000001F01C00F8E70020F6E781607047014612
:10161000886870474162704731B1D0F8202842F0A5
:101620000102C0F8202805E0D0F8202822F00102AD
:10163000C0F82028704731B1D0F8202822F00202EB
:10164000C0F8202805E0D0F8202842F00202C0F8B7
:10165000202870470146D1F804087047C0F80818E0
:1016600070470146D1F808087047D0F8042F6FF38F
:101670000F02C0F8042FD0F8042F0A43C0F8042F3B
:101680007047D0F8041F41F48041C0F8041F704730
:10169000D0F8042F92B2C0F8042FD0F8042F0A43D8
:1016A000C0F8042F7047D0F8041F41F08041C0F803
:1016B000041F70470146D1F8080F704700BFD0F8EB
:1016C000082F02F00202002AF9D1C0F8001F70476B
:1016D0000246D2F8080F00F0020008B1002070475F
:1016E000C2F8001F0120FAE7014600BFD1F8080F39
:1016F00000F480300028F9D1D1F8000F704702467D
:10170000D2F8080F00F4803008B100207047D2F8FA
:10171000000F08700120F9E7016370470146486B2C
:101720007047154A1268154B1A40154B9A4202D160
:10173000C2680A43C260104A1268104B1A40154B27
:101740009A4207D1826B42EA11328263026A42F006
:1017500040020262704741F00102C0F8042870475D
:101760000121C0F804187047016A41F001010162CB
:1017700070470000A46B010000E00F400000FF7004
:1017800000000A10D46B0100801A0600A086010038
:10179000804737010000051000BFFEE710B5FEF7D7
:1017A000BAFD08B1012010BD0020FCE710B5FEF71E
:1017B000ABFD08B1012010BD0020FCE730B50246AA
:1017C000B64C2468B64DAC420ED0B44C2368002011
:1017D00005E053F82040B24D45F82040401C9B28BE
:1017E000F7D3AF4CAD4D2C60AD4C44F8221030BD5A
:1017F000AC49AB4A42F820107047AB4951F8201071
:10180000AA4A1143A54A121D11607047A34A121D2E
:10181000126802F4E061002006E0A34A52F820209A
:101820008A4200D102E0401C0828F6D300BF70476E
:1018300010B50A4683089E4C54F823301968830774
:10184000DC0EFF23A34099438307DB0E02FA03F368
:1018500019438308964C54F82330196010BD014693
:101860008808934A52F8200000688A07D20ED040B8
:10187000C0B27047042808D188491C31096841F476
:101880008031864A1C3211602FE0052808D1834937
:101890001C31096841F40031804A1C32116024E097
:1018A000062808D17D491C31096841F480217B4A12
:1018B0001C32116019E00F2808D14FF0E0210969AE
:1018C00041F002014FF0E02211610EE010280CD32C
:1018D000A0F1100101F01F0201219140A0F11002BE
:1018E0005209744B53F8222011607047042808D124
:1018F0006A491C31096821F48031684A1C32116040
:101900002FE0052808D165491C31096821F4003110
:10191000624A1C32116024E0062808D15F491C315C
:10192000096821F480215D4A1C32116019E00F28FA
:1019300008D14FF0E021096921F002014FF0E022C7
:1019400011610EE010280CD3A0F1100101F01F026C
:1019500001219140A0F110025209574B53F8222067
:101960001160704710B501460020042905D14B4A8B
:101970001C32126802F4803028E0052905D1474A5C
:101980001C32126802F4003020E0062905D1434AD7
:101990001C32126802F4802018E00F2905D14FF0A4
:1019A000E022126902F0020010E010290ED3A1F12A
:1019B000100252093F4B53F822201268A1F1100384
:1019C00003F01F040123A34002EA030010BD022814
:1019D00008D13249091F096841F000412F4A121FFE
:1019E000116024E00E2808D12C49091F096841F034
:1019F00080512A4A121F116019E00F2808D1274987
:101A0000091F096841F08061244A121F11600EE02D
:101A100010280CD3A0F1100101F01F020121914008
:101A2000A0F110025209254B53F822201160704793
:101A30000E2808D11949091F096841F00061174AA9
:101A4000121F116019E00F2808D11449091F0968F5
:101A500041F00071114A121F11600EE010280CD3E2
:101A6000A0F1100101F01F0201219140A0F110022C
:101A70005209134B53F822201160704710B50446E9
:101A80002046FEF74EFC10BD10B5FEF74DFC10BD14
:101A9000A0F110010B4A11607047000008ED00E052
:101AA0000004002099170000246C01000000FA05D2
:101AB000446C0100E06C0100F46C0100086D010051
:101AC0001C6D010000EF00E030B50246744B0424A9
:101AD00074480068744D2840744DA84201D1744B7D
:101AE00000BF002108E053F83100904203D103EB1E
:101AF000C100406830BD491CA142F4D30020F9E781
:101B00002DE9F04F0C461D46DDE909C815B94FF027
:101B1000000A01E04FF0040A57464760B4FBFCF6A8
:101B2000002100BF891CB6FBF1FAAAF10103FF2BCB
:101B3000F8D801614FEA827A4FEA1A6902F030025E
:101B400049EA032A4AEA020AA8F1010B4AEA0B070A
:101B50000760BDE8F08F416841F0020141607047C5
:101B6000416821F002014160704770B504460D469E
:101B70002046FFF7A9FF064629463046FFF71EFE1E
:101B80003046FFF777FE70BD70B504462046FFF77C
:101B90009BFF05462846FFF7A9FE2846FFF728FECB
:101BA00070BD42690A434261704742698A4342619B
:101BB0007047024609B1D06970479069FCE701623D
:101BC000704700BFC26802F00202002AFAD08160AA
:101BD00070470246D06800F0020010B19160012009
:101BE00070470020FCE700BFC26802F00402002A30
:101BF000FAD082680A6070470246D06800F004009C
:101C000018B190680860012070470020FCE7426A24
:101C10000A4342627047426A8A4342627047014601
:101C2000C868C0F300107047C0F8C81F704701466D
:101C3000D1F8C80F7047426822F4E0720A4342604C
:101C4000704700BFC26802F00202002AFAD0426860
:101C500042F400624260816070470246D06800F042
:101C6000020030B1506840F4006050609160012083
:101C700070470020FCE7416841F480614160704793
:101C8000416821F4806141607047416841F0010181
:101C900041607047416821F00101416070470000D8
:101CA000306D010000E00F400000FF7000000A10DE
:101CB000506D0100024600210AE0F74850F831005B
:101CC000904204D3F44800EBC10040687047491CBF
:101CD0000629F2D30020F9E7F0B50146DFF8BCC3CE
:101CE000DCF860C1CCF38923DFF8B0C3DCF860C155
:101CF000CCF30905DFF8A4C3DCF864C1CCF3042CF1
:101D00000CF10106DFF894C3DCF864C10CF01F0C81
:101D10000CF10107B1FBF7F15A09A3EB421401FBE7
:101D200005F001FB02FC00EB5C1001FB04FC00EB86
:101D30009C20B0FBF6F0F0BDD8483C380068401C51
:101D400000027047D5480068D5490840D549884207
:101D500006D1D24880680004400900F50060704751
:101D6000CE484038006880B2401CC002F7E7CB483C
:101D70000068CB490840CC49884209D1C74840385F
:101D80000068C0F302400A30012101FA00F07047F8
:101D90004FF48060FBE70146C1F30720C34A1044BB
:101DA00000F0704040F00070C1F30722BF4B1A44AE
:101DB000C2F3130240EA4210CAB240EA820000684D
:101DC00008B1012070470020FCE70146C1F307205D
:101DD000B74A104400F0704040F00070C1F3072291
:101DE000B34B1A44C2F3130240EA4210CAB240EAAB
:101DF0008200006808B1012070470020FCE710B5A0
:101E00000121C0F30722AB4B1A4402F0704242F0AA
:101E10000072C0F30723A74C2344C3F3130342EA21
:101E20004312C3B242EA8302116010BD10B5002113
:101E3000C0F307229F4B1A4402F0704242F0007236
:101E4000C0F307239B4C2344C3F3130342EA43121A
:101E5000C3B242EA8302116010BD18B50121C0F37C
:101E60000722954B1A4402F0704242F00072C0F310
:101E70000723914C2344C3F3130342EA4312C3B232
:101E800042EA830211600021009102E00099491C9E
:101E9000009100991029F9D30021C0F30722864B45
:101EA0001A4402F0704242F00072C0F30723824CE1
:101EB0002344C3F3130342EA4312C3B242EA830248
:101EC000116018BD10B50121C0F307227B4B1A44E5
:101ED00002F0704242F00072C0F30723774C2344B3
:101EE000C3F3130342EA4312C3B242EA830211600E
:101EF00010BD10B50021C0F30722704B1A4402F048
:101F0000704242F00072C0F307236C4C2344C3F3C9
:101F1000130342EA4312C3B242EA8302116010BDC6
:101F200010B50121C0F30722654B1A4402F070423C
:101F300042F00072C0F30723614C2344C3F3130340
:101F400042EA4312C3B242EA8302116010BD10B5E7
:101F50000021C0F307225A4B1A4402F0704242F0AB
:101F60000072C0F30723564C2344C3F3130342EA21
:101F70004312C3B242EA8302116010BD10B50121C1
:101F8000C0F307224F4B1A4402F0704242F0007235
:101F9000C0F307234B4C2344C3F3130342EA431219
:101FA000C3B242EA8302116010BD10B50021C0F334
:101FB0000722444B1A4402F0704242F00072C0F310
:101FC0000723404C2344C3F3130342EA4312C3B232
:101FD00042EA8302116010BD30490968304A11405D
:101FE000304A91420ED130B12C49096E41F0006166
:101FF0002A4A116618E02949096E21F00061274A32
:10200000116611E040B12549B031096841F0005135
:10201000224AC2F8B01007E02049B031096821F027
:1020200000511E4AC2F8B010704710B50446214650
:102030002C20FFF7C3FB2C20FFF71CFC10BD10B5B4
:102040002C20FFF753FC2C20FFF7D2FB10BD1349C7
:10205000496D0143114A516570471049496D8143EB
:102060000E4A516570470D4988657047014611B1A8
:102070000A48806D70470948006DFBE71249086007
:1020800070471148006870470F4908310860704771
:102090000D480830006870478C6F010000E00F4069
:1020A0000000FF700000051000000A1000E30F4060
:1020B00000EA0F4000E90F4000E50F4000E60F4046
:1020C00000E70F4000E80F40B4E10F40FE49086010
:1020D0007047FD49091D08607047FC48FC490860CD
:1020E00000BFFEE710B5FEF71AF910BD10B5F848AD
:1020F000001D006840F00400F549091D0860FEF766
:102100000EF9F348001D006820F00400F049091D95
:10211000086010BDEF48C06D7047EE49C96D81433E
:10212000EC4AD1657047EB49C86770470146EA48F9
:10213000084050B101F00040E34A383A1060E648E8
:1021400081380840E34AC2F85001DF48383801605E
:1021500001F4007088B100BFDB483438006800F437
:1021600040700028F8D0D8483438006800F4407037
:10217000B0F5807F01D0002070470120FCE7D249F4
:10218000503108607047D0485030006870472DE9E2
:10219000FE4F05468A46CF480068D0490840D049DE
:1021A000884202D10020BDE8FE8FC5F3841705F0F8
:1021B0003800102805D1DFF82C93002600BF152722
:1021C00048E005F03800302804D147F230594FF488
:1021D00000163FE005F03800382804D14FF40049DC
:1021E0004FF4800636E005F0380078BB1A2F01DC8A
:1021F000092F01DA0020D6E7BB4850F827904FF4AA
:10220000401646F04076B348C06F20F01C000190A5
:10221000072F03DB019840F010000190AD490198B1
:10222000C8674FF40020009005E00098401E009021
:10223000009800B905E0A748006D00F48070002800
:10224000F3D000BF009828B90020ACE7FFE74FF0BB
:102250000009002605F46050002874D105F038000C
:1022600028B105F03800102801D000209BE7C5F305
:10227000026002909D48FFF71DFD9649C03108603D
:102280009448D0F8B0009A4900EA010444F00044B0
:102290009048B0300460093F9649029851F82000F8
:1022A0005044401EB0FBFAF88A48D0F8B0003043E2
:1022B0008849B0310860029800EBC00000EB400094
:1022C0008D4901EBC00007EB470100EB810040683E
:1022D0008049C1F864017C4824380168A8F10100F4
:1022E00041EA00207B49C1F86401029800EBC0007C
:1022F00000EB4000804901EBC00007EB470150F8BC
:10230000210071492839096801F4000108436E4928
:10231000283908604846FFF7DFFC4FEA500A50466C
:10232000FFF7C8FC6B49C1F8C0000846D0F860014F
:1023300000F4000040B16748B030006840F08040D1
:10234000C1F8B00008E02BE05F482838006840F48E
:1023500000006049C1F860014FF4004B08E05A48A2
:102360002038006800F0010000B104E0ABF1010B7F
:10237000BBF1000FF3DC00BFBBF1000F0DD05548DF
:10238000B030046846F0010040F08050044344F04F
:1023900000445048C0F8B0403CE04FF0000A39E03B
:1023A0005048FFF787FC4B49C03108604948D0F8D6
:1023B000600120F400004749C1F860010846D0F8E8
:1023C000B0404E48044044F000444248B0300460FD
:1023D000BAF1000F02D14FF000080AE0B9FBFAF899
:1023E000B8F1000F01D0A8F1010808F10100B9FB14
:1023F000F0FA5046FFF75EFC3649C03108603548B8
:10240000D0F8B04046EA8820044344F00044314804
:10241000B03004602F48B030006820F470002D49BF
:10242000C1F8B0005046BEE62DE9F0410646294805
:10243000046E056F44F4006424F4800445F40065E0
:102440000466056704F00100D8B106F00100C0B9C8
:1024500066F0010004404FF480701E49886508460C
:1024600004664FF4002702E07F1E07B905E0194813
:10247000006D00F480700028F6D000BF0FB9BDE8F1
:10248000F08124F4FE6406F4FE6004431C48054019
:102490001B49A13106EA0100054306F0080045EAA0
:1024A000C0050C480466056724F4005406F4005087
:1024B000044325F4005506F4005005434020054927
:1024C000886505F000401DE088E10F400400FA0532
:1024D0000CED00E000E00F40000100800000FF7004
:1024E000000005100024F400706D010040787D01AB
:1024F00000FC0FE0BC6F0100DC6D0100FF0300EF8A
:102500008FFFFF7F18B108460567046602E0D648D2
:1025100004660567D5480440C14306EA0100044348
:1025200025F0FC5506F0FC50054306F0804040B114
:1025300044F4800425F48005CD4906EA01000543F2
:1025400001E025F0804506F4006080B94FF40047B3
:1025500006E0C848006800F0010000B102E07F1EFC
:10256000002FF6D100BF24F4006425F40065BE48B6
:10257000046605671020FDF7DBFE00BF7FE7F0B5BE
:10258000B948036E026F02F0004010B102F0700013
:1025900001E003F03000202811D003DC38B110280E
:1025A00015D10AE030280CD0702810D10CE0B248C8
:1025B000C3F3841750F827100BE0B04909E0B04985
:1025C00007E047F2305104E04FF4004101E0002001
:1025D000F0BD00BF4FF0FF3402F0004010B102F434
:1025E000006028B102F0004098BB03F4006080BB9B
:1025F000A048083805689C48D0F8646106F01F00C0
:10260000401CC6F304277F1C10FB07F04000B1FB01
:10261000F0F1C5F309004843C5F389274F4300EBA8
:10262000972143F480039048006900F47040B0F5AE
:10263000804F13D006DCB0F5005F0BD0B0F5405FE3
:1026400012D109E0B0F5E04F0AD0B0F5104F0BD130
:1026500008E00BE08B4C08E08B4C06E08B4C04E070
:102660008B4C02E08B4C00E000BF00BF03F4800005
:1026700018B302F00040D8B102F0804090B102F0EF
:10268000004010B102F4006028B102F0004048B9E7
:1026900003F4006030B94F00C2F38650401CB7FB12
:1026A000F0F10AE0C2F3C550401CB1FBF0F104E0C8
:1026B000C3F3C350401CB1FBF0F18C4200D2214661
:1026C000084685E76B4924390860704710B5024613
:1026D000654B1B68704C2340704CA34208D121F01D
:1026E000FC54531E44EAC353624C243C236023E051
:1026F000501E01F0700333B1102B0ED0302B05D0DB
:10270000702B09D105E040F4401007E040F40010C0
:1027100004E040F4800001E000BF00BF00BF01F012
:1027200002030BB140F0004001F080430BB140F0D8
:102730008040504B243B186010BD4B49096E21F47A
:10274000F0110143484A116670474748006E00F493
:10275000801008B9002070474348006E00F4F01064
:10276000F9E74149C96E00F00F0301229A40114375
:102770003D4AD16670473C49C96E00F00F03012203
:102780009A409143384AD16670473748006F20F429
:1027900080403549086770473348006F40F48040F7
:1027A0003149086770473049886370472E48006E8A
:1027B00070472D49096E01432B4A116670472DE978
:1027C000F04F054628480068DFF8CCE000EA0E002C
:1027D000DFF8C8E0704503D100200860BDE8F08F45
:1027E0002148B030076807F08050B0F1805F02D018
:1027F00000200860F2E7C5F384161F4850F8264011
:102800001C48083802681848D0F86431C2F3090C33
:10281000C2F3892803F01F09C3F3042A04FB0CF058
:1028200004FB08FE00EB9E2B09F101000AF1010EEA
:1028300010FB0EF0BBFBF0FBC1F800B00120CDE7B0
:102840000948406E70470849496E8143064A5166FF
:1028500070474A1ED2B20243064B203B1A607047B3
:10286000044930390860704700E00F40FEFF3FF830
:102870000000404068E10F40706D01000024F4004A
:1028800000093D0000B4C40480F0FA02005A62025C
:1028900040787D01002D31010000FF70000005101F
:1028A000F0B503460C46C24D0C26C2480068C24F24
:1028B0003840C24FB84201D1C14D082600210DE079
:1028C00055F83100984208D105EBC1004268B4F5D3
:1028D0007F4F00D1521C1046F0BD491CB142EFD3CE
:1028E0000020F9E7C26840F201130B401A43C260AE
:1028F0007047C26840F201130B409A43C2607047B0
:10290000C26840F201139A43C2600A0E0260A94AEB
:102910001268A94B1A40A94B9A4211D1CAB201F4CC
:10292000702342EA131242F40072426001F4700212
:10293000C1F3072343EA122242F40072826008E0E6
:10294000CAB242F400724260C1F3072242F400723C
:102950008260704744F24003194012B1C3680B43D0
:1029600001E0C3688B43C360704710B5914B1B688F
:10297000914C2340914CA3420AD140F201130B40E9
:1029800012B1046F1C4301E0046F9C43046700BF55
:1029900042F22003194012B1C3680B4301E0C3683F
:1029A0008B43C36010BD10B540F60C431940C3689B
:1029B0008B4302EA01042343C36010BD40F20223AB
:1029C000194012B1C3680B4301E0C3688B43C36075
:1029D0007047CBB24BB122B1436843F04003436030
:1029E00003E0436823F04003436001F47F434BB1AD
:1029F00022B1836843F04003836003E0836823F0DF
:102A0000400383607047C16841F01001C1607047A6
:102A1000C16821F01001C1607047C0F8C81F70473D
:102A20000146D1F8C80F7047CBB203B1826301F4FD
:102A30007F4303B1C26370470246FF2901D1906B07
:102A40007047D06BFCE7CBB203B1026401F47F4363
:102A500003B1426470470246FF2901D1106C7047F0
:102A6000506CFCE7CBB203B1826201F47F4303B147
:102A7000C26270470246FF2901D1906A7047D06A4E
:102A8000FCE7C3628262704730B5034600BFDA6A72
:102A90009C6ADD6AAA42FAD1002001462043114314
:102AA00030BD0246FF2901D1906C7047D06CFCE725
:102AB00030B5034600BFDA6C9C6CDD6CAA42FAD1DB
:102AC000002001462043114330BDCBB203B1026365
:102AD00001F47F4303B1426370470246FF2901D1ED
:102AE000106B7047506BFCE743630263704730B56F
:102AF000034600BF5A6B1C6B5D6BAA42FAD10020E3
:102B000001462043114330BD2DE9F04105460E46F4
:102B1000144631462846FFF7C3FE0746214638468D
:102B2000FEF74CFE3846FEF7A5FEBDE8F08170B515
:102B300004460D4629462046FFF7B2FE06463046BB
:102B4000FEF7D4FE3046FEF753FE70BD82690A439D
:102B50008261704782698A4382617047024609B187
:102B6000106A7047D069FCE74162704701617047A5
:102B7000016770470146086F7047C166704701469C
:102B8000C86E704710B50B46DCB2FF2C04D1446808
:102B900024F4A0611143416003F47F44B4F57F4FF6
:102BA00004D1846824F4A0611143816010BD000049
:102BB000C46F010000E00F400000FF7000000A1029
:102BC0002470010030B50246C74B0824C74800688E
:102BD000C74D2840C74DA84201D1C74B00BF0021B7
:102BE00008E053F83100904203D103EBC100406884
:102BF00030BD491CA142F4D30020F9E7C26A22F09B
:102C000086020A43C26270470146C86A00F0860025
:102C1000704741EA02034363704710B5436B03F00A
:102C200007040C6003F03804146010BDC16A41F061
:102C30001001C162016B40F2013211430163704720
:102C400000BF816901F008010029FAD1C16A21F0B1
:102C50001001C162016B40F2013291430163704780
:102C6000F0B504460E4615461F462046FFF7E8FF1E
:102C7000B6EB051F05D2206B40F0200020636D08E5
:102C800003E0206B20F020002063F000B0FBF5F0A3
:102C9000401C43089809606203F03F00A062E762AD
:102CA0000020A0612046FFF7C1FFF0BDF0B5446AE7
:102CB000856A8E00402707FB0457B6FBF7F61660BF
:102CC000066B06F0200616B1166876001660C66A16
:102CD00006F0EE061E60F0BDC16A41F01001C1624F
:102CE0007047C16A21F01001C162704721B1026BC7
:102CF00042F00602026303E0026B42F0020202634A
:102D00007047016B21F0060101637047C16A21F031
:102D1000E60141F06E01C162026B42F008020263FB
:102D20007047016B21F0080101637047026B01F4E9
:102D300040631A4302637047026B01F440639A4395
:102D4000026370470146086B00F44060704701461B
:102D5000886940F2071210407047026B22F440422B
:102D60000A43026370470146086B00F44040704715
:102D7000026B22F010020A43026370470146086B9F
:102D800000F01000704701468869012222EA101005
:102D9000704701468869012222EA501070470146B7
:102DA000886900F0100008B9086870474FF0FF30DC
:102DB000FBE7014600BF886900F010000028FAD147
:102DC000086870470246906900F0200010B9116051
:102DD000012070470020FCE700BF826902F020025A
:102DE000002AFAD10160704719B1C26A42F00102AB
:102DF00002E0C26A22F00102C2627047014688699D
:102E0000C0F3C000704770B504460D462046FFF77A
:102E1000D9FE064629463046FEF7D0FC3046FEF77E
:102E200029FD70BD70B504462046FFF7CBFE054670
:102E30002846FEF75BFD2846FEF7DAFC70BD826B84
:102E40000A4382637047826B8A43826370470246FB
:102E500009B1106C7047D06BFCE741647047826C1D
:102E60000A4382647047826C8A43826470470146D9
:102E7000486800F00F007047002141607047C0F8BB
:102E8000C81F70470146D1F8C80F7047D0F8A4108A
:102E900041F40041C0F8A4107047D0F8A41021F408
:102EA0000041C0F8A4107047C0F8A410C0F8A820D2
:102EB00070470A4600BF836903F08803802BFAD16C
:102EC000C16A21F0040343F08203C362026000BFC1
:102ED000836903F08803802BFAD1C1627047016BCC
:102EE00041F08001016370476470010000E00F4011
:102EF0000000FF7000000A10A470010001468868FD
:102F000000F001007047816841F001018160704765
:102F1000816841F0020181607047816821F00201FF
:102F2000816070470121C0F8001C70472449C0F837
:102F3000001C70470146D1F8000C012800D17047F1
:102F40000020FCE7016070470146086870470146B1
:102F50004868704770B505460C4621462220FEF7AA
:102F60002DFC2220FEF786FC70BD10B50446222001
:102F7000FEF7BCFC2220FEF73BFC10BD816841F04F
:102F8000010181607047024609B1506970471069BC
:102F9000FCE70121C1607047826822F004020A4305
:102FA00082607047D0F8181441F48071C0F818148A
:102FB0007047D0F8181421F48071C0F818147047C5
:102FC00051E5CC1AEFF3098141B1F1EE101A40F846
:102FD000041D20ED200A29490A6810607047B0ECF2
:102FE000200A02C8E1EE101A25490A6810607047ED
:102FF000EFF3108072B6704780F310887047214855
:103000004FF0FF010170002080F309881E4801681D
:1030100081F308881D48012101701D484FF080513F
:10302000016062B6FEE71A484FF0805101607047B8
:1030300017484FF080510160704772B6EFF3098076
:1030400028B1203880E8F00F0C490968086000B505
:10305000104880475DF804EB0F4810490A78027069
:10306000064807490A680260106890E8F00F2030AF
:1030700080F309884EF0F40E62B670473C000020E1
:103080004400002022ED00E008000020360000206F
:1030900004ED00E0BB3200002B0000202C000020DB
:1030A000A648802102E0491E002204C00029FAD16E
:1030B000A34AA44B1A601A46126822F007021A604B
:1030C0000022A14B1A807047704710B50446204675
:1030D00012F0F0FC10BD10B50446204612F0EBFCD7
:1030E00010BD10B512F0E8FC10BD10B50446204626
:1030F00012F0E4FC10BD10B512F0DFFC10BD70B58D
:103100000446101D20F007004FF08076051F28466A
:103110002E60051F28462C608C4E051F28462E6009
:103120004FF01236051F28462E604FF00336051F5C
:1031300028462E604FF00236051F28462E60761076
:10314000051F28462E60051F284629604FF01136BE
:10315000051F28462E604FF01036051F28462E60AA
:103160004FF00936051F28462E604FF00836051F20
:1031700028462E604FF00736051F28462E604FF078
:103180000636051F28462E604FF00536051F2846D7
:103190002E604FF00436051F28462E6003F004050C
:1031A000002D7DD0F605051F28462E60684E051FB0
:1031B00028462E60674E051F28462E60664E051F66
:1031C00028462E60654E051F28462E60644E051F5A
:1031D00028462E60634E051F28462E60624E051F4E
:1031E00028462E60614E051F28462E60604E051F42
:1031F00028462E605F4E051F28462E605E4E051F36
:1032000028462E605D4E051F28462E605C4E051F29
:1032100028462E605B4E051F28462E605A4E051F1D
:1032200028462E604FF08346051F28462E60574ED5
:10323000051F28462E60564E051F28462E60554E07
:10324000051F28462E60544E051F28462E60534EFB
:10325000051F28462E60524E051F28462E60514EEF
:10326000051F28462E604FF08246051F28462E6017
:103270004D4E051F28462E604C4E051F28462E60D9
:103280004B4E051F28462E604FF08146051F2846ED
:103290002E60484E051F28462E603602051F00E0AE
:1032A0000AE028462E604FF07E56051F28462E6005
:1032B0000026051F28462E6070BD10B512F0FFFBDA
:1032C00010BD10B50446204612F0FAFB10BD10B533
:1032D00012F0F7FB1C480088401C1B490880084678
:1032E000008818B10020088003F0E0F810BD10B588
:1032F000FFF77EFE044630480078401C2E490870D7
:103300002046FFF779FE00F0CDFD00F0CFFC10BDA8
:1033100001464A1E4FF0E0235A61284A106820F007
:103320007F4000BF10601A46126942F005021A6120
:103330001A46126942F002021A6170476C060020B8
:103340006C080020080000200C000020195E00001E
:103350000000F8410000F0410000E8410000E041B9
:103360000000D8410000D0410000C8410000C04129
:103370000000B8410000B0410000A8410000A04199
:103380000000984100009041000088410000704119
:103390000000604100005041000040410000304109
:1033A00000002041000010410000E0400000C0404B
:1033B0000000A040000040402900002020ED00E077
:1033C0001D481E481E481F481F48204820482148C5
:1033D0002148224822482348234824482448254895
:1033E0002548264826482748274828482848294865
:1033F00029482A482A482B482B482C482C482D4835
:103400002D482E482E482F482F4830483048314804
:1034100031483248324833483348344834483548D4
:1034200035483648364837483748384838483948A4
:10343000394800BF70470000E4700100E8700100E7
:10344000EE700100F0700100EC700100F2700100FC
:10345000F4700100F6700100F8700100FA700100CC
:10346000FC700100FE70010000710100027101009A
:103470000471010006710100087101000A71010068
:103480000C7101000E710100107101001271010038
:103490001471010016710100187101001A71010008
:1034A0001C7101001E7101002071010022710100D8
:1034B0002471010026710100287101002A710100A8
:1034C0002C7101002E710100307101003271010078
:1034D00034710100367101003A7101003C71010044
:1034E0003E71010040710100B4270020342C0020FF
:1034F0004471010046710100487101004A710100E8
:103500004C7101004E7101005071010052710100B7
:103510005471010042710100567101000146002002
:1035200002E0491C421CD0B20A78002AF9D1704747
:103530002DE9F04105460E4614460027FB48007869
:1035400020B1112020700020BDE8F08128780128EA
:1035500008D0022807D0032802D0042804D100E0B4
:1035600000BF00BF00BF03E0012020700020EBE798
:1035700000BFFFF73DFD0746686930603068FFF720
:10358000CDFF80463846FFF737FD002020704046CB
:10359000DAE72DE9F04105460E4614460027E348D8
:1035A000007818B112202070BDE8F0812878012839
:1035B00008D0022807D0032802D0042804D100E054
:1035C00000BF00BF00BF02E001202070ECE700BF99
:1035D000FFF70EFD07466E613846FFF70DFD002030
:1035E000207000BFE0E7F0B5024612F8384F95783A
:1035F0005678383A0B4618680FE000F10B073F5D2C
:10360000B74300F10B0C0CF8047067463F5D17B927
:10361000877AAF4387721B1D18680028EDD1F0BD73
:10362000C349C44A1278885CC349095CC04A515CEA
:1036300001EBC001C14A1170704710B50024FFF7BB
:10364000D7FC0446B9480078F8B9BD480078E0B91D
:10365000FFF7E6FFBB48B949097850F82100BA499D
:103660000860B6480078B949097888420DD0B64854
:103670000068C06B401CB4490968C863B44800685E
:10368000401CB3490860FFF7CEFC2046FFF7B4FCAE
:1036900010BD70B501460024AE4D2D68EC61AD4CF7
:1036A000246821620B4618681BE0AA4C246894F831
:1036B000385000F10B04645DA64D2D6895F8395023
:1036C0002C43A44D2D6895F8386000F10B05AC55DE
:1036D000847AA04D2D6895F83A502C4384721B1DB6
:1036E00018680028E1D19B4C246894F83820924C4B
:1036F000A45C984D2D6895F83950AC438E4DAC5470
:103700002C46A45C44B9934C246894F83A50894CF4
:103710002478AC43874D2C7070BD2DE9FF4F83B0EA
:1037200081460E461546DDF840800020009030604E
:10373000CA46DAF8004018E02078062807D2DFE809
:1037400000F00604050307080AE009E008E000BFEE
:1037500000BF012088F80000002007B0BDE8F08F0E
:1037600000BF0AF1040ADAF80040002CE4D16F48E7
:10377000007820B1022088F800000020EDE77048B2
:10378000007820B10D2088F800000020E5E7002037
:10379000029001908346CA46DAF80040FFF728FC01
:1037A000009057E02078062843D2DFE800F0421569
:1037B00026034344208960B12089401E208110C621
:1037C00001200290002001C50198401C80B20190A8
:1037D00001E04BF0010B38E0606858B1606801C54A
:1037E0000020606010C6012002900198401C80B249
:1037F000019001E04BF0020B27E06768F88AA8B15E
:103800003969081D3861086801C5B9683869884296
:1038100001D178683861F88A401EF88210C601200C
:1038200002900198401C80B2019001E04BF0040B23
:103830000BE000BF00BF0098FFF7DEFB0020306008
:10384000012088F80000019887E700BF0AF1040A08
:10385000DAF80040002CA5D10298012809D10020F7
:1038600030600098FFF7C8FB002088F8000001983E
:1038700073E73848006890F834004BF08001084343
:103880003449096881F8340000203249096881F818
:10389000350030490698096808634846FFF7F9FE85
:1038A0000098FFF7A9FBFFF7C8FEFFF7A1FB009008
:1038B0002848006890F8350020B1012819D0022866
:1038C00016D100E000BF23480068C4692CB110C6BF
:1038D000002030600120019009E001201D490968A5
:1038E00081F8350049461B480068FFF77CFE06E07A
:1038F00000BF494617480068FFF775FE00BF00BFCC
:103900001448006890F8350020B1012842D0022800
:103910003FD138E02078062824D2DFE800F0231DCC
:103920001E032425002001C528E0000029000020F6
:10393000587101002D0000202E0000202C000020D6
:103940002A000020F4120020440000202B00002058
:10395000100000203C00002000BFFD480068406AC5
:1039600001C50BE000BF00BF0098FFF745FB00203A
:103970003060012088F800000198EEE600BF0020CA
:1039800088F800000CE0002001C50E2088F8000037
:1039900006E000BF002001C50A2088F8000000BF33
:1039A00000BF0020EA49096881F83400E849096845
:1039B00081F83500E6490968C861E5490968086287
:1039C000E349096848620098FFF716FB0198C4E6CE
:1039D0007CB5002514E06946284602F00EF906463B
:1039E00066B9DC4850F8254044B1012C06D0D4E932
:1039F000020100EB8100A0640198E064681CC5B27C
:103A00003F2DE8D97CBD00BF00BF02E0C82002F016
:103A10001BFAD14800780028F8D0D048006864210B
:103A2000B0FBF1F0CD4908600846006828B90020D5
:103A3000CB490870FF2002F020F9FFF7D9FA0446BD
:103A4000C648006864214843C64908602046FFF71D
:103A5000D3FA00BFFFF7CCFA0446C2480068C24957
:103A600008600020BF4908602046FFF7C5FABE483D
:103A70000068BA490968B0FBF1F0C0F16400B849C8
:103A80000870FFF738FBFFF7A3FF642002F0DCF9B2
:103A9000E0E700B587B0032000218022B34BCDE9D9
:103AA0000132CDE903104FF6FE703E23B04A00907C
:103AB000AFF2AD0001F0B3FE06AAAEA13E2002F0C7
:103AC0001EF807B000BD002400BF00BFFFF790FA4A
:103AD0000446A4480068401CA24908602046FFF73D
:103AE0008BFAFFF7FEFAF1E700B587B0032000215B
:103AF0008022A44BCDE90132CDE903104FF6FF70CF
:103B00003F23A14A0090AFF2410001F088FE06AACF
:103B10009EA13F2001F0F3FF07B000BD04E00022AA
:103B200000F8012B4A1E91B20029F8D1704770B5F8
:103B30004FF4BD619948FFF7F1FF002411E0601CCC
:103B400085B204EB4400954901EBC00305EB450049
:103B500001EBC006002018705E6091A05861601CE7
:103B600084B23E2CEBD304EB44008C4901EBC00340
:103B70000020187058608AA058610846894908607A
:103B800070BD70B54FF48F518748FFF7C7FF4FF4F2
:103B900080717048FFF7C2FF002413E0601CC5B2BB
:103BA00004EB440000EBC4007F4901EBC00305EBCC
:103BB000450000EBC50001EBC0065E6178A018650A
:103BC000601CC4B2332CE9D304EB440000EBC40006
:103BD000754901EBC0030020586171A018650020F1
:103BE0007249086070487249086070BD0021714ACE
:103BF0001170002004E000216F4A1154411CC8B22A
:103C00000828F8D300216D4A11706D4A11706D4A71
:103C100011604F4A1160704700206B4908606B4982
:103C200008706B4908706B4908706B4908706B49E4
:103C300008604C4908604C4908604849086046499A
:103C4000087067490870704710B5FFF729FAFFF749
:103C5000E3FFFFF7CBFFFFF794FFFFF768FF00F0EC
:103C6000CFFE00F0C0FF01F0C2FAFFF73DFFFFF703
:103C700010FF02F075FCFFF727FAFFF7A1FB10BD5C
:103C800010B50024FFF7B4F9044653480078012822
:103C900008D14E480078FF2804D24C480078401CD8
:103CA0004A4908702046FFF7A7F910BD10B5002457
:103CB00049480078012830D1FFF79AF90446434873
:103CC000007820B141480078401E404908703F48C4
:103CD0000078F8B93E480078E0B9FFF7A1FC1D482C
:103CE0003749097850F8210036490860344800788F
:103CF0003249097888420DD032480068C06B401CB8
:103D000030490968C86335480068401C3349086079
:103D1000FFF78EF92046FFF76FF910BD10B50024AC
:103D20002D480078012811D1FFF762F90446274891
:103D3000007840B926480078FF2804D2244800784B
:103D4000401C234908702046FFF756F910BD0000BB
:103D50003C000020F4120020280000202000002059
:103D60001C0000203800002024000020F40E002059
:103D7000F010002075432F4F532D49492053746193
:103D800074000000F4100020F012002075432F4F43
:103D9000532D49492049646C650000006C080020DF
:103DA0003F00000014000020F41300204800002011
:103DB000400000202D0000202E0000202B000020BD
:103DC0002C000020440000205C000020290000207E
:103DD0002A000020370000203600002010000020BC
:103DE0005800002010B50024FD480078012821D19A
:103DF000FFF7FEF80446FB480078C0B9FA4800789F
:103E000088B1F9480078401EF749087008460078E4
:103E100028B92046FFF7F0F8FFF70FFC0AE020462C
:103E2000FFF7EAF806E02046FFF7E6F802E0204652
:103E3000FFF7E2F810BD10B5E948007890B9FFF738
:103E4000EFFBEA480078EA490870EA48E749097850
:103E500050F82100E849086008460068E749086012
:103E6000FFF7CDF810BD10B50024022001F0ECFFE3
:103E7000FFF7BEF804460020E14908602046FFF73E
:103E8000BBF8642001F0E0FFFFF7B2F80446DC481D
:103E90000068DC4908600120DB4908702046FFF714
:103EA000ABF810BD70B50026FFF711FAFFF7A0F8C8
:103EB0000646D6480068401CD44908603046FFF7E3
:103EC0009BF8C7480078012853D1D148007820B129
:103ED000012804D0022809D103E001250BE00025C8
:103EE00009E001250120CA49087004E001250020ED
:103EF000C749087000BF00BF05B970BDC548046858
:103F000033E0FFF775F80646206B50B3206B401E78
:103F10002063206B28BB94F8340000F0370040B1D8
:103F200014F8340F00F0C800207001206070343C99
:103F300002E0002084F8350094F8340000F0080016
:103F400078B93834A078B44909780843B249087080
:103F50002078B249085C6178084314F83819AF4AF0
:103F6000505464693046FFF747F894F836003F280C
:103F7000C7D100BFC1E747F21A207047704710B59C
:103F800090F8382001F10B039B5C90F83940A34373
:103F900001F10B04A35423469B5C23B98B7A90F860
:103FA0003A40A3438B720023C36110BD2DE9F04F4B
:103FB00005460F4690469946A87A99490E5C05F148
:103FC0000B00805D11F800B00BEBC60000F0FF0A9B
:103FD000884850F82A4000202434E0602760207C84
:103FE00020EA0800207484F81190207C243C00F022
:103FF000080068B994F83A00874909780843864967
:1040000008708648805D94F83910084383498855C4
:1040100029462046FFF7B3FF206A20B12046216AD7
:10402000FFF7E1FAE5615046BDE8F08F10B5734A3D
:104030001268D061714A126892F8383000F10B02B0
:10404000D25C6E4B1B6893F839301A436B4B1B687C
:1040500093F8384000F10B031A55827A674B1B68BE
:1040600093F83A301A438272644A126892F8381010
:104070006A4A525C614B1B6893F839309A43674B2C
:104080005A541A46525C42B95C4A126892F83A3065
:10409000614A12789A43604B1A7010BD01460022A3
:1040A0008A72002005E0002301F10B021354421C28
:1040B000D0B20828F7D3704705E011F8013B00F8AB
:1040C000013B531E9AB2002AF7D170472DE9F84FF1
:1040D00005460F4690469946DDE90AAB0020009060
:1040E000FEF786FF00904F480468002C77D01C3400
:1040F00054F8080C4B4908600098FEF77DFF44F81F
:104100001C7CA576002020766076606144F818BC9F
:1041100044F810AC44F8148C0C9824F80C0C24F8D7
:104120000A9C0020E077E810207705F00700E07691
:10413000217F01208840A077E17E012088406077C0
:10414000002020606060E060A0602062A062606289
:10415000E0622063AFF2B83060631C3C002606E0EA
:10416000002104F1540040F82610701CC6B2002E45
:10417000F6D02046FFF7A5F8FEF73AFF00901D485D
:1041800040F825400098FEF737FF2046FEF79DFFD8
:10419000FEF72EFF00901F48006860610020A061BC
:1041A0001C48006810B11B4800688461194804600D
:1041B0003834A078184909780843174908702078DE
:1041C0001649085C6178084314F83819134A5054AA
:1041D00015480078401C14490870009826E02AE031
:1041E00036000020290000202A0000202C0000209A
:1041F0002B000020F4120020440000203C0000208E
:104200003800002020000020280000205C00002052
:104210004C000020480000202D0000202E0000202F
:10422000587101004000002037000020FEF7E4FE36
:104230000020BDE8F88F0098FEF7DEFE4220F8E788
:104240002DE9F05F04460F4691461E464FF0000BE5
:104250002078052804D0012030700020BDE8F09FB0
:1042600009F0800ABAF1000F04D029F080094FF05C
:10427000010801E04FF0000800203070FEF7B8FEA2
:104280008346B9F1000F2CD0B9F1010F3BD0B9F141
:10429000020F03D0B9F1030F46D111E0208900EAE3
:1042A0000705BD4206D1B8F1010F05D12089A84309
:1042B000208101E0702030705846FEF79DFE3AE004
:1042C000208900EA070535B1B8F1010F05D1208931
:1042D000A843208101E0702030705846FEF78CFE24
:1042E00029E0208927EA0005BD4206D1B8F1010F77
:1042F00005D120892843208101E070203070584684
:10430000FEF77AFE17E0208927EA000535B1B8F1FB
:10431000010F05D120892843208101E070203070F1
:104320005846FEF769FE06E05846FEF765FE002592
:104330006F20307000BF00BF28468FE72DE9F041A5
:1043400006460D460027FC48007820B11020287052
:104350000020BDE8F081FEF74BFE0746F7480468F1
:1043600084B100684068F549086005202070268106
:1043700000206060F2A0E0603846FEF73DFE0020BD
:10438000287004E03846FEF737FE72202870204679
:10439000DFE730B501464A6808682AB9CC68606032
:1043A00028B10025456002E0106000B142608B68D2
:1043B00000259D6230BD2DE9F0410646884617462E
:1043C000B468002044F8300F24F8048C207900F001
:1043D000DF00207167712079303C88B93834A078CB
:1043E000D84909780843D74908702078D649085C2D
:1043F0006178084314F83819D34A5054012500E075
:1044000000253046FFF7C5FF2846BDE8F0812DE9BD
:10441000F0470446894615464FF0000AC648007822
:1044200020B10F2028702046BDE8F08720780528AD
:1044300003D0012028702046F6E7FEF7D9FD82461A
:10444000606808B1012700E00027B9F1000F03D030
:10445000B9F1010F3DD119E08FB9B9A0E06000209A
:104460002070B6480068606000202081B348046076
:104470005046FEF7C1FD00202870002605E050469A
:10448000FEF7BAFD49202870264629E0D4F80480BA
:1044900006E0022200214046FFF78DFFD8F8008099
:1044A000B8F1000FF5D1A6A0E06000202070A3486D
:1044B0000068606000202081A04804605046FEF73C
:1044C0009BFD012F01D1FFF7B8F8002028700026CE
:1044D00006E05046FEF790FD07202870264600BFF4
:1044E00000BF3046A0E72DE9F04105460E461446D0
:1044F00000279148007820B1112020700020BDE8ED
:10450000F081FEF775FD07462878052806D0384665
:10451000FEF772FD012020700020F0E7E8683060AF
:104520003068FEF7FBFF80463846FEF765FD002049
:1045300020704046E3E72DE9F04105460E4614465B
:1045400000277D48007818B112202070BDE8F08166
:10455000FEF74EFD07462878052805D03846FEF7B9
:104560004BFD01202070F1E7EE603846FEF744FD78
:104570000020207000BFE9E7F0B51446059E734F98
:104580003F6897F8347047F02007DFF8C0C1DCF8C7
:1045900000C08CF834700027DFF8B0C1DCF800C030
:1045A0008CF83570694F3F683E63684F3F68B96269
:1045B0000C828B74654F3F688F6047680F600027DF
:1045C0004F60C860456805B1696041605F4F3F68F2
:1045D00097F838205C4FBF5CDFF870C1DCF800C092
:1045E0009CF839C027EA0C07DFF85CC10CF80270B0
:1045F0006746BF5C5FB9554F3F6897F83AC0514F67
:104600003F7827EA0C07DFF83CC18CF80070F0BD5A
:104610002DE9F04F89B005460F4691469A46129E05
:10462000002002904448007828B102203070002019
:1046300009B0BDE8F08F4648007818B10D20307001
:104640000020F5E72878052803D0012030700020ED
:10465000EEE709F0800BBBF1000F04D009F07F09F1
:104660004FF0010801E04FF00008FEF7C1FC029096
:10467000B9F1000F4AD0B9F1010F78D0B9F1020FAA
:1046800003D0B9F1030F71D120E0288900EA0704B3
:10469000BC420FD1B8F1010F02D12889A043288173
:1046A0002A48006884850298FEF7A6FC0020307036
:1046B0002046BDE74B463A4604A92846CDF800A05F
:1046C000FFF75AFF0298FEF797FC78E0288900EA86
:1046D00007047CB1B8F1010F02D12889A0432881D9
:1046E0001A48006884850298FEF786FC0020307026
:1046F00020469DE74B463A4604A92846CDF800A03F
:10470000FFF73AFF0298FEF777FC58E0288927EA7E
:104710000004BC421ED1B8F1010F02D12889204308
:1047200028810A48006884850298FEF765FC00200D
:10473000307020467CE71AE0290000201800002095
:104740003F0000002D0000202E0000203C00002033
:104750002A0000204B463A4604A92846CDF800A07E
:10476000FFF70AFF0298FEF747FC28E01FE02889C0
:1047700027EA00047CB1B8F1010F02D12889204357
:104780002881B348006884850298FEF735FC002034
:10479000307020464CE74B463A4604A92846CDF8EF
:1047A00000A0FFF7E9FE0298FEF726FC07E002985A
:1047B000FEF722FC00246F203070204638E700BF4F
:1047C000FEF73BFFFEF714FC0290A148006890F84A
:1047D000350020B39E48006890F835000390002013
:1047E0009B49096881F8350004A8FFF7D2FD002035
:1047F0009749096881F834000298FEF7FDFB002410
:104800000398012805D0022802D10E20307003E061
:1048100000BF0A20307000BF00BF204608E78C4868
:104820000068848DB8F1010F1ED1B9F1000F0ED0D0
:10483000B9F1010F0CD0B9F1020F03D0B9F1030F98
:104840000AD100E000BF2889A04328810BE000BF07
:1048500028892043288106E00298FEF7CDFB6F20CF
:1048600030700020E4E600BF0298FEF7C5FB002090
:1048700030702046DCE670B50025FEF7B9FB054632
:1048800073480068848D2846FEF7B6FB204670BD4D
:104890002DE9FC5F0446894692461E4600200090A2
:1048A0002078052804D0012030700020BDE8FC9F4E
:1048B000FEF79EFB0090BAF1000F03D0BAF1010F92
:1048C0000AD104E0208920EA090020810BE0208938
:1048D00040EA0900208106E00098FEF78DFB712078
:1048E00030700020E2E700BF4FF0000B656859E030
:1048F000A87C50B301283BD0022802D0032848D11D
:1049000012E02089298A00EA0107288AB8420AD1E0
:10491000002239462846FFF74EFD8046B8F1010FC8
:1049200001D14FF0010B3BE02089298A00EA010701
:1049300057B1002239462846FFF73DFD8046B8F1C1
:10494000010F01D14FF0010B2AE0288A218920EACA
:104950000107288AB8420AD1002239462846FFF7C3
:104960002AFD8046B8F1010F01D14FF0010B17E08D
:10497000288A218920EA010757B1002239462846B2
:10498000FFF719FD8046B8F1010F01D14FF0010B7F
:1049900006E00098FEF730FB6F203070002085E7BE
:1049A00000BF2D68002DA3D10098FEF725FBBBF1B9
:1049B000010F01D1FEF741FEFEF71AFB009020899E
:1049C00001900098FEF718FB0020307001986DE709
:1049D0002DE9F04104460D4600272078052804D033
:1049E000012028700020BDE8F081FEF701FB07469A
:1049F00026893846FEF700FB002028703046F2E793
:104A00002DE9F041A0211348FFF788F800250EE0BA
:104A1000681C86B20F4800EB051400EB0617002057
:104A200020706760AFF2E820E060681C85B2092D55
:104A3000EED3084800EB0514002020706060AFF250
:104A40000030E060034804490860BDE8F0810000E0
:104A50003C000020540E0020180000202DE9FC5FCF
:104A600005460F4691469A4600200090FEF7C0FA90
:104A700000906F480468006820B16D480068406885
:104A80006B4908600098FEF7B7FA2CB95A208AF8EB
:104A900000000020BDE8FC9FA8462E46781E01902D
:104AA0004FF0000B05E04E44C8F80060B0460BF133
:104AB000010B01988345F6D30020C8F8000025605B
:104AC00065602761E760C4F808908AF80000204616
:104AD000E0E72DE9F04104460D460027FEF788FA8D
:104AE0000746206968B16668306860602069401ECA
:104AF00020613846FEF780FA002028703046BDE875
:104B0000F0813846FEF778FA5D2028700020F6E73D
:104B10002DE9F04106460C46154600274548007829
:104B200020B1112028700020BDE8F081FEF760FA66
:104B30000746706920602068FEF7F0FC8046384622
:104B4000FEF75AFA002028704046EDE72DE9F041C3
:104B500005460E46144600273648007818B1122044
:104B60002070BDE8F081FEF743FA07466E613846D3
:104B7000FEF742FA0020207000BFF2E770B504464D
:104B80000D460026FEF734FA0646D4E903108842A3
:104B900004D33046FEF730FA5E2070BD60682860AE
:104BA00065602069401C20613046FEF725FA002030
:104BB000F3E770B505460C460026FEF719FA0646DF
:104BC0002868206068686060A868A060E868E060A5
:104BD000286920613046FEF70FFAD4E90301401A34
:104BE0006061002070BD70B5F0211348FEF796FF9C
:104BF00000240EE004EB44000F4901EBC005601CEB
:104C000000EB400001EBC00068600CA06861601C14
:104C100084B2092CEED304EB4400074901EBC00534
:104C20000020686005A0686108460149086070BD01
:104C30005000002029000020D42500203F00000063
:104C40002DE9F04106460D464FF000083078022865
:104C500004D0012028700020BDE8F081FEF7C8F9DB
:104C600080467468E08A78B12169081D20610F6868
:104C7000E08A401EE082A1682069884201D1606814
:104C800020610020287002E01F2028700027404685
:104C9000FEF7B2F93846DFE72DE9F04106460F4648
:104CA0004FF00008F748007810B10020BDE8F0810F
:104CB000FEF79EF98046F4480468006820B1F24887
:104CC00000684068F04908604046FEF795F9FCB17D
:104CD000FEF78EF98046ED480568D5B1006800689A
:104CE000EA4908604046FEF787F96E6006EB8700E8
:104CF000A860EE602E61AF820020E8820220207062
:104D0000002020816560E2A060612046FFF7C6F9BF
:104D100008E0DD4800686060DB4804604046FEF75C
:104D20006BF900242046C1E72DE9F0470446894687
:104D300015464FF0000A2078022804D00120287080
:104D40002046BDE8F087CF48007818B10F202870C2
:104D50002046F6E7FEF74CF98246A07A10B14FF0F4
:104D6000010801E04FF00008B9F1000F03D0B9F1DC
:104D7000010F49D121E0B8F1000F17D1C4A0606143
:104D80006668C24800683060C04806600020207035
:104D9000BD480068606000202081BB480460504628
:104DA000FEF72AF900202870002705E05046FEF79C
:104DB00023F94920287027462DE005E0022304222C
:104DC00000212046FFF7F2F8A07A0028F6D1B0A023
:104DD00060616668AD4800683060AC4806600020DD
:104DE0002070A9480068606000202081A648046007
:104DF0005046FEF701F9B8F1010F01D1FEF71DFC95
:104E000000202870002706E05046FEF7F5F807203E
:104E10002870274600BF00BF384692E770B50546A8
:104E20000026FEF7E5F806466C686068E06060689A
:104E300020610020E0823046FEF7DEF8002070BDE1
:104E40002DE9F0470746884615464FF000093878A7
:104E5000022804D0012028700020BDE8F08789488E
:104E6000007818B1022028700020F6E78948007801
:104E700018B10D2028700020EFE7FEF7B9F8814641
:104E80007C68E08A98B12169081D20610E68E08A7B
:104E9000401EE082A1682069884201D160682061DB
:104EA0004846FEF7A9F8002028703046D5E77A4832
:104EB000006890F8340040F004007749096881F8F0
:104EC000340000207449096881F835007248006890
:104ED000C0F830803846FFF7A9F84846FEF78CF84E
:104EE000FEF7ABFBFEF784F881466B48006890F84C
:104EF000350020B101280DD002280AD105E066480E
:104F00000068466A002028700DE000260E202870F8
:104F100009E000BF394660480068FFF730F8002616
:104F20000A20287000BF00BF00205B49096881F893
:104F300034005949096881F8350057490968C86142
:104F40005549096808625449096848624846FEF7AD
:104F500053F8304681E72DE9F04104460F461546E7
:104F60004FF000082078022804D00120287000208B
:104F7000BDE8F081FEF73CF88046A07A20B3002619
:104F80007FB1012F0CD107E002230422002120462B
:104F9000FFF70CF8701CC6B2A07A0028F4D109E023
:104FA00000BF0223042200212046FEF7FFFF701CF1
:104FB000C6B200BF00BF4046FEF71EF8FEF73DFB3D
:104FC0000E2028703046D3E74046FEF715F8002043
:104FD000287000BFCCE72DE9F04105460E460027BA
:104FE0002878022802D00120BDE8F081FEF700F801
:104FF0000746A87A60B10023042231462846FEF70E
:10500000D5FF3846FDF7F8FFFEF717FB0020EBE76A
:105010006C68E08AA18A884204DB3846FDF7ECFF21
:105020001E20E1E7E168081DE0600E60E08A401C98
:10503000E082D4E90210884201D16068E06038461D
:10504000FDF7DAFF0020CFE72DE9F04105460E46D7
:1050500000272878022802D00120BDE8F081FDF762
:10506000C7FF0746A87AC8B1002304223146284664
:10507000FEF79CFF3846FDF7BFFFFEF7DEFA002083
:10508000EBE700002900002014000020540000205D
:105090003F0000002A0000203C0000206C68E08AED
:1050A000A18A884204DB3846FDF7A6FF1E20D4E71C
:1050B00061682069884201D1A06820612069001FD1
:1050C000206120690660E08A401CE0823846FDF7D6
:1050D00093FF0020C1E72DE9F04105460F46164633
:1050E0004FF000082878022802D00120BDE8F081A6
:1050F000FDF77EFF8046A87AE8B106F0010050B1C6
:1051000005E00023042239462846FEF74FFFA87A1F
:105110000028F6D105E00023042239462846FEF790
:1051200045FF4046FDF768FF06F0040008B9FEF7AA
:1051300084FA0020DAE76C68E08AA18A884204DBFE
:105140004046FDF759FF1E20D0E706F0020058B197
:1051500061682069884201D1A06820612069001F30
:1051600020612069076009E0E168081DE0600F60C8
:10517000D4E90210884201D16068E060E08A401CF6
:10518000E0824046FDF738FF0020AFE72DE9F04709
:1051900005460C464FF0000A2878022802D001206C
:1051A000BDE8F087FDF724FF8246A87A207405F158
:1051B0000B0804F10809002705E018F8010B09F8AD
:1051C000010B781CC7B2082FF7D36E68F08A18B1AC
:1051D00030690068206001E000202060F08AA08033
:1051E000B08AE0805046FDF707FF0020D8E72DE9A0
:1051F000F041F0211048FEF791FC00240DE0601C06
:1052000086B204EB44000C4901EBC00506EB4600F6
:1052100001EBC0072F60601C84B2092CEFD304EBB4
:105220004400054901EBC0050020286008460349F9
:105230000860BDE8F0810000C42600205400002072
:1052400070B5044600262078032801D0002070BDE8
:10525000FDF7CEFE0646258915B12089401E208126
:105260003046FDF7C9FE2846F1E770B50546002631
:10527000D748007808B1002070BDFDF7B9FE06469A
:10528000D4480468006820B1D24800684068D14919
:1052900008603046FDF7B0FE4CB103202070258138
:1052A00000206060CCA060612046FEF7F7FE20463B
:1052B000E2E72DE9F0470446884615464FF000091D
:1052C0002078032804D0012028702046BDE8F0870C
:1052D000BF48007818B10F2028702046F6E7FDF788
:1052E00087FE8146A07A08B1012700E00027B8F1C7
:1052F000000F03D0B8F1010F3AD119E08FB9B6A071
:10530000606100202070B348006860600020208148
:10531000B04804604846FDF76FFE00202870002664
:1053200005E04846FDF768FE49202870264626E03D
:1053300005E00223012200212046FEF737FEA07A75
:105340000028F6D1A4A0606100202070A148006868
:105350006060002020819F4804604846FDF74CFEB5
:10536000012F01D1FEF769F900202870002606E020
:105370004846FDF741FE07202870264600BF00BFC3
:105380003046A3E72DE9F04105460E4614460027B6
:105390002878032803D001202070BDE8F0818C48D4
:1053A000007810B102202070F7E78C48007810B127
:1053B0000D202070F1E7FDF71BFE0746288940B15C
:1053C0002889401E28813846FDF716FE00202070EF
:1053D000E3E78348006890F8340040F0010080491A
:1053E000096881F8340000207D49096881F835009A
:1053F0007B48006806632846FEF718FE3846FDF72E
:10540000FBFDFEF71AF9FDF7F3FD07467448006847
:1054100090F8350020B1012809D0022806D102E019
:10542000002020700BE00E20207008E000BF29460D
:105430006B480068FEF7A3FD0A20207000BF00BF84
:1054400000206749096881F834006549096881F8D6
:10545000350063490968C8616149096808623846CE
:10546000FDF7CAFD00BF98E72DE9F04104460F465D
:1054700015464FF000082078032804D0012028703A
:105480000020BDE8F081FDF7B3FD8046A07A20B38F
:1054900000267FB1012F0CD107E002230122002159
:1054A0002046FEF783FD701CC6B2A07A0028F4D116
:1054B00009E000BF0223012200212046FEF776FD0D
:1054C000701CC6B200BF00BF4046FDF795FDFEF759
:1054D000B4F80E2028703046D3E74046FDF78CFD27
:1054E0000020287000BFCCE770B504460025207866
:1054F000032801D0012070BDFDF77AFD0546A07A92
:1055000060B10023012219462046FEF74FFD2846D0
:10551000FDF772FDFEF791F80020ECE720894FF6C9
:10552000FF71884207D22089401C20812846FDF760
:1055300063FD0020DFE72846FDF75EFD3320DAE754
:105540002DE9F04704460D464FF000092078032866
:1055500002D00120BDE8F087FDF74AFD8146A07A20
:10556000A87204F10B0705F10208002605E017F800
:10557000010B08F8010B701CC6B2082EF7D3208966
:1055800028804846FDF738FD0020E3E72DE9F0418B
:1055900004460E46154600272078032803D0012034
:1055A0002870BDE8F081FDF723FD07460020287034
:1055B000208908B1268105E0A07A08B9268101E09A
:1055C000492028703846FDF717FD00BFE9E70000C5
:1055D00029000020140000203F0000002A000020C5
:1055E0003C0000202DE9F34F85B088460020019053
:1055F000FDF7FEFC0190FE4850F8280030B10198FC
:10560000FDF7FAFC282007B0BDE8F08F0598FF28C9
:1056100004D1F848006890F836000590F4490598E0
:1056200051F8205025B90198FDF7E6FC2920EAE75A
:10563000012D04D10198FDF7DFFC4320E3E74FEA99
:10564000E80708F0070003900120B84000F0FF09C8
:1056500001210398814001F0FF0A0021E44A0598E6
:1056600042F82010104640F8285095F8386095F818
:105670003A00029095F839B0DF48805D00EA0B00EF
:10568000D0B1DD48805D20EA0B00DB498855084633
:10569000805D28B9D948007802998843D7490870B5
:1056A000D648007840EA0900D4490870D248C05D65
:1056B00040EA0A00D049C855EC69D4B104F10B00A6
:1056C000805D20EA0B0004F10B0188550846805DDF
:1056D00018B9A07A02998843A072A07A40EA09001A
:1056E000A07204F10B00C05D40EA0A0004F10B0156
:1056F000C855286A30B3286A0490049804681FE0EB
:1057000004F10B00805D20EA0B0004F10B018855C9
:105710000846805D18B9A07A02998843A072A07AE1
:1057200040EA0900A07204F10B00C05D40EA0A00E3
:1057300004F10B01C8550498001D049004980468F6
:10574000002CDDD185F8368085F83870039885F80F
:10575000370085F83A9085F839A00198FDF74CFCA0
:10576000A7480078012801D1FDF767FF00204AE72C
:105770002DE9FE4F06460F4690461C464FF00009A5
:10578000FDF736FC81469F48007828B14846FDF772
:1057900033FC3C20BDE8FE8F954850F8240060BBE8
:1057A0000120934941F824004846FDF725FC0023D9
:1057B000424639463046FDF7A2FC82460020009062
:1057C000019003460246514602902046FEF77EFCB9
:1057D000054635B98A48007801280CD1FDF72DFF20
:1057E00009E0FDF705FC81460020814941F82400CD
:1057F0004846FDF701FC2846CCE74846FDF7FCFB90
:105800002820C7E702F0010343B102F002032BB1E5
:1058100002E0491E002308C00029FAD170472DE993
:10582000F04F85B081468A4693461C46DDE90F78E5
:10583000129D00200390FDF7DBFB03907148007878
:1058400030B10398FDF7D8FB3C2005B0BDE8F08FE0
:10585000674850F8240088BB0120654941F82400BE
:105860000398FDF7C9FB2A4641463846FFF7CAFFB1
:105870002B465A4651464846FDF741FC0490119884
:10588000CDE9008002953A4620460E9B0499FEF72A
:105890001DFC064636B95A48007801280CD1FDF7A0
:1058A000CCFE09E0FDF7A4FB03900020504941F82D
:1058B00024000398FDF7A0FB3046C6E7FFE70398F6
:1058C000FDF79AFB2820C0E72DE9F04105460027A7
:1058D0004C48007810B14020BDE8F0813F2D01D147
:1058E0003E20F9E7FDF784FB0746FF2D03D1414831
:1058F000006890F836503E4850F8254024B93846A4
:10590000FDF77AFB4320E7E7012C04D13846FDF789
:1059100073FB3D20E0E714F8380F3749085C6178E5
:1059200088432178344A505414F838091146085CE9
:1059300030B994F83A103148007888432F490870FC
:10594000E06918B12046E169FEF719FB206A18B139
:105950002046216AFDF747FEA66A16B13046FEF7DB
:1059600018FD0020206384F8340084F835002648B0
:105970000078FF2804D224480078401C224908708F
:105980003846FDF739FBFEF7F9FAFDF731FB07461C
:105990001D48007820B11C480078401E1A49087044
:1059A0002046FDF798FB19480078401E17490870FB
:1059B00000200F4941F82500A06930B90020616935
:1059C000886113496069086005E0D4E90501486110
:1059D000D4E9051088610F48006860610D480460D3
:1059E0000DA020653846FDF707FB0548007815E057
:1059F000F41200203C0000202E0000202D0000208A
:105A000036000020290000202A0000203700002056
:105A100048000020400000203F000000012801D184
:105A2000FDF70BFE002057E72DE9F0410446002763
:105A30003F2C02D13E20BDE8F081FF2C0BD1FDF7B9
:105A4000D7FA0746F948006890F83B603846FDF7FA
:105A5000D3FA3046EFE7FDF7CBFA0746F44850F8A3
:105A6000245025B93846FDF7C7FA4320E3E7012D56
:105A700004D13846FDF7C0FA3D20DCE73F2085F829
:105A80003B003846FDF7B8FA0020D4E72DE9F0478F
:105A900006460F4614464FF00008E648007820B14D
:105AA000112020700020BDE8F087FDF7A1FA8046A4
:105AB000FF2E03D1DD48006890F83660DC4850F8CE
:105AC000265035B94046FDF797FA43202070002054
:105AD000E9E7012D06D14046FDF78EFA43202070FC
:105AE0000020E0E7286D38603868FDF717FD814633
:105AF0004046FDF781FA002020704846D3E72DE9A3
:105B0000F04106460F4614464FF00008C948007899
:105B100018B112202070BDE8F081FDF769FA8046C7
:105B2000FF2E03D1C148006890F83660C04850F895
:105B300026502DB94046FDF75FFA43202070EAE772
:105B4000012D05D14046FDF757FA43202070E2E7CA
:105B50002F654046FDF750FA0020207000BFDAE7BD
:105B600070B505460026FDF743FA0646B04850F8E2
:105B7000254024B93046FDF73FFA462070BD012C80
:105B800004D13046FDF738FA4320F7E794F83400A3
:105B900000F0080060B314F8340F00F0F700207034
:105BA00014F83409F8B9206BC8B93834A078A24980
:105BB00009780843A04908702078A049085C6178FA
:105BC000084314F838199D4A50543046FDF714FA2A
:105BD0009B480078012809D1FDF72FFD06E03046EB
:105BE000FDF70AFA02E03046FDF706FA0020C5E7A5
:105BF0003046FDF701FA4420C0E72DE9F04707469B
:105C00000D464FF0000A002028606860FDF7F0F9AB
:105C10008246FF2F03D18548006890F8367084488B
:105C200050F827402CB95046FDF7E6F94320BDE86F
:105C3000F087012C04D15046FDF7DEF94320F6E74A
:105C4000207C00F0010020B95046FDF7D5F9452031
:105C5000EDE70026D4F80C90D4F808805046FDF704
:105C6000CBF900E0761C58F8041B0029FAD02E600E
:105C7000A9EB060068600020D9E72DE9F041054650
:105C80004FF00008FDF7B4F98046FF2D05D16748B5
:105C9000006890F83650012608E06448006890F8E3
:105CA0003600A84201D1012600E00026604850F8E5
:105CB00025402CB94046FDF79FF94820BDE8F0810A
:105CC000012C04D14046FDF797F94320F6E794F8FC
:105CD00038705A48C05D94F8391088435749C85500
:105CE0000846C05D30B994F83A10534800788843AC
:105CF0005149087094F8340040F0080084F83400EA
:105D00004046FDF779F9012E01D1FDF796FC002000
:105D1000D4E72DE9F04105460E460027FDF768F966
:105D20000746FF2D03D14148006890F8365040489F
:105D300050F825402CB93846FDF75EF92920BDE81A
:105D4000F081012C04D13846FDF756F94320F6E7DF
:105D5000582221463046FEF7AFF93846FDF74CF998
:105D60000020ECE72DE9F04704460E4617464FF0B9
:105D70000009FDF73DF98146FF2C02D12B4805684B
:105D800002E02B4850F8245005F1540050F82680CA
:105D90004846FDF731F9002038704046BDE8F087ED
:105DA00070B504460026FDF723F90646254800781D
:105DB00030B1962020703046FDF71EF9012070BDED
:105DC000204805780078401C1E4908703046FDF7D1
:105DD00013F9002020702846F1E72DE9F04704462A
:105DE0000E46174698464FF00009FDF701F9814627
:105DF000FF2C02D10D48056802E00D4850F82450F0
:105E000005F1540040F826704846FDF7F5F80020EB
:105E100088F80000BDE8F08710B504480068FDF779
:105E200064F9FF20FFF750FD10BD00003C0000208A
:105E3000F4120020290000202D0000202E00002058
:105E4000360000205800002070B505460026634843
:105E5000007800B170BD6248007800B1FAE71DB368
:105E6000FDF7C6F806465F48006890F838405E487F
:105E7000005D5C49096891F8391088435A49085512
:105E80000846005D40B95748006890F83A105748F6
:105E900000788843554908705248006805633046C9
:105EA000FDF7AAF8FDF7C9FB00BFD3E72DE9F041E4
:105EB00005460E4617461C464848007810B1552046
:105EC000BDE8F0814648007808B13220F8E74FF489
:105ED0007A7060434FF47A71B0FBF1F14FF4616076
:105EE0006843C6EB061200EB8200384400EB400228
:105EF000C2EBC01001EBC0084046FFF7A5FF002031
:105F0000DEE770B5054600263F2D01D32A2070BD7F
:105F1000FDF76EF80646364850F8254024B930465D
:105F2000FDF76AF84320F2E7012C04D13046FDF773
:105F300063F84320EBE7206B20B93046FDF75CF8AF
:105F40005020E4E70020206394F8340000F037008C
:105F500040B114F8340F20F0370020700120607039
:105F6000343C02E0002084F8350094F8340000F05E
:105F70000800A8B93834A0781C49097808431B499F
:105F8000087020781849085C6178084314F83819BB
:105F9000154A50543046FDF72FF8FDF74EFB02E04E
:105FA0003046FDF729F80020B1E770B50025FDF770
:105FB0001FF805460F4804682846FDF71DF82046DF
:105FC00070BD70B504460025FDF712F80546094876
:105FD00004602846FDF710F870BD0000290000207D
:105FE0002A0000203C0000202E0000202D00002070
:105FF000F41200205C000020F848006808B9002076
:106000007047F6480168F54AC86810600020C8600B
:106010000861F3480088401CF14A1080F14800886C
:10602000401EF04A10800846EAE72DE9F05F064678
:106030000F4690469946DDE90ABA0C9DEA48007879
:1060400020B18B2028700020BDE8F09FFDF766FE90
:10605000FFF7D2FF04462CB9FDF7C4FE8620287056
:106060000020F1E7012084F82500A661E76184F8AB
:106070002480C4F80490C4F808B0BAF1000F02D12B
:10608000DAA0206201E0C4F820A0FDF7ABFE0020FA
:1060900028702046D8E7002180F8251080F82410C9
:1060A000C161416141608160D0A101620021016153
:1060B000CA490968C160C9490860C9490988491EB7
:1060C000C74A1180C7490988491CC64A11807047D0
:1060D00030B5057D05F00704C54D05EBC4031D680B
:1060E000854205D1C168196039B100250D6104E010
:1060F0000169C268CA6002B11161012580F82550AA
:106100000025C56005619D886D1E9D8030BD70B500
:1061100005460C462878642803D08920207000208A
:1061200070BDB148007818B18B2020700020F7E7CF
:10613000FDF7F4FD95F82500D8B101280FD002280D
:106140000ED003281BD12846FFF7C2FF2846FFF7D1
:10615000A2FFFDF747FE002020700120E0E700BF0E
:106160002846FFF798FFFDF73DFE00202070012034
:10617000D6E7FDF737FE872020700020D0E7FDF737
:1061800031FE8D2020700020CAE72DE9F041054640
:106190000E4614462878642804D0892020700020F8
:1061A000BDE8F0819048007818B1112020700020DF
:1061B000F6E7FDF7B3FD95F8250098B1012804D066
:1061C000022803D0032813D100BF00BF286A306023
:1061D0003068FDF7A3F90746FDF704FE00202070A4
:1061E0003846DDE7FDF7FEFD872020700020D7E769
:1061F000FDF7F8FD8D2020700020D1E770B5044632
:106200000D462078642803D089202870002070BDB6
:106210007548007818B18B2028700020F7E7FDF74B
:106220007DFD94F8250070B301280DD0022825D0FB
:1062300003282FD16F4960690968461AFDF7D2FD1E
:10624000002028703046E2E794F8240001280CD0A2
:10625000022809D1A06908B9E66900E0A669FDF73E
:10626000C1FD0020287006E000BFA669FDF7BAFD59
:106270000020287000BF00BF3046C8E7FDF7B2FD20
:1062800000202870C3E7FFE7FDF7ACFD87202870EA
:106290000020BCE7FDF7A6FD8D2028700020B6E7A2
:1062A00070B505460C462878642803D089202070F4
:1062B000002070BD4C48007818B18B202070002061
:1062C000F7E7FDF72BFD95F8256036B1012E05D0D7
:1062D000022E04D0032E06D102E000BF00BF00BF93
:1062E0000020207002E08D20207000BF00BFFDF76D
:1062F00079FD3046DDE770B50B46032580F8255063
:10630000012B05D13B4EC5693668354445610CE02B
:1063100085692DB9374EC56936683544456104E055
:10632000344E8569366835444561057D05F00704BE
:106330002F4D05EBC4010D682DB908600025C5601F
:1063400001258D8006E00A680860C26010618D88B2
:106350006D1C8D800025056170BD70B505460C462D
:106360002878642803D089202070002070BD1E4842
:10637000007818B18B2020700020F7E7FDF7CEFCE5
:1063800095F82500E8B1012810D002280FD0032885
:106390001DD12846FFF79CFE00212846FFF7ABFFE2
:1063A000FDF720FD002020700120DFE700BF002165
:1063B0002846FFF7A0FFFDF715FD00202070012003
:1063C000D4E7FDF70FFD872020700020CEE7FDF712
:1063D00009FD8D2020700020C8E70000700000201B
:1063E0006200002060000020290000203F00000023
:1063F000342C0020640000202DE9F04105460F46B2
:1064000090461C462878642804D0892020700020FB
:10641000BDE8F0817D48007818B18B202070002005
:10642000F6E7FDF77BFC95F82500002832D001281F
:106430002AD0022827D0032832D12846FFF748FE69
:1064400000202070B7B1032F02D0042F13D108E031
:106450006E681EB12846A968B04701E08F20207001
:106460000CE06E681EB141462846B04701E08F201F
:10647000207003E002E08420207000BF00BFFDF721
:10648000B1FC0120C4E700BFFDF7ACFC8E202070FA
:106490000120BDE7FDF7A6FC872020700020B7E7AC
:1064A000FDF7A0FC8D2020700020B1E710B5584802
:1064B0000068FFF719F80446204610BD08B500BF74
:1064C00000BF6A46002152480068FEF75BFFFDF7F7
:1064D00025FC50480068401C4E490860084600787A
:1064E00000F007084C4800EBC8073C681AE0E66873
:1064F000484960690968884213D12046FFF7E8FDE2
:1065000094F82400022804D101212046FFF7F3FE6D
:1065100002E0022084F82500656815B12046A168D4
:10652000A8473446002CE2D1FDF75CFCC9E700B572
:1065300087B0032000218022384BCDE90132CDE91C
:1065400003104FF6FD703D23354A00903548FFF7A4
:1065500066F906AA34A13D20FFF7D1FA07B000BDC5
:10656000F8B54FF420713448FDF7D8FA40212A4895
:10657000FDF7D4FA002515E0681C86B205EB85000E
:106580002D4901EBC00406EB860001EBC007642037
:106590002070002084F82500E760AFF2B010206280
:1065A000681C85B20F2DE7D305EB8500224901EB6E
:1065B000C00464202070002084F82500E060AFF261
:1065C000D41020620020134908601C490880102064
:1065D0001B49088018481B4908600120FEF745FE4A
:1065E000194908600020FEF740FE094908606A4624
:1065F00016A115480068FCF7CCFF6A4618A10448AC
:106600000068FCF7C6FFFFF792FFF8BD29000020E5
:106610006C00002064000020342C0020342A00206C
:10662000302C0020BD64000075432F4F532D494985
:1066300020546D7200000000B4270020620000208A
:1066400060000020700000206800002075432F4F7C
:10665000532D494920546D724C6F636B000000004C
:1066600075432F4F532D494920546D725369676EFE
:10667000616C00000146412903DB5A2901DC01223B
:1066800000E00022012A08D0612903DB7A2901DC1D
:10669000012200E00022012A01D1012200E00022B3
:1066A000104670470146412903DB5A2901DC0122CB
:1066B00000E00022012A08D0612903DB7A2901DCED
:1066C000012200E00022012A01D1012200E0002283
:1066D000012A08D0302903DB392901DC012200E03E
:1066E0000022012A01D1012200E000221046704759
:1066F0000146612903DB7A2901DC012200E0002246
:10670000104670470146412903DB5A2901DC01226A
:1067100000E00022104670470146302903DB39298A
:1067200001DC012200E000221046704701463029BA
:1067300003DB372901DC012200E00022104670470C
:106740000146302901DB392907DD412901DB4629D2
:1067500003DD612903DB662901DC012200E0002260
:10676000104670470146202901D0092901D1012294
:1067700000E00022104670470146202909D00D296B
:1067800007D00A2905D00C2903D0092901D00B29EB
:1067900001D1012200E00022104670470146202965
:1067A00003DB7E2901DC012200E000221046704755
:1067B0000146212903DB7E2901DC012200E00022C1
:1067C000104670470146202903DB7E2901DC0122A7
:1067D00000E00022012A35D1202909D00D2907D057
:1067E0000A2905D00C2903D0092901D00B2901D190
:1067F000012200E000222ABB412903DB5A2901DCE7
:10680000012200E00022012A08D0612903DB7A2955
:1068100001DC012200E00022012A01D1012200E076
:106820000022012A08D0302903DB392901DC0122AA
:1068300000E00022012A01D1012200E000220AB971
:10684000012200E000221046704701464AB2002AA9
:1068500001DB1F2901DD7F2901D1012200E0002297
:10686000104670470146412903DB5A2901DC012209
:1068700000E00022012A02D101F1200200E00A46D4
:10688000D0B270470146612903DB7A2901DC01227D
:1068900000E00022012A02D1A1F1200200E00A4614
:1068A000D0B27047F0B504460B462046FFF7EAFF2A
:1068B00005461846FFF7E6FF0646B54201D101201E
:1068C00000E0002007463846F0BD0000FD48FE49C4
:1068D00001600146416000218160C1600161416148
:1068E0008161C16101620163C1624162F7498163F3
:1068F000C1634FF48061016441640146F44A116050
:1069000070472DE9F04103460C4617460FB9BDE824
:10691000F08103B9FBE70025002202E02D022543A8
:10692000521C042AFAD3384603F0030C1946BCF172
:10693000000F08D0624603E001F8014B401E521CD4
:1069400008B1042AF8D30E4601E020C6001F04282F
:10695000FBD2314602E001F8014B401E0028FAD17B
:1069600000BFD4E730B505460C4622460021284634
:10697000FFF7C7FF30BD2DE9F04F85B007468846C9
:106980009146B9F1000F02D105B0BDE8F08F07B90B
:10699000FAE7B8F1000F00D1F6E746463D46AE42B1
:1069A00005D94A464146384601F088FBECE74C469B
:1069B0003819451E08EB0400461EA81B04900498D5
:1069C000042834D305F00300029006F0030101917E
:1069D000DDE90110884201D1012000E00020009093
:1069E0000098012823D10298032810D0029840B2C1
:1069F000039008E016F8010905F80109641E0398E0
:106A0000401E40B2039014B103980028F2DAA5F1B9
:106A1000030AA6F1030B04E05BF804094AF8040931
:106A2000241F042CF8D20AF103050BF1030604E03D
:106A300016F8010905F80109641E002CF8D100BF01
:106A4000A2E72DE9F84F80468946154615B9012081
:106A5000BDE8F88FB8F1000F01D10020F8E7B9F1D7
:106A6000000F01D10020F3E70124294608EB0502BD
:106A700009EB050302F0030C03F0030BDC4501D125
:106A8000012000E0002000900098012829D1BCF1ED
:106A9000000F12D0E2460AE0521E5B1E107893F8F7
:106AA00000E0704500D00024491EAAF1010A012C23
:106AB00003D111B1BAF1000FEED1012C11D116465C
:106AC0001F4608E0361F3F1F3068D7F800E07045CA
:106AD00000D00024091F012C01D10429F2D2324632
:106AE0003B4608E0521E5B1E107893F800E07045AC
:106AF00000D00024491E012C01D10029F2D12046EA
:106B0000A6E7F0B503460D461646DA6BB2FBF6F083
:106B100006FB102CBCF1000F02D0A6EB0C0400E029
:106B200000246119586C884201D20020F0BDA142B6
:106B300001D3A94201D20020F8E75718974201D2A9
:106B40000020F3E72244DF63586C401A5864104673
:106B5000ECE72DE9F04F81468C461C46B9FBF4F07A
:106B600004FB109BBBF1000F02D0A4EB0B0600E06E
:106B70000026B2FBF4F004FB102BBBF1000F02D097
:106B8000A4EB0B0300E00023D018ACF1010E00FBD6
:106B90000E60871806EB0208B04501D3904502D27B
:106BA0000020BDE8F08FBCF1010F22D9D5189D421D
:106BB00001D3954201D20020F3E7ACF1010000FBC4
:106BC00005F1A94203D3994201D3914201D2002099
:106BD000E7E701EB020A8A4501D3924501D2002082
:106BE000DFE7474503D38F4201D3574501D2002049
:106BF000D7E73846D5E72DE9FE4F074688461546C4
:106C00001C46002000901CB900BF01F08DFB00BFA6
:106C10000DB901AD00BF002028602FB942F2747099
:106C200020800020BDE8FE8FB8F1000F04D142F2B1
:106C3000757020800020F5E7DFF8889000BF00BF66
:106C400001F0A4FC009000BF00BFD9F83C00029006
:106C5000D9F844B043463A4601210298FFF779FF3C
:106C6000064666B900BF00BF009801F093FC00BF64
:106C700000BF2F6042F2E37020800020D2E75E4523
:106C80000ED900BF00BF009801F084FC00BF00BF18
:106C9000A6EB0B00286042F2E27020800020C1E7E2
:106CA000424639464846FFF72CFF8246BAF1000FAC
:106CB00015D100BF00BF009801F06CFC00BF00BF01
:106CC0002E6007E0742C002048454150BC2C002069
:106CD0007400002042F2E27020800020A2E700BF92
:106CE00000BF009801F056FC00BF00BF42F21070D8
:106CF0002080504696E72DE9FC5F06460D46144677
:106D0000002000901CB900BF01F00EFB00BF2DB9A0
:106D100042F2757020800020BDE8FC9FB5F5805FD1
:106D200004D942F2757020800020F5E726B942F2BE
:106D3000117020800020EFE700BF00BF01F026FCAB
:106D4000009000BF00BFFE493068084440B1FD49D3
:106D5000084418B1FC49084408B900BF0CE000BF62
:106D600000BF00BF009801F015FC00BF00BF42F259
:106D7000887020800020CFE700BFD6F80490D9F8B3
:106D8000380008B1484600E0F0488246DAF844701E
:106D9000DAF83CB000BF00BF009801F0FBFB00BF79
:106DA00000BF012D0DD9BBFBF5F005FB10B8B8F104
:106DB000000F02D0A5EB080000E000200190019830
:106DC0003F1A42F2107020803846A5E770B504469D
:106DD0000D462A462146DD48FFF78DFF0646304620
:106DE00070BD70B504460D461DB900BF01F09CFA98
:106DF00000BF1CB942F21170288070BDD0484042DB
:106E0000206000206060A060E06020616061A0619F
:106E1000E0612062A06260632063E0626062A06360
:106E2000E0632064606442F21070288000BFE4E7F1
:106E30002DE9FF4F91B00446DDE920950020009038
:106E40001DB900BF01F070FA00BFB9F1000F02D107
:106E50000DF1100900BF0020C9F8000029462046A6
:106E6000FFF7BFFF288842F21071884202D015B0A8
:106E7000BDE8F08F129828B1139818B942F27E70CD
:106E80002880F4E7149818B942F292702880EEE74F
:106E90001E9818B942F293702880E8E71F9818B935
:106EA00042F294702880E2E7A948006818B942F2DB
:106EB000E7702880DBE7A54810904FF0000A00BF7C
:106EC00000BF01F063FB009000BF00BF12980028D4
:106ED0005BD1109E109E0E96109E3746109EF06B52
:106EE0000B9004231A4614990B98FFF732FE039077
:106EF000039850B900BF00BF009801F04BFB00BFE2
:106F000000BF42F2E3702880B1E703990B98084470
:106F10000A90DDE91E2314990A98FFF71AFE8346AA
:106F2000BBF1000F0AD100BF00BF009801F032FB97
:106F300000BF00BF42F2E370288098E7039800EB9F
:106F40000B0A0398824501D3DA450AD200BF00BF7D
:106F5000009801F01FFB00BF00BF42F2E3702880E1
:106F600085E71098D0F84480C2457DD900BF00BFA6
:106F7000009801F00FFB00BF00BFAAEB0800C9F8A2
:106F8000000042F2E270288071E712980990DDE972
:106F900012010844401E0890DDE9081081420AD21F
:106FA00000BF00BF009801F0F5FA00BF00BF42F239
:106FB000977028805BE7002600200E9064480768E1
:106FC0003AE0B96B1298814205D1396C139881422D
:106FD00001D13E4632E0B86B0790396CB86B08447B
:106FE000401E0690DDE90701814200D226E00799A4
:106FF0000998884203D8DDE9071088420FD2079923
:107000000998884203D306990898884207D90699B7
:10701000099888420ED80699089888420AD300BF7A
:1070200000BF009801F0B6FA00BF00BF42F27F70C7
:1070300028801CE70E97FF68002FC2D100BF46B919
:1070400026461298A0631298E06313982064139860
:1070500060641098C06B0B9004231A4614990B9827
:10706000FFF777FD039000E04CE0039850B900BFB4
:1070700000BF009801F08EFA00BF00BF42F2E3703B
:107080002880F4E61098D0F84480039840450FD942
:1070900000BF00BF009801F07DFA00BF00BF039859
:1070A000A0EB0800C9F8000042F2E2702880DEE69A
:1070B000F06B0A90DDE91E2314990A98FFF749FD49
:1070C0008346BBF1000F0AD100BF00BF009801F05A
:1070D00061FA00BF00BF42F2D9702880C7E6D6F837
:1070E0004480C3450ED900BF00BF009801F052FA9A
:1070F00000BF00BFABEB0800C9F8000042F2D87037
:107100002880B4E614988000029004220299109816
:10711000FFF7F7FC0D900D9878BB1098D0F84480DD
:1071200000BF00BF009801F035FA00BF00BF129801
:1071300098B9C2450ED9AAEB0800C9F8000018E0BA
:10714000B2B0B1BAFEFFFEF8080A0EFC742C0020A3
:1071500074000020C9F800A00BE00298404505D952
:107160000298A0EB0800C9F8000002E00298C9F8F4
:10717000000042F2E270288079E6FFE700200190EB
:1071800032E03046DDE91E12FFF7BBFC0C900C9894
:1071900010BBF06B0A90D6F8448000BF00BF009887
:1071A00001F0F8F900BF00BF01991498401A05904A
:1071B000DDE91E2305990A98FFF7CBFC8246C245FC
:1071C00004D9AAEB0800C9F8000001E0C9F800A042
:1071D00042F2D87028804AE6019ADDE90C0141F8B4
:1071E00022000198401C0190149901988842C8D34C
:1071F000A6420CD10E98A060E7600E9810B10E98D0
:10720000C46001E0FE4804605FB1BC6009E07069E1
:107210000F9026610F98606174610F9808B10F9804
:107220000461F848206066600A98A0610A98584492
:10723000401EE0610D982062C4F828B01F9860637A
:107240001E9820631498E0621498606200BF00BF2B
:10725000009801F09FF900BF00BF42F21070288033
:1072600000BF04E62DE9F04105460C4600271CB995
:1072700000BF01F059F800BF2DB942F21170208013
:107280000020BDE8F08100BF00BF01F07FF9074694
:1072900000BF00BFDC492868084440B1DB4908440E
:1072A00018B1DB49084408B902E00DE000BF00BF97
:1072B00000BF00BF384601F06DF900BF00BF42F2C9
:1072C000887020800020DCE700BF6E6A00BF00BF2E
:1072D000384601F05FF900BF00BF42F21070208015
:1072E0003046CEE72DE9F04104460E4615464FF0F4
:1072F00000081DB900BF01F017F800BF2CB942F219
:10730000117028800020BDE8F08126B942F2937008
:1073100028800020F7E700BF00BF01F037F9804662
:1073200000BF00BFB749206888420BD000BF00BF34
:10733000404601F02FF900BF00BF42F2887028805C
:107340000020E0E7206BB0420BD200BF00BF4046F8
:1073500001F020F900BF00BF42F2937028800020A6
:10736000D1E7606A58B900BF00BF404601F012F98A
:1073700000BF00BF42F2DE7028800020C3E7E16A50
:10738000606A88420BD900BF00BF404601F002F995
:1073900000BF00BF42F2957028800020B3E7606A0A
:1073A000401E6062D4E9080150F8217000BF00BFA0
:1073B000404601F0EFF800BF00BF42F21070288095
:1073C0003846A0E72DE9F04704460F4615464FF032
:1073D00000091DB900BF00F0A7FF00BF2CB942F2A1
:1073E000117028800020BDE8F08700BF00BF01F0C9
:1073F000CDF8814600BF00BF8249206888420BD08B
:1074000000BF00BF484601F0C5F800BF00BF42F210
:10741000887028800020E6E7E16A606A88420BD322
:1074200000BF00BF484601F0B5F800BF00BF42F200
:10743000957028800020D6E7E06AC01B461EE06AEF
:10744000B0420BD800BF00BF484601F0A3F800BF10
:1074500000BF42F2957028800020C4E7606AB04205
:107460000BD900BF00BF484601F094F800BF00BF31
:1074700042F2957028800020B5E7206A50F82680F7
:1074800000BF00BF484601F085F800BF00BF42F2D0
:10749000107028804046A6E72DE9F04F02460C46C2
:1074A0009569D2F81CB0AC4201D35C4502D90020EA
:1074B000BDE8F08F536BB5FBF3F003FB105111B136
:1074C000A3EB010C01E04FF0000C176BB7FBF3F0DE
:1074D00003FB107109B15E1A00E0002605EB0C08F1
:1074E000A4EB080A07EB0609BAFBF9F009FB10A0A8
:1074F00008B9012000E0002086467046D8E72DE953
:10750000F04704460F4615464FF0000A1DB900BF6C
:1075100000F00AFF00BF24B942F211702880BDE8D4
:10752000F0871FB942F211702880F8E700BF00BF52
:1075300001F02CF8824600BF00BF32492068884223
:107540000AD000BF00BF504601F024F800BF00BFC2
:1075500042F288702880E2E739462046FFF79CFF18
:107560008046B8F1010F0AD000BF00BF504601F0BD
:1075700011F800BF00BF42F297702880CFE70026C5
:1075800010E0206A50F82600B8420AD100BF00BFC0
:10759000504600F0FFFF00BF00BF42F29870288005
:1075A000BDE7761C606AB042EBD8E16A606A884247
:1075B0000AD300BF00BF504600F0ECFF00BF00BF81
:1075C00042F2DD702880AAE74FF00008666A08E002
:1075D000206A50F82690B94502D14FF0010803E027
:1075E000761CE06AB042F3D800BFB8F1010F11D1A8
:1075F000D4E9080150F82100216A41F8260014E07E
:1076000074000020504F4F4CB2B0B1BAFEFFFEF8EC
:10761000080A0EFC00BF00BF504600F0BBFF00BFD1
:1076200000BF42F28870288079E7D4E9080140F869
:107630002170606A401C606200BF00BF504600F0CD
:10764000A9FF00BF00BF42F21070288000BF66E7AC
:107650002DE9F84F04460F461546002000904FF0E4
:10766000FF3B1DB900BF00F05FFE00BF2CB942F226
:10767000117028805846BDE8F88F27B942F2117082
:1076800028805846F7E700BF00BF00F07FFF00905A
:1076900000BF00BF3D49206888420BD000BF00BF3B
:1076A000009800F077FF00BF00BF42F2887028808A
:1076B0005846E0E739462046FFF7EEFE8046B8F12F
:1076C000010F0BD000BF00BF009800F063FF00BFA8
:1076D00000BF42F2977028805846CCE7002611E0A0
:1076E000206A50F82600B8420BD100BF00BF0098B6
:1076F00000F050FF00BF00BF42F29870288058464B
:10770000B9E7761C606AB042EAD8E16A606A8842EA
:107710000BD300BF00BF009800F03CFF00BF00BFCC
:1077200042F2DD7028805846A5E74FF00008666AEF
:1077300008E0206A50F82690B94502D14FF00108C0
:1077400003E0761CE06AB042F3D800BFB8F1010F45
:107750000FD1E06A401EA0EB060A00BF00BF0098F0
:1077600000F018FF00BF00BF42F2107028805046A2
:1077700081E700BF00BF009800F00CFF00BF00BF12
:1077800042F288702880584675E70000504F4F4CF1
:1077900010B502460B461146002001E0491C401C72
:1077A00019B10C780CB19842F8D310BD30B504462D
:1077B0004FF0FF312046FFF7EBFF0546284630BD6E
:1077C00070B504460D4616460CB9002070BD0DB9C3
:1077D0000020FBE721462A46002304E010780870C9
:1077E000491C521C5B1C21B11AB1107808B1B3427C
:1077F000F4D301B10AB90020E8E7B34201D2002076
:1078000008702046E2E770B504460D464FF0FF329F
:1078100029462046FFF7D4FF0646304670BD70B5B6
:1078200003460C4615460BB9002070BD0CB900206C
:10783000FBE70DB91846F8E7194600E0491C11B1FD
:1078400008780028FAD109B90020EEE72246002680
:1078500004E010780870491C521C761C21B11AB142
:10786000107808B1AE42F4D301B10AB90020DCE7C8
:10787000002008701846D8E770B504460D464FF052
:10788000FF3229462046FFF7CAFF0646304670BD44
:107890002DE9F04305460B469446BCF1000F02D19A
:1078A0000020BDE8F08335B90BB90020F9E718785E
:1078B00042421046F5E713B92A781046F1E7294607
:1078C0001C460F4626467F1C761C4FF0000805E03C
:1078D000491C641C7F1C761C08F10108087894F888
:1078E0000090484505D1087818B117B10EB1E045B0
:1078F000EED3E04501D10020D3E7087894F800905A
:10790000484505D0087894F80090A0EB09020BE0F8
:10791000087808B9002207E02FB90EB9002203E069
:107920003078424200E03A781046BAE770B5044633
:107930000D464FF0FF3229462046FFF7A9FF0646C5
:10794000304670BD2DE9F74F82B080460E46049850
:1079500018B9002005B0BDE8F08FB8F1000F09D1CB
:107960000EB90020F6E73078FEF77CFF07467C4230
:107970002046EFE73EB998F80000FEF773FF054692
:107980002C462046E6E7C146B246C846C3465646A0
:10799000CDF804A0D8460BF1010B019E701C01909C
:1079A000C84699F80000FEF75DFF054656469AF86E
:1079B0000000FEF757FF07460020009015E009F190
:1079C00001090AF1010A0BF1010B0198401C019019
:1079D0000098401C009099F80000FEF743FF054610
:1079E0009AF80000FEF73EFF0746BD420BD199F81A
:1079F000000040B1BBF1000F05D0019818B1049907
:107A000000988842DBD304990098884201D1002075
:107A1000A0E7BD4201D0EC1B16E00DB9002413E035
:107A2000BBF1000F0AD1019808B900240CE00199BC
:107A30000878FEF717FF07467C4205E09BF8000038
:107A4000FEF710FF05462C46204683E770B5044636
:107A50000D464FF0FF3229462046FFF773FF0646DA
:107A6000304670BD30B504460B4615460CB90020B3
:107A700030BD0BB90020FBE72146002201E0491C84
:107A8000521C31B1087820B10878A84201D09A423E
:107A9000F5D309B90020EBE79A4201D30020E7E7CC
:107AA0000878A84201D00020E2E70846E0E770B578
:107AB00005460C4622464FF0FF312846FFF7D2FF1D
:107AC0000646304670BD2DE9F04305460E46174682
:107AD00015B90020BDE8F0830EB90020FAE72C4666
:107AE000A6F1010949462046FFF752FE804644446C
:107AF0000CB90020EEE700E0641EAC4202D0207812
:107B0000B842F9D12078B84201D00020E2E72046FF
:107B1000E0E770B505460C4622464FF0FF31284697
:107B2000FFF7D1FF0646304670BD70B504460D46DE
:107B300016460CB9002070BD0BB90020FBE72146AA
:107B40001A4605E00878A84200D10E70491C521E62
:107B500019B1087808B1002AF4D12046EBE7F0B556
:107B600004460D4616464FF0FF333246294620465E
:107B7000FFF7DBFF07463846F0BD2DE9FF4F06460D
:107B80000F4615461EB9002004B0BDE8F08F0FB9AE
:107B90000020F9E70DB90020F6E7681C00B101E00C
:107BA0004FF0FF30039029463046FFF7F1FD804645
:107BB00038460399FFF7ECFD04460CB93046E3E77D
:107BC000444501D90020DFE706EB080BBBF1000FAD
:107BD00001D10020D8E707EB040BBBF1000F01D166
:107BE0000020D1E7A8EB040002904FF0000900202C
:107BF000019000BF06EB090000902246394600982C
:107C0000FFF746FE8246BAF1000F01D1012000E0E5
:107C10000020019009F10109019810B902988145ED
:107C2000E8D9BAF1000F01D00020ADE70098ABE72A
:107C300070B504460D464FF0FF3229462046FFF747
:107C40009CFF0646304670BD2DE9FF4F8DB00F46B4
:107C500015461A9E1D9818B9002011B0BDE8F08F86
:107C6000002003900490012F01DA01200390022DDF
:107C700001D3242D01D90120039096B33046FEF79D
:107C80008DFD02900298012802D00120039028E087
:107C9000302E26D0A6F13000C0B207901B980128E4
:107CA00004D0A6F14100C0B2069003E0A6F1610045
:107CB000C0B206900A2D02D80798A84209DB0A2D07
:107CC00009D907980A2804D3A5F10A000699884221
:107CD00001D9012000E0002005900598012800D17D
:107CE00003901D9C0398002846D1DDF834A0DDF8F0
:107CF00034A0CDF830A001200B9007E00B98401C79
:107D0000C0B20B900C98B0FBF5F00C900C98A84208
:107D1000F4D21098012800D100E0002009900B99BE
:107D200009980844B84225DC002001900B98B8421D
:107D300001DA0B9800E038460A903EB1B8460A983E
:107D4000391A0998081AC0B2089006E0DDE909104E
:107D5000084400F0FF08002008900898002806DD7D
:107D6000302E01D1012000E00020049004E000202A
:107D7000049001E001200390039800B1B846444408
:107D80001C9808B100202070641E4FF0000941E0EB
:107D90000398A8BBBAF1000F02D1B9F1000F1CD1B2
:107DA000BAFBF5F005FB10A000F0FF0BBBF10A0FCA
:107DB00004D20BF1300004F801090BE01B980128F4
:107DC00004D00BF1370004F8010903E00BF1570070
:107DD00004F80109BAFBF5FA1AE01098012810D14D
:107DE000049808B9019828B1049850B1A8F101008D
:107DF000484506D12D2004F801090120019007E033
:107E000003E02EB104F8016902E03F2004F8010903
:107E100009F10109C145BBD3039808B100201CE753
:107E20001D981AE72DE9FF5F05460E4617461C46CA
:107E3000DDE90F9ADDF8388000233A4631462846BE
:107E40008DE81007FFF700FF8346584604B0BDE8F1
:107E5000F09F2DE9FF4F85B0044689461F46DDE9B6
:107E600013AB002C02DA6542012601E0254600260C
:107E700012983346CDE902ABCDE900704946284659
:107E8000079AFFF7E1FE8046404609B0BDE8F08F53
:107E90002DE9FF4F8BB0064689461546B9F1000F14
:107EA00002D10DF1240900BFC9F80060189810B97B
:107EB00007A8189000BF0021189801701EB9002073
:107EC0000FB0BDE8F08F012D01D0242D01D9002085
:107ED000F6E734462078FEF74FFC039004E0641C7C
:107EE0002078FEF749FC039003980128F7D020780A
:107EF0002B2802D02D280BD103E0641C4FF0000B7F
:107F000009E00E98012800D1641C4FF0010B02E03B
:107F10004FF0000B00BF00BF0A9425B1082D1CD004
:107F2000102D36D11EE02078302814D1641C207822
:107F3000582802D078280BD100BF10256778384622
:107F4000FEF7FEFB8246BAF1010F00D1641C01E08E
:107F5000082500BF00E00A251CE02078302800D169
:107F6000641C17E02078302812D1641C207858282F
:107F700002D078280AD100BF67783846FEF7E0FBC8
:107F80008246BAF1010F00D1641C00E000BF00BFBF
:107F900000E000BF00BF4FF00008002002900190F9
:107FA00040E027783846FEF77DFB059005980128CC
:107FB00036D13846FEF7B0FB06900698012804D16A
:107FC000A7F13000C0B208900FE03846FEF790FBF2
:107FD00004900498012804D1A7F15700C0B208907A
:107FE00003E0A7F13700C0B208900898A84214DA5D
:107FF000029880B9304850F82500404509D308FB65
:1080000005F8089880440898804504D20120029021
:1080100001E001200290641C04E00120019001E0D5
:108020000120019001980028BBD00298012801D1BD
:108030004FF0FF380A98844202D0C9F8004001E0AE
:10804000C9F80060189880F800B0404638E7F8B5E5
:1080500004460D4616460020034632462946009047
:108060002046FFF715FF07463846F8BD2DE9FC41CD
:1080700005460E46174601A801233A4631460090B0
:108080002846FFF705FF04469DF8040040B9B4F107
:10809000004F02D36FF0004000E02046804607E02A
:1080A000B4F1004F02D34FF0004000E06042804640
:1080B0004046BDE8FC81000058720100002800D154
:1080C0007047002900D17047002A00D170472DE980
:1080D000F81F00F0030301F00304A34211D1C3F120
:1080E000040303F00303012B1DD3012A00D2F2E0A5
:1080F00011F8014B00F8014BA3F10103A2F10102B9
:10810000F1E700F0010301F00104A34200D094E084
:10811000012B44D311F8014B00F8014BA3F10103EB
:10812000A2F10102F4E7B2F5B47F26D3B1E8F81F5B
:10813000A0E8F81FB1E8F81FA0E8F81FB1E8F81FA1
:10814000A0E8F81FB1E8F81FA0E8F81FB1E8F81F91
:10815000A0E8F81FB1E8F81FA0E8F81FB1E8F81F81
:10816000A0E8F81FB1E8F81FA0E8F81FB1E8F81F71
:10817000A0E8F81FA2F5B472D5E7282A06D3B1E823
:10818000F81FA0E8F81FA2F12802F6E7042A06D398
:1081900051F8043B40F8043BA2F10402F6E7202A20
:1081A00042D331F8023B20F8023B31F8023B20F881
:1081B000023B31F8023B20F8023B31F8023B20F849
:1081C000023B31F8023B20F8023B31F8023B20F839
:1081D000023B31F8023B20F8023B31F8023B20F829
:1081E000023B31F8023B20F8023B31F8023B20F819
:1081F000023B31F8023B20F8023B31F8023B20F809
:10820000023B31F8023B20F8023B31F8023B20F8F8
:10821000023B31F8023B20F8023B31F8023B20F8E8
:10822000023BA2F12002BAE7022A06D331F8023B50
:1082300020F8023BA2F10202F6E7102A42D311F81D
:10824000013B00F8013B11F8013B00F8013B11F83C
:10825000013B00F8013B11F8013B00F8013B11F82C
:10826000013B00F8013B11F8013B00F8013B11F81C
:10827000013B00F8013B11F8013B00F8013B11F80C
:10828000013B00F8013B11F8013B00F8013B11F8FC
:10829000013B00F8013B11F8013B00F8013B11F8EC
:1082A000013B00F8013B11F8013B00F8013B11F8DC
:1082B000013B00F8013B11F8013B00F8013BA2F142
:1082C0001002BAE7012A06D311F8013B00F8013B7E
:1082D000A2F10102F6E7BDE8F81F704710B50024CF
:1082E00000BF00BF00F052F9044600BF00BF1021DC
:1082F000A148FEF737FB00BF00BF204600F04AF957
:1083000000BF00BF10BD10B5FFF7E8FF10BD10B5EE
:1083100000209A49086001F051F810BD10B5FFF730
:10832000F6FFFFF7F0FF10BD00BFFEE770B5054692
:108330000C46002614B900BFFFF7F6FF15B90A2056
:10834000208070BD00BF00BF00F020F9064600BFCE
:1083500000BF102288492846FFF732FA00BF00BF4D
:10836000304600F017F900BF00BF0020208000BF9A
:10837000E7E72DE9F04105460C46002714B900BF98
:10838000FFF7D2FF1DB90A202080BDE8F08110213F
:108390002846FFF7FDF90646102E15D200BF00BF94
:1083A00000F0F4F8074600BF00BF102229467248CB
:1083B000FFF706FA00BF00BF384600F0EBF800BF39
:1083C00000BF0020208002E04FF47A70208000BFC0
:1083D000DBE710B501F008F80446204610BD7047F1
:1083E00000B5014611B900BFFFF79EFF634A106850
:1083F00008B1002201E04FF4FA620A8000BD5F4933
:108400000860704770B50546284600F0CAF8044673
:10841000183C204670BD70B50546284600F0C1F8EE
:108420000446103C204670BD70B50546284600F055
:10843000B8F8044600BF204670BD30B502460B4672
:108440000024D2F1FF359C4126D24FF6FF74D2F1C1
:10845000FF359C410FD26FF07F44D2F1FF359C4134
:1084600003D2190E464C605C44E0190C444C645C29
:1084700004F108003EE0FF24D2F1FF359C4105D213
:10848000190A3F4C645C04F1100033E019463C4C7F
:10849000645C04F118002DE04FF6FF750024AD1A5E
:1084A0009C4115D26FF07F450024AD1A9C4107D244
:1084B000140E44EA0321324C645C04F1200019E0FC
:1084C000140C44EA03412E4C645C04F1280011E0D2
:1084D0000024D2F1FF059C4107D2140A44EA03614B
:1084E000274C645C04F1300004E01146244C645CC9
:1084F00004F1380030BD70B504460CB9082070BDD9
:10850000204600F051F805462846F8E770B50446C5
:108510000CB9102070BD204600F046F805462846EC
:10852000F8E770B504460CB9202070BD204600F075
:108530003BF805462846F8E72DE9F04304460D468A
:10854000002184EA01006940084302D14020BDE8CF
:10855000F083E243E843521C40F1000102EA0406C2
:1085600001EA050730463946FFF767FF8046C8F144
:108570003F094846EBE70000BC30002078000020AF
:10858000EC72010072B6704762B67047EFF310806C
:1085900072B6704780F31088704730BF704720BFB5
:1085A0007047B0FA80F0704790FAA0F0B0FA80F00F
:1085B000704790FAA0F0704710B5B0F1005F0AD391
:1085C000FE4CA04207D8440104EB810303F108529A
:1085D000002414600CE0B0F1804F09D3F84CA042A5
:1085E00006D8440104EB810303F1844200241460A3
:1085F00010BD10B5B0F1005F0AD3F04CA04207D80F
:10860000440104EB810303F10852012414600CE0DF
:10861000B0F1804F09D3EA4CA04206D8440104EBE4
:10862000810303F184420124146010BD2DE9F0415F
:1086300004464FF00008102C6BD2DFE804F0080E5F
:108640000F1014293E090A0B0C11120D135300BF11
:1086500000BF00BF00BF00BF89E000BF00BF00BF78
:1086600000BF00BF83E000BF00BFFFF78FFF804661
:1086700000BF00BFD348006820F48030D1490860B3
:1086800000BF00BF4046FFF785FF00BF00BF6EE0A0
:1086900000BF00BFFFF77AFF804600BF00BFC94898
:1086A000006820F40030C749086000BF00BF4046A2
:1086B000FFF770FF00BF00BF59E000BF00BFFFF72A
:1086C00065FF804600BF00BFBE48006820F48020E0
:1086D000BC49086000BF00BF4046FFF75BFF00BF1A
:1086E00000BF44E000BF00BFFFF750FF804600BF5F
:1086F00000BF4FF0E020006920F001004FF0E021C2
:10870000086100BF00BF4046FFF744FF00BF00BF45
:108710002DE04FF0E0204068401C102101EB40109C
:10872000C6B2B44222DAA4F11000C11700EBD16145
:10873000C1F34715C11700EBD1614911A0EB4111FD
:10874000CFB200BF00BFFFF721FF804600BF00BFD0
:108750000120B840A90001F1E021C1F8800100BF6B
:1087600000BF4046FFF716FF00BF00BF00BF00BFBD
:10877000BDE8F0812DE9F04104464FF00008102CCF
:108780006BD2DFE804F0080E0F1014293E090A0B23
:108790000C11120D135300BF00BF00BF00BF00BF7C
:1087A00089E000BF00BF00BF00BF00BF83E000BF83
:1087B00000BFFFF7EBFE804600BF00BF81480068A6
:1087C00040F480307F49086000BF00BF4046FFF79B
:1087D000E1FE00BF00BF6EE000BF00BFFFF7D6FEA6
:1087E000804600BF00BF7748006840F400307549FC
:1087F000086000BF00BF4046FFF7CCFE00BF00BFCF
:1088000059E000BF00BFFFF7C1FE804600BF00BFB8
:108810006C48006840F480206A49086000BF00BFCF
:108820004046FFF7B7FE00BF00BF44E000BF00BFF7
:10883000FFF7ACFE804600BF00BF4FF0E0200069AC
:1088400040F001004FF0E021086100BF00BF40464A
:10885000FFF7A0FE00BF00BF2DE04FF0E020406812
:10886000401C102101EB4010C7B2BC4222DAA4F137
:108870001000C11700EBD161C1F34715C11700EB20
:10888000D1614911A0EB4111CEB200BF00BFFFF78B
:108890007DFE804600BF00BF0120B040A90001F16D
:1088A000E021C1F8000100BF00BF4046FFF772FEA3
:1088B00000BF00BF00BF00BFBDE8F0812DE9F0415F
:1088C00004464FF00008102C19D2DFE804F0080E1F
:1088D0000F10111516090A0B0C12130D141700BFF7
:1088E00000BF00BF00BF00BF37E000BF00BF00BF38
:1088F00000BF00BF00BF00BF00BF00BF2DE04FF0B2
:10890000E0204068401C102101EB4010C7B2BC427F
:1089100022DAA4F11000C11700EBD161C1F34715B1
:10892000C11700EBD1614911A0EB4111CEB200BFDC
:1089300000BFFFF72BFE804600BF00BF0120B04004
:10894000A90001F1E021C1F8800200BF00BF40464C
:10895000FFF720FE00BF00BF00BF00BFBDE8F081F1
:108960002DE9F04706460D464FF0000A102E73D24F
:10897000DFE806F0080E0F10112F45090A0B0C5BFB
:10898000730D89A000BF00BF00BF00BF00BFE5E0BE
:1089900000BF00BFE2E000BF00BFFFF7F7FD824667
:1089A00000BF00BF07480C38046824F0FF042C43C4
:1089B000046000BF00BF504606E00000FFFF0F202C
:1089C000FFFF0F4024ED00E0FFF7E4FD00BF00BF14
:1089D000C4E000BF00BFFFF7D9FD824600BF00BF63
:1089E000CC48046824F47F4444EA0524046000BFB2
:1089F00000BF5046FFF7CEFD00BF00BFAEE000BF96
:108A000000BFFFF7C3FD824600BF00BFC148046836
:108A100024F47F0444EA0544046000BF00BF5046CC
:108A2000FFF7B8FD00BF00BF98E000BF00BFFFF731
:108A3000ADFD824600BF00BFB648001D046824F0AB
:108A40007F4444EA0564046000BF00BF5046FFF75E
:108A5000A1FD00BF00BF81E043E000BF00BFFFF702
:108A600095FD824600BF00BFAA480830046824F084
:108A7000FF042C43046000BF00BF5046FFF78AFD8F
:108A800000BF00BF6AE000BF00BFFFF77FFD824666
:108A900000BF00BF9F480830046824F47F0444EA04
:108AA0000544046000BF00BF5046FFF773FD00BFE0
:108AB00000BF53E000BF00BFFFF768FD824600BF64
:108AC00000BF94480830046824F07F4444EA0564F9
:108AD000046000BF00BF5046FFF75CFD00BF00BF51
:108AE0003CE04FF0E0204068401C102101EB4010BA
:108AF00000F0FF094E4530DAA6F11000C11700EB77
:108B00009171C1F38707C11700EB91718910A0EB38
:108B1000810101F0FF0800BF00BFFFF737FD82466B
:108B200000BF00BFB80000F1E020D0F800444FEAD9
:108B3000C801FF20884084434FEAC80105FA01F0CC
:108B40000443B80000F1E020C0F8004400BF00BFBB
:108B50005046FFF71FFD00BF00BF00BF00BFBDE8CC
:108B6000F0872DE9F04706464FF0000A102E70D22C
:108B7000DFE806F0080F1215182A3D090A0B0C4908
:108B80005C0D708400BF00BF00BF00BF00BF624C1F
:108B9000BCE06FF00204B9E06FF00104B6E04FF002
:108BA000FF34B3E000BF00BFFFF7F0FC824600BF18
:108BB00000BF58480568ECB200BF00BF5046FFF741
:108BC000E9FC00BF00BFA1E000BF00BFFFF7DEFC73
:108BD000824600BF00BF4F480568C5F3072400BFA9
:108BE00000BF5046FFF7D6FC00BF00BF8EE000BFBD
:108BF00000BFFFF7CBFC824600BF00BF45480568B9
:108C0000C5F3074482E000BF00BFFFF7BFFC824608
:108C100000BF00BF3F48001D05682C0E00BF00BF0D
:108C20005046FFF7B7FC00BF00BF6FE000BF00BFBA
:108C3000FFF7ACFC824600BF00BF3648083005682D
:108C4000ECB200BF00BF5046FFF7A4FC00BF00BF5E
:108C50005CE026E000BF00BFFFF798FC824600BF43
:108C600000BF2C4808300568C5F3074400BF00BFAB
:108C70005046FFF78FFC00BF00BF47E000BF00BFBA
:108C8000FFF784FC824600BF00BF22480830056819
:108C90002C0E00BF00BF5046FFF77CFC00BF00BF9A
:108CA00034E04FF0E0204068401C102101EB401000
:108CB00000F0FF094E4527DAA6F11000C11700EBBE
:108CC0009171C1F38707C11700EB91718910A0EB77
:108CD000810101F0FF0800BF00BFFFF757FC82468B
:108CE00000BF00BFB80000F1E020D0F8005400BF82
:108CF00000BF5046FFF74EFC00BF00BF4FEAC80060
:108D000025FA00F0C4B200E0034C00BF00BF2046CB
:108D1000BDE8F08718ED00E00080FFFF10B500F01F
:108D200036F800F091FA10BD704710B50446702C6B
:108D300004D204F11001C8B2FFF778FC10BD10B5E1
:108D4000FFF720FC10BD10B50446702C04D204F1CE
:108D50001001C8B2FFF70EFD10BD70B504460D46F8
:108D60000026702C10D200BF00BFFFF70FFC064694
:108D700000BF00BFF84840F8245000BF00BF304695
:108D8000FFF708FC00BF00BF70BD00BFFEE710B5D5
:108D9000002404E0E0B2F149FFF7DFFF641C702C0F
:108DA000F8D310BD70B50446002600BF00BFFFF722
:108DB000EDFB064600BF00BFFAF762FF00BF00BF31
:108DC0003046FFF7E7FB00BF00BF702C04D2E2483B
:108DD00050F8245005B1A847FAF768FF70BD10B5E8
:108DE0000020FFF7DFFF10BD10B50120FFF7DAFF0D
:108DF00010BD10B50220FFF7D5FF10BD10B5032040
:108E0000FFF7D0FF10BD10B50420FFF7CBFF10BD5A
:108E100010B50520FFF7C6FF10BD10B50620FFF7FF
:108E2000C1FF10BD10B50720FFF7BCFF10BD10B586
:108E30000820FFF7B7FF10BD10B50920FFF7B2FFFC
:108E400010BD10B50A20FFF7ADFF10BD10B50B2007
:108E5000FFF7A8FF10BD10B50C20FFF7A3FF10BD52
:108E600010B50D20FFF79EFF10BD10B50E20FFF7C7
:108E700099FF10BD10B50F20FFF794FF10BD10B57E
:108E80001020FFF78FFF10BD10B51120FFF78AFFEC
:108E900010BD10B51220FFF785FF10BD10B51320CF
:108EA000FFF780FF10BD10B51420FFF77BFF10BD4A
:108EB00010B51520FFF776FF10BD10B51620FFF78F
:108EC00071FF10BD10B51720FFF76CFF10BD10B576
:108ED0001820FFF767FF10BD10B51920FFF762FFDC
:108EE00010BD10B51A20FFF75DFF10BD10B51B2097
:108EF000FFF758FF10BD10B51C20FFF753FF10BD42
:108F000010B51D20FFF74EFF10BD10B51E20FFF756
:108F100049FF10BD10B51F20FFF744FF10BD10B56D
:108F20002020FFF73FFF10BD10B52120FFF73AFFCB
:108F300010BD10B52220FFF735FF10BD10B523205E
:108F4000FFF730FF10BD10B52420FFF72BFF10BD39
:108F500010B52520FFF726FF10BD10B52620FFF71E
:108F600021FF10BD10B52720FFF71CFF10BD10B565
:108F70002820FFF717FF10BD10B52920FFF712FFBB
:108F800010BD10B52A20FFF70DFF10BD10B52B2026
:108F9000FFF708FF10BD10B52C20FFF703FF10BD31
:108FA00010B52D20FFF7FEFE10BD10B52E20FFF7E7
:108FB000F9FE10BD10B52F20FFF7F4FE10BD10B55F
:108FC0003020FFF7EFFE10BD10B53120FFF7EAFEAD
:108FD00010BD10B53220FFF7E5FE10BD10B53320EF
:108FE000FFF7E0FE10BD10B53420FFF7DBFE10BD2B
:108FF00010B53520FFF7D6FE10BD10B53620FFF7AF
:10900000D1FE10BD10B53720FFF7CCFE10BD10B556
:109010003820FFF7C7FE10BD10B53920FFF7C2FE9C
:1090200010BD10B53A20FFF7BDFE10BD10B53B20B6
:10903000FFF7B8FE10BD10B53C20FFF7B3FE10BD22
:1090400010B53D20FFF7AEFE10BD10B53E20FFF776
:10905000A9FE10BD10B53F20FFF7A4FE10BD10B54E
:109060004020FFF79FFE10BD10B54120FFF79AFE8C
:1090700010BD10B54220FFF795FE10BD10B543207E
:10908000FFF790FE10BD10B54420FFF78BFE10BD1A
:1090900010B54520FFF786FE10BD10B54620FFF73E
:1090A00081FE10BD10B54720FFF77CFE10BD10B546
:1090B0004820FFF777FE10BD10B54920FFF772FE7C
:1090C00010BD10B54A20FFF76DFE10BD10B54B2046
:1090D000FFF768FE10BD10B54C20FFF763FE10BD12
:1090E00010B54D20FFF75EFE10BD10B54E20FFF706
:1090F00059FE10BD10B54F20FFF754FE10BD10B53E
:109100005020FFF74FFE10BD10B55120FFF74AFE6B
:1091100010BD10B55220FFF745FE10BD10B553200D
:10912000FFF740FE10BD10B55420FFF73BFE10BD09
:1091300010B55520FFF736FE10BD10B55620FFF7CD
:1091400031FE10BD10B55720FFF72CFE10BD10B535
:109150005820FFF727FE10BDCC3000208B8D00007B
:1091600010B55920FFF71EFE10BD10B55A20FFF7AD
:1091700019FE10BD10B55B20FFF714FE10BD10B531
:109180005C20FFF70FFE10BD10B55D20FFF70AFE53
:1091900010BD10B55E20FFF705FE10BD10B55F20B5
:1091A000FFF700FE10BD10B56020FFF7FBFD10BDFE
:1091B00010B56120FFF7F6FD10BD10B56220FFF776
:1091C000F1FD10BD10B56320FFF7ECFD10BD10B52B
:1091D0006420FFF7E7FD10BD10B56520FFF7E2FD45
:1091E00010BD10B56620FFF7DDFD10BD10B567207E
:1091F000FFF7D8FD10BD10B56820FFF7D3FD10BDF7
:1092000010B56920FFF7CEFD10BD10B56A20FFF73D
:10921000C9FD10BD10B56B20FFF7C4FD10BD10B522
:109220006C20FFF7BFFD10BD10B56D20FFF7BAFD34
:1092300010BD10B56E20FFF7B5FD10BD10B56F2045
:10924000FFF7B0FD10BD00005348C06F20F01C00B8
:109250005149C8670846C06F40F01000C8674E48C3
:10926000C03000684D4908404B49C1F8C0004A4829
:10927000C03000684A4908434749C0310860480681
:109280004549B03108604FF04C7008606020454996
:10929000086004204049C1F864014248A0380068D1
:1092A0003E4908403C49C1F8C0003E48A03800682B
:1092B0003D4908433849C1F8C0000846D0F860016C
:1092C00040F40000C1F8600100BF36480830006873
:1092D00000F0010080F001000028F6D12E48B030E7
:1092E0000068324908432C49C1F8B00070472DE9A5
:1092F000F043DFF8A4C0DCF8B0C0CCF3007CBCF1D4
:10930000000F3ED0DFF890C0DCF860C1CCF38A26B5
:10931000DFF884C0DCF860C1CCF30A0303EB9622CB
:10932000DFF874C0DCF864C1CCF30424DFF868C053
:10933000DCF864C10CF01F05DFF85CC0DCF8B0C0DD
:10934000CCF3036111B1032904D101E0184902E013
:10935000184900E000BF00BF01FB02F804F1010C56
:1093600005F101090CFB09FCB8FBFCF0DFF828C093
:10937000DCF8B0C0CCF3090C0CF10107B0FBF7F03E
:1093800000E00020DFF830C0CCF80000BDE8F0833A
:10939000094800687047000000E00F4010FC10FC16
:1093A0008100010060E10F4085018501030000900C
:1093B0000024F40040787D017C00002010B519489D
:1093C000006840F080701749086000201649486026
:1093D0000846006840F001000860FFF788FF044677
:1093E0002046FFF70CF810BD0F49486870472DE97B
:1093F000F0478246FFF77BFF4FF0000980460B4A9B
:109400000023404649460CF0D1FC064632460B4646
:10941000504600210CF0CAFC04460D462046294661
:10942000BDE8F087FCED00E0001000E040420F00D6
:1094300010B50024FAF724FCF9F7DAFD0446002100
:10944000FA48F7F719F8FA4A0021F848F7F7A3F8AD
:109450000020F84908700120F74908702046F9F704
:10946000CBFDFAF723FC10BD10B50024FAF708FC79
:10947000F9F7BEFD04460121F048F6F7FDFFEC4A7E
:10948000203A0121ED48F7F786F80020EC490870F2
:109490000120EC4908702046F9F7AEFDFAF706FC0A
:1094A00010BD10B50024FAF7EBFBF9F7A1FD044657
:1094B0000021E248F6F7E0FFDD4A403A0021DF48AC
:1094C000F7F769F80020E04908700120DF490870CB
:1094D0002046F9F791FDFAF7E9FB10BD10B5DC481D
:1094E0000078012801D1002010BDDA48F8F7EAFC25
:1094F000D848401CF8F7E6FCD748F8F7E3FC082109
:10950000D648F7F791FDD448F8F7DCFC0421D3489E
:10951000F7F78AFDD048F8F7D5FC0221CF48F7F7D6
:1095200083FDCD48F8F7CEFC0121CC48F7F77CFD50
:10953000C948401EF8F7C6FC8021C948F7F774FDFA
:10954000C548401EF8F7BEFC4021C548F7F76CFD42
:10955000C148401EF8F7B6FC2021C148F7F764FD6A
:10956000BD48401EF8F7AEFC1021BD48F7F75CFD82
:10957000B948F8F7A7FC2021B848F7F755FDB648D9
:10958000F8F7A0FC1021B548F7F74EFDB248C01E11
:10959000F8F798FC1021B348F7F746FDAE48C01E17
:1095A000F8F790FC2021AF48F7F73EFDAA48401D90
:1095B000F8F788FC0121AC48F7F736FDA648401DB6
:1095C000F8F780FC0221A848F7F72EFDA248401DBD
:1095D000F8F778FC0421A448F7F726FD9E48401DC3
:1095E000F8F770FC0821A048F7F71EFD00231A4683
:1095F00019469248F6F750FF0123002219468F487A
:10960000F6F74AFF00231A4619468848F6F744FF42
:1096100008218A48F7F75FF808218448F7F75BF8D4
:1096200000231A4619468548F6F75DFF01231A46BE
:1096300000218248F6F757FF02231A4600217F488F
:10964000F6F751FF03231A4600217C48F6F74BFF3B
:1096500004231A4600217948F6F745FF05231A46E8
:1096600000217648F6F73FFF06231A46002173488B
:10967000F6F739FF6723072200217048F6F733FF1A
:109680000823002201216D48F6F72DFF092301224E
:1096900011466A48F6F727FF0A230222012167488C
:1096A000F6F721FF6B23032201216448F6F71BFF25
:1096B0004FF48073002211465C48F6F714FF40F225
:1096C0000113012200215948F6F70DFF4FF4817371
:1096D000022200215548F6F706FF40F263130322E9
:1096E00000215248F6F7FFFE60490E20FFF735FBD8
:1096F0005F490F20FFF731FB5E492E20FFF72DFB5E
:109700000E20FFF720FB0F20FFF71DFB2E20FFF799
:109710001AFB00214948F6F78BFE01214748F6F76E
:1097200087FE00214148F6F783FE1E20F8F7A2F8D5
:109730001F20F8F79FF83E20F8F79CF800213F48DB
:10974000F6F79EFE01213D48F6F79AFE00213748C4
:10975000F6F796FE00213948F6F78EFE01213748CC
:10976000F6F78AFE00213148F6F786FE0020BBE6B8
:1097700070B504460D4615B94FF0FF3070BD3E4838
:10978000005D08287DD2DFE800F0041D3637387907
:109790007A7B00BF2C4800780028FBD101202A49A1
:1097A000087000202949087000212448F6F764FE5B
:1097B00000212248F6F700FF00BF24480078002867
:1097C000FBD05EE000BF1E4800780028FBD10120DE
:1097D0001B49087000201B49087001211748F6F743
:1097E0004BFE01211548F6F7E7FE00BF154800784B
:1097F0000028FBD045E044E043E000BF0D4800787E
:109800000028FBD101200B49087000200A4908708C
:1098100000210648F6F730FE00210448F6F7CCFE9A
:1098200000BF054800780028FBD02AE000900340E4
:10983000CC320020840000208500002000800340FE
:109840008200002083000020800000208100002092
:109850009A000020003800F0040800F000400240A8
:10986000007000400050004000100640A39400002B
:1098700069940000319400008600002001E000E0BF
:1098800000BF00BF094850F8240000EE100AB8EEEF
:10989000400ADFED070A20EE200ADFED060A80EE1F
:1098A000201A85ED001A002068E700008C320020A5
:1098B00000404E450000804510B52548F8F702FBF2
:1098C00000BF2348F8F781FA0028FAD0F6F7DEFF48
:1098D00004460CB100BFFEE710BD2DE9F04104467F
:1098E0000D46164604F0030018B14FF0FF30BDE8F6
:1098F000F0810027F9F77CFB0746324621462846CF
:10990000F7F706F820B1324621462846F7F700F867
:109910003846F9F771FB0020E9E72DE9F0410446EC
:109920000D46164604F0030018B14FF0FF30BDE8B5
:10993000F0810027F9F75CFB0746324621462846AE
:10994000F6F7CCFF3846F9F757FB0020EFE70000A9
:10995000005800F02DE9F04104460D4616461F461A
:10996000082C03DB4FF0FF30BDE8F08100BF04EBB3
:109970004400F94901EB8000C0780128F7D004EBDE
:10998000440001EB800000790128F0D0002004EBB6
:109990004401F14A02F8210004EB4400114601EBB6
:1099A0008000467004EB440001EB8000877004EBFC
:1099B000440001EB8000856014BBE848F8F782FAA8
:1099C000E748F8F77FFAE648F8F77CFAE548F7F752
:1099D000B7FCE548F7F7B4FC0421E448F7F7E7FBE8
:1099E0000821E248F7F7D4FBA6B9E148854208D13F
:1099F000FFF7CEFC804600224146DE48F7F70BFD1C
:109A00000CE0FFF7C5FC804601224146D948F7F734
:109A100002FD03E03946D748F7F72CFD012C33D17E
:109A2000CE48401CF8F74EFACD48401DF8F74AFAE8
:109A3000CB48401DF8F746FACF48F7F781FCCF48EE
:109A4000F7F77EFC0121CE48F7F7B1FB0221CC48A5
:109A5000F7F79EFBA6B9C648854208D1FFF798FCE8
:109A6000804600224146C748F7F7D5FC0CE0FFF7D7
:109A70008FFC804601224146C248F7F7CCFC03E048
:109A80003946C048F7F7F6FC022C33D1B348801CA6
:109A9000F8F718FAB2480930F8F714FAB048093064
:109AA000F8F710FAB848F7F74BFCB848F7F748FC56
:109AB0000221B748F7F77BFB0121B548F7F768FBB0
:109AC000A6B9AB48854208D1FFF762FC8046002268
:109AD0004146B048F7F79FFC0CE0FFF759FC804681
:109AE00001224146AB48F7F796FC03E03946A94806
:109AF000F7F7C0FC032C33D19848C01CF8F7E2F903
:109B000097480830F8F7DEF995480830F8F7DAF9A1
:109B1000A148F7F715FCA148F7F712FC1021A0485F
:109B2000F7F745FB20219E48F7F732FBA6B990488E
:109B3000854208D1FFF72CFC804600224146994817
:109B4000F7F769FC0CE0FFF723FC80460122414651
:109B50009448F7F760FC03E039469248F7F78AFC2F
:109B6000042C33D17D48001DF8F7ACF97C4808304F
:109B7000F8F7A8F97A480830F8F7A4F98A48F7F70F
:109B8000DFFB8A48F7F7DCFB40218548F7F70FFB3E
:109B900080218348F7F7FCFAA6B97548854208D1B9
:109BA000FFF7F6FB8046002241468148F7F733FC79
:109BB0000CE0FFF7EDFB8046012241467C48F7F7B9
:109BC0002AFC03E039467A48F7F754FC052C31D1DA
:109BD0006248401DF8F776F96148F8F773F9604874
:109BE000F8F770F97348F7F7ABFB7348F7F7A8FB82
:109BF00001215E48F7F7DBFA02215C48F7F7C8FA63
:109C0000A6B95B48854208D1FFF7C2FB8046002217
:109C100041466A48F7F7FFFB0CE0FFF7B9FB8046C7
:109C2000012241466548F7F7F6FB03E039466348F1
:109C3000F7F720FC062C37D14848801DF8F742F989
:109C40004748401EF8F73EF94548401EF8F73AF9F4
:109C500041F60200F7F774FB41F60240F7F770FB9C
:109C600040214FF04020F7F7A2FA80214FF040202A
:109C7000F7F78EFAA6B93E48854208D1FFF788FB70
:109C80008046002241464E48F7F7C5FB0CE0FFF73F
:109C90007FFB8046012241464948F7F7BCFB03E0C1
:109CA00039464748F7F7E6FB072C33D12B48C01D50
:109CB000F8F708F92A48801CF8F704F92848801CAE
:109CC000F8F700F93F48F7F73BFB3F48F7F738FB59
:109CD00001213E48F7F76BFA02213C48F7F758FAA2
:109CE000A6B92348854208D1FFF752FB80460022DF
:109CF00041463748F7F78FFB0CE0FFF749FB8046FA
:109D0000012241463248F7F786FB03E039463048E6
:109D1000F7F7B0FB012004EB44010F4A02F82100E1
:109D2000002021E62DE9F0470546884616461F46E5
:109D30004FF00009082D03DB4FF0FF30BDE8F0873E
:109D400036B12FB105EB4500034911F8200010B9D9
:109D50004FF0FF30F2E73DE0DC320020002000F061
:109D6000010800F002080100020C01000050004050
:109D7000A086010000000240020006000204060066
:109D8000006002400010024002040A0002000A00C3
:109D900000200640002002400210090002140900C1
:109DA000001006400030024002180900021C0900A1
:109DB00000000C40020001000204010000100C40F1
:109DC00000200C4002000300020403000070004069
:109DD00000300C40F9F70CF98146012005EB4501F4
:109DE000FE4A02EB8101087105EB4500114601EBCB
:109DF00080004078002876D1002D75D100BFF8484A
:109E0000F7F7E0FB0028FAD100224146F448F7F7C3
:109E1000D2FB012F28D13178F148F7F7F6FB072163
:109E2000EF48F7F7E1FBEE48F7F7E0FB58B1002009
:109E300005EB4501E94A02EB810108714846F9F753
:109E4000DBF8B81E7AE700BFE548F7F7BBFB002850
:109E5000FAD105EB4501E14A02EB81010871484660
:109E6000F9F7CAF8002069E7002445E044B9315DFC
:109E7000DB48F7F7CAFB0321D948F7F7B5FB13E036
:109E8000781EA04208D1315DD548F7F7BEFB052109
:109E9000D348F7F7A9FB07E0315DD148F7F7B5FBE9
:109EA0000121CF48F7F7A0FBCD48F7F79FFBE0B1C2
:109EB000781EA0420AD0CA48F7F798FB00F01000BD
:109EC000102803D00421C648F7F78EFB002005EBCD
:109ED0004501C24A02EB810108714846F9F78CF846
:109EE0004FF0FF302AE71CE209E000BFBC48F7F75B
:109EF00069FB0028FAD1641CBC42B7D3A4E3012D4E
:109F00007FD100BFB748F7F75DFB0028FAD10022E8
:109F10004146B448F7F74FFB012F28D13178B148BB
:109F2000F7F773FB0721AF48F7F75EFBAD48F7F78C
:109F30005DFB58B1002005EB4501A84A02EB810109
:109F400008714846F9F758F8B81EF7E600BFA5486B
:109F5000F7F738FB0028FAD105EB45019F4A02EBE1
:109F6000810108714846F9F747F80020E6E6002429
:109F700044E044B9315D9B48F7F747FB032199481A
:109F8000F7F732FB13E0781EA04208D1315D954807
:109F9000F7F73BFB05219348F7F726FB07E0315D18
:109FA0009048F7F732FB01218E48F7F71DFB8D48EB
:109FB000F7F71CFBD8B1781EA0420AD08948F7F702
:109FC00015FB00F01000102803D004218548F7F796
:109FD0000BFB002005EB4501804A02EB8101087173
:109FE0004846F9F709F84FF0FF30A7E609E000BF4F
:109FF0007C48F7F7E7FA0028FAD1641CBC42B8D3D2
:10A0000022E3022D7FD100BF7748F7F7DBFA002863
:10A01000FAD1002241467448F7F7CDFA012F28D132
:10A0200031787148F7F7F1FA07216F48F7F7DCFA52
:10A030006D48F7F7DBFA58B1002005EB4501674A98
:10A0400002EB810108714846F8F7D6FFB81E75E6A5
:10A0500000BF6548F7F7B6FA0028FAD105EB4501CD
:10A060005E4A02EB810108714846F8F7C5FF0020FF
:10A0700064E6002444E044B9315D5B48F7F7C5FA73
:10A0800003215948F7F7B0FA13E0781EA04208D12F
:10A09000315D5548F7F7B9FA05215348F7F7A4FAA7
:10A0A00007E0315D5048F7F7B0FA01214E48F7F765
:10A0B0009BFA4D48F7F79AFAD8B1781EA0420AD019
:10A0C0004948F7F793FA00F01000102803D0042154
:10A0D0004548F7F789FA002005EB45013F4A02EBB6
:10A0E000810108714846F8F787FF4FF0FF3025E6F9
:10A0F00009E000BF3C48F7F765FA0028FAD1641C74
:10A10000BC42B8D3A0E2032D72D100BF3748F7F7A5
:10A1100059FA0028FAD1002241463448F7F74BFAA1
:10A12000012F28D131783148F7F76FFA07212F48EE
:10A13000F7F75AFA2D48F7F759FA58B1002005EB0E
:10A140004501264A02EB810108714846F8F754FFA1
:10A15000B81EF3E500BF2548F7F734FA0028FAD116
:10A1600005EB45011D4A02EB810108714846F8F7ED
:10A1700043FF0020E2E500244FE044B9315D1B4875
:10A18000F7F743FA03211948F7F72EFA13E0781E80
:10A19000A04208D1315D1548F7F737FA0521134879
:10A1A000F7F722FA07E0315D1048F7F72EFA0121A0
:10A1B0000E48F7F719FA0D48F7F718FA30B3781E7A
:10A1C000A0420AD00948F7F711FA00F01000102851
:10A1D00003D004210548F7F707FA0AE0DC32002033
:10A1E0000000024000100240002002400030024007
:10A1F00016E0002005EB4501FE4A02EB81010871E3
:10A200004846F8F7F9FE4FF0FF3097E500BFFA48EF
:10A21000F7F7D8F90028FAD1641CBC42ADD313E299
:10A22000042D7FD100BFF548F7F7CCF90028FAD10B
:10A2300000224146F148F7F7BEF9012F28D13178C5
:10A24000EE48F7F7E2F90721EC48F7F7CDF9EB48CC
:10A25000F7F7CCF958B1002005EB4501E54A02EBD0
:10A26000810108714846F8F7C7FEB81E66E500BFD1
:10A27000E248F7F7A7F90028FAD105EB4501DD4AD6
:10A2800002EB810108714846F8F7B6FE002055E55B
:10A29000002444E044B9315DD848F7F7B6F903210A
:10A2A000D648F7F7A1F913E0781EA04208D1315D36
:10A2B000D248F7F7AAF90521D048F7F795F907E052
:10A2C000315DCE48F7F7A1F90121CC48F7F78CF9B9
:10A2D000CA48F7F78BF9D8B1781EA0420AD0C74810
:10A2E000F7F784F900F01000102803D00421C348C8
:10A2F000F7F77AF9002005EB4501BE4A02EB810130
:10A3000008714846F8F778FE4FF0FF3016E509E08F
:10A3100000BFBA48F7F756F90028FAD1641CBC42CE
:10A32000B8D391E1052D7FD100BFB548F7F74AF9C1
:10A330000028FAD100224146B148F7F73CF9012F35
:10A3400028D13178AE48F7F760F90721AC48F7F724
:10A350004BF9AB48F7F74AF958B1002005EB450136
:10A36000A44A02EB810108714846F8F745FEB81E81
:10A37000E4E400BFA248F7F725F90028FAD105EB7D
:10A3800045019C4A02EB810108714846F8F734FE0A
:10A390000020D3E4002444E044B9315D9848F7F745
:10A3A00034F903219648F7F71FF913E0781EA0420D
:10A3B00008D1315D9248F7F728F905219048F7F761
:10A3C00013F907E0315D8E48F7F71FF901218C483A
:10A3D000F7F70AF98A48F7F709F9D8B1781EA042C9
:10A3E0000AD08748F7F702F900F01000102803D0D0
:10A3F00004218348F7F7F8F8002005EB45017D4A72
:10A4000002EB810108714846F8F7F6FD4FF0FF3086
:10A4100094E409E000BF7A48F7F7D4F80028FAD1AD
:10A42000641CBC42B8D30FE1062D7FD100BF754834
:10A43000F7F7C8F80028FAD1002241467148F7F72B
:10A44000BAF8012F28D131786E48F7F7DEF80721E6
:10A450006C48F7F7C9F86B48F7F7C8F858B100200F
:10A4600005EB4501634A02EB810108714846F8F7A4
:10A47000C3FDB81E62E400BF6248F7F7A3F80028E6
:10A48000FAD105EB45015B4A02EB810108714846B0
:10A49000F8F7B2FD002051E4002444E044B9315DF6
:10A4A0005848F7F7B2F803215648F7F79DF813E03C
:10A4B000781EA04208D1315D5248F7F7A6F8052171
:10A4C0005048F7F791F807E0315D4E48F7F79DF8EF
:10A4D00001214C48F7F788F84A48F7F787F8D8B1D0
:10A4E000781EA0420AD04748F7F780F800F0100025
:10A4F000102803D004214348F7F776F8002005EB35
:10A5000045013C4A02EB810108714846F8F774FDA9
:10A510004FF0FF3012E409E000BF3A48F7F752F875
:10A520000028FAD1641CBC42B8D38DE0072D60D15D
:10A5300000BF3548F7F746F80028FAD10022414617
:10A540003148F7F738F8012F28D131782E48F7F73E
:10A550005CF807212C48F7F747F82B48F7F746F83F
:10A5600058B1002005EB4501224A02EB8101087138
:10A570004846F8F741FDB81E64E400BF2248F7F7EB
:10A5800021F80028FAD105EB45011A4A02EB8101B6
:10A5900008714846F8F730FD002053E4002451E0EC
:10A5A00044B9315D1848F7F730F803211648F7F73A
:10A5B0001BF813E0781EA04208D1315D1248F7F76E
:10A5C00024F805211048F7F70FF807E0315D0E4831
:10A5D000F7F71BF801210C48F7F706F80A48F7F7D8
:10A5E00005F840B3781EA04218D00748F6F7FEFFE2
:10A5F0000CE029E0DC3200200030024000000C407A
:10A6000000100C4000200C4000300C4000F0100006
:10A61000102803D00421FD48F6F7E6FF002005EBE3
:10A620004501FB4A02EB810108714846F8F7E4FC5A
:10A630004FF0FF3006E400BFF448F6F7C3FF0028F0
:10A64000FAD1641CBC42ABD3002005EB4501F04AB3
:10A6500002EB810108714846F8F7CEFC002041E486
:10A660002DE9F0470546884617461E464FF000097B
:10A67000082D03DB4FF0FF30BDE8F08737B12EB176
:10A6800005EB4500E24911F8200010B94FF0FF300A
:10A69000F2E7F8F7ADFC8146012005EB4501DC4A05
:10A6A00002EB8101C87005EB4500114601EB80000B
:10A6B0004078002878D1002D78D100BFD548F6F732
:10A6C00081FF0028FAD101224146D248F6F773FFF4
:10A6D000012E29D10721CF48F6F786FFCD48F6F79E
:10A6E00085FF58B1002005EB4501C94A02EB810105
:10A6F000C8704846F8F780FCB01EBDE700BFC548EB
:10A70000F6F760FF0028FAD1C248F6F780FF3870EC
:10A71000002005EB4501BE4A02EB8101C8704846A6
:10A72000F8F76AFC0020A7E700243BE024B90B21DE
:10A73000B848F6F759FF0BE0701EA04204D105217E
:10A74000B448F6F751FF03E00921B248F6F74CFF91
:10A75000B048F6F74BFFD0B1701EA0420AD0AD480A
:10A76000F6F744FF00F01000102803D00421A94898
:10A77000F6F73AFF002005EB4501A54A02EB8101FF
:10A78000C8704846F8F738FC4FF0FF3074E700BF58
:10A79000A048F6F717FF0028FAD19E48F6F737FFD2
:10A7A0003855641CB442C1D375E3FFE7012D78D15D
:10A7B00000BF9948F6F706FF0028FAD1012241466A
:10A7C0009548F6F7F8FE012E29D107219248F6F7B1
:10A7D0000BFF9148F6F70AFF58B1002005EB450141
:10A7E0008B4A02EB8101C8704846F8F705FCB01EA1
:10A7F00042E700BF8848F6F7E5FE0028FAD1864810
:10A80000F6F705FF3870002005EB4501804A02EBA2
:10A810008101C8704846F8F7EFFB00202CE70024C0
:10A820003BE024B90B217C48F6F7DEFE0BE0701EFE
:10A83000A04204D105217848F6F7D6FE03E00921AD
:10A840007548F6F7D1FE7448F6F7D0FED0B1701E09
:10A85000A0420AD07048F6F7C9FE00F01000102898
:10A8600003D004216C48F6F7BFFE002005EB45013C
:10A87000674A02EB8101C8704846F8F7BDFB4FF00C
:10A88000FF30F9E600BF6448F6F79CFE0028FAD1D5
:10A890006148F6F7BCFE3855641CB442C1D3FAE2F5
:10A8A000FFE7022D78D100BF5C48F6F78BFE002849
:10A8B000FAD1012241465948F6F77DFE012E29D1F1
:10A8C00007215648F6F790FE5448F6F78FFE58B128
:10A8D000002005EB45014E4A02EB8101C870484655
:10A8E000F8F78AFBB01EC7E600BF4C48F6F76AFED1
:10A8F0000028FAD14948F6F78AFE3870002005EBA7
:10A900004501434A02EB8101C8704846F8F774FBE1
:10A910000020B1E600243BE024B90B213F48F6F7C4
:10A9200063FE0BE0701EA04204D105213B48F6F700
:10A930005BFE03E009213948F6F756FE3748F6F783
:10A9400055FED0B1701EA0420AD03448F6F74EFE34
:10A9500000F01000102803D004213048F6F744FE20
:10A96000002005EB45012A4A02EB8101C8704846E8
:10A97000F8F742FB4FF0FF307EE600BF2748F6F7BE
:10A9800021FE0028FAD12548F6F741FE3855641C0F
:10A99000B442C1D37FE2FFE7032D76D100BF204848
:10A9A000F6F710FE0028FAD1012241461C48F6F7BE
:10A9B00002FE012E36D107211948F6F715FE184878
:10A9C000F6F714FE58B1002005EB4501104A02EBE2
:10A9D0008101C8704846F8F70FFBB01E4CE600BF77
:10A9E0000F48F6F7EFFD0028FAD10D48F6F70FFEF5
:10A9F0003870002005EB4501054A02EB8101C87063
:10AA00004846F8F7F9FA002036E6000000300C401E
:10AA1000DC32002000000240001002400020024012
:10AA20000030024000243CE024B90B21F748F6F73F
:10AA3000DBFD0BE0701EA04204D10521F348F6F7C0
:10AA4000D3FD03E00921F148F6F7CEFDEF48F6F714
:10AA5000CDFDD8B1701EA0420AD0EC48F6F7C6FD75
:10AA600000F01000102803D00421E848F6F7BCFDE0
:10AA7000002005EB4501E64A02EB8101C87048461B
:10AA8000F8F7BAFA4FF0FF30F6E50DE000BFDF4807
:10AA9000F6F798FD0028FAD1DC48F6F7B8FD3855EE
:10AAA000641CB442C0D3F6E1042D78D100BFD9486C
:10AAB000F6F788FD0028FAD101224146D548F6F77D
:10AAC0007AFD012E29D10721D248F6F78DFDD14814
:10AAD000F6F78CFD58B1002005EB4501CC4A02EB9E
:10AAE0008101C8704846F8F787FAB01EC4E500BF78
:10AAF000C848F6F767FD0028FAD1C648F6F787FD83
:10AB00003870002005EB4501C14A02EB8101C87095
:10AB10004846F8F771FA0020AEE500243BE024B97E
:10AB20000B21BC48F6F760FD0BE0701EA04204D17B
:10AB30000521B848F6F758FD03E00921B548F6F7B6
:10AB400053FDB448F6F752FDD0B1701EA0420AD0B2
:10AB5000B048F6F74BFD00F01000102803D0042198
:10AB6000AC48F6F741FD002005EB4501A84A02EB91
:10AB70008101C8704846F8F73FFA4FF0FF307BE597
:10AB800000BFA448F6F71EFD0028FAD1A148F6F749
:10AB90003EFD3855641CB442C1D37CE1FFE7052D6E
:10ABA00078D100BF9C48F6F70DFD0028FAD10122AC
:10ABB00041469948F6F7FFFC012E29D10721964816
:10ABC000F6F712FD9448F6F711FD58B1002005EB99
:10ABD00045018F4A02EB8101C8704846F8F70CFA2C
:10ABE000B01E49E500BF8C48F6F7ECFC0028FAD10E
:10ABF0008948F6F70CFD3870002005EB4501844AC2
:10AC000002EB8101C8704846F8F7F6F9002033E5F9
:10AC100000243BE024B90B217F48F6F7E5FC0BE06C
:10AC2000701EA04204D105217B48F6F7DDFC03E04D
:10AC300009217948F6F7D8FC7748F6F7D7FCD0B168
:10AC4000701EA0420AD07448F6F7D0FC00F0100045
:10AC5000102803D004217048F6F7C6FC002005EB4D
:10AC600045016B4A02EB8101C8704846F8F7C4F908
:10AC70004FF0FF3000E500BF6748F6F7A3FC00285F
:10AC8000FAD16548F6F7C3FC3855641CB442C1D309
:10AC900001E1FFE7062D78D100BF6048F6F792FC8E
:10ACA0000028FAD1012241465C48F6F784FC012EC7
:10ACB00029D107215948F6F797FC5848F6F796FC32
:10ACC00058B1002005EB4501514A02EB8101C870E3
:10ACD0004846F8F791F9B01ECEE400BF4F48F6F7AA
:10ACE00071FC0028FAD14D48F6F791FC387000202D
:10ACF00005EB4501464A02EB8101C8704846F8F76A
:10AD00007BF90020B8E400243BE024B90B21434840
:10AD1000F6F76AFC0BE0701EA04204D105213F4803
:10AD2000F6F762FC03E009213C48F6F75DFC3B487E
:10AD3000F6F75CFCD0B1701EA0420AD03748F6F797
:10AD400055FC00F01000102803D004213348F6F71A
:10AD50004BFC002005EB45012D4A02EB8101C87038
:10AD60004846F8F749F94FF0FF3085E400BF2B481B
:10AD7000F6F728FC0028FAD12848F6F748FC3855A1
:10AD8000641CB442C1D386E0FFE7072D75D100BF34
:10AD90002348F6F717FC0028FAD101224146204843
:10ADA000F6F709FC012E29D107211D48F6F71CFCF6
:10ADB0001B48F6F71BFC58B1002005EB4501144A6F
:10ADC00002EB8101C8704846F8F716F9B01E53E44B
:10ADD00000BF1348F6F7F6FB0028FAD11048F6F743
:10ADE00016FC3870002005EB4501094A02EB810191
:10ADF000C8704846F8F700F900203DE4002448E018
:10AE000084B90B210648F6F7EFFB17E0003002404B
:10AE1000DC32002000000C4000100C4000200C40F0
:10AE200000300C40701EA04204D10521FE48F6F708
:10AE3000DBFB03E00921FC48F6F7D6FBFA48F6F7FE
:10AE4000D5FBD8B1701EA0420AD0F748F6F7CEFB6A
:10AE500000F01000102803D00421F348F6F7C4FBDB
:10AE6000002005EB4501F14A02EB8101C87048461C
:10AE7000F8F7C2F84FF0FF300AE40CE000BFEA48F0
:10AE8000F6F7A0FB0028FAD1E748F6F7C0FB3855E3
:10AE9000641CB442B4D3002005EB4501E34A02EB45
:10AEA0008101C8704846F8F7A7F8002025E42DE98D
:10AEB000F04104460D4616461F46082C03DB4FF0B2
:10AEC000FF30BDE8F08104EB4400D84911F82000C0
:10AED00010B94FF0FF30F4E700BF04EB4400D34952
:10AEE00001EB8000C0780128F7D004EB440001EBAF
:10AEF000800000790128F0D0002004EB4401CB4A07
:10AF000002F82100FCB900BFC948F6F75BFB002836
:10AF1000FAD104EB4400C54901EB8000407818B930
:10AF2000C348F6F7BEFA02E0C148F6F7BFFAA6B981
:10AF3000C048854208D1FEF72BFA804600224146E0
:10AF4000BB48F6F768FA0CE0FEF722FA80460122C9
:10AF50004146B748F6F75FFA03E03946B448F6F7DA
:10AF600089FA012C2DD100BFB348F6F72BFB00283E
:10AF7000FAD104EB4400AD4901EB8000407818B9E8
:10AF8000AD48F6F78EFA02E0AB48F6F78FFAA6B9AD
:10AF9000A848854208D1FEF7FBF9804600224146C9
:10AFA000A548F6F738FA0CE0FEF7F2F980460122E0
:10AFB0004146A148F6F72FFA03E039469E48F6F7D6
:10AFC00059FA022C2DD100BF9C48F6F7FBFA002855
:10AFD000FAD104EB4400954901EB8000407818B9A0
:10AFE0009648F6F75EFA02E09448F6F75FFAA6B9DB
:10AFF0009048854208D1FEF7CBF9804600224146B1
:10B000008E48F6F708FA0CE0FEF7C2F980460122F6
:10B0100041468A48F6F7FFF903E039468748F6F7D4
:10B0200029FA032C2DD100BF8548F6F7CBFA00286A
:10B03000FAD104EB44007D4901EB8000407818B957
:10B040007F48F6F72EFA02E07D48F6F72FFAA6B908
:10B050007848854208D1FEF79BF980460022414698
:10B060007748F6F7D8F90CE0FEF792F9804601220E
:10B0700041467348F6F7CFF903E039467048F6F7D2
:10B08000F9F9042C2DD100BF6E48F6F79BFA002881
:10B09000FAD104EB4400654901EB8000407818B90F
:10B0A0006848F6F7FEF902E06648F6F7FFF9A6B938
:10B0B0006048854208D1FEF76BF980460022414680
:10B0C0006048F6F7A8F90CE0FEF762F98046012225
:10B0D00041465C48F6F79FF903E039465948F6F7D0
:10B0E000C9F9052C2DD100BF5748F6F76BFA002897
:10B0F000FAD104EB44004D4901EB8000407818B9C7
:10B100005148F6F7CEF902E04F48F6F7CFF9A6B965
:10B110004848854208D1FEF73BF980460022414667
:10B120004948F6F778F90CE0FEF732F9804601223B
:10B1300041464548F6F76FF903E039464248F6F7CD
:10B1400099F9062C2DD100BF4048F6F73BFA0028AC
:10B15000FAD104EB4400354901EB8000407818B97E
:10B160003A48F6F79EF902E03848F6F79FF9A6B993
:10B170003048854208D1FEF70BF98046002241464F
:10B180003248F6F748F90CE0FEF702F98046012252
:10B1900041462E48F6F73FF903E039462B48F6F7CB
:10B1A00069F9072C2DD100BF1F48F6F70BFA0028CC
:10B1B000FAD104EB44001D4901EB8000407818B936
:10B1C0001948F6F76EF902E01748F6F76FF9A6B9D5
:10B1D0001848854208D1FEF7DBF880460022414638
:10B1E0001148F6F718F90CE0FEF7D2F88046012274
:10B1F00041460D48F6F70FF903E039460A48F6F7DD
:10B2000039F904EB4400094901EB8000467004EB76
:10B21000440001EB8000877004EB440001EB8000E8
:10B220008560012014E0000000300C40DC3200207A
:10B2300000000240A08601000010024000200240F1
:10B240000030024000000C4000100C4000200C4078
:10B2500004EB4401024A02F82100002031E600001C
:10B26000DC3200202DE9FE4304460F4690461E4680
:10B270000A9D042C03DA042D01DB102D03DD4FF0B1
:10B28000FF30BDE8FE8300BF04EB4400F74901EB4B
:10B290008000C07A0128F7D0002004EB4401F34A73
:10B2A00002F82100002C48D1F148F6F70BFEF148D6
:10B2B000F6F708FEEF48F6F705FEEE48F6F702FE51
:10B2C000EC48F6F7FFFD40F60F00F6F739F840F6C8
:10B2D0000F40F6F735F841F20F00F6F731F841F27A
:10B2E0000F40F6F72DF804214FF04020F5F7AAFFA4
:10B2F00008214FF04020F5F7A5FF10214FF0402026
:10B30000F5F7A0FF20214FF04020F5F79BFFFEF757
:10B310003FF8814643463A464946D748CDE900655D
:10B32000F6F7EEFBD448F6F716FC00BF02A9D248A8
:10B33000F6F762FC0028F9D1D6E0012C45D1CC48C3
:10B34000401CF6F7BFFDCB48401CF6F7BBFDC948D3
:10B35000401CF6F7B7FDC748001DF6F7B3FDC5481A
:10B36000001DF6F7AFFDC548F5F7EAFFC448F5F74D
:10B37000E7FFC448F5F7E4FFC348F5F7E1FF2021F4
:10B38000C248F5F75FFF1021C048F5F75BFF1021B9
:10B39000BF48F5F757FF2021BD48F5F753FFFDF7EC
:10B3A000F7FF814643463A464946BA48CDE900652B
:10B3B000F6F7A6FBB748F6F7CEFB00BF02A9B548E3
:10B3C000F6F71AFC0028F9D18EE0022C45D1A848E6
:10B3D000801CF6F777FDA748C01CF6F773FDA5485B
:10B3E000C01CF6F76FFDA348C01CF6F76BFDA14823
:10B3F000C01CF6F767FDA848F5F7A2FFA748F5F7C8
:10B400009FFFA748F5F79CFFA648F5F799FF08218D
:10B41000A548F5F717FF0421A348F5F713FF02210C
:10B42000A148F5F70FFF01219F48F5F70BFFFDF746
:10B43000AFFF814643463A4649469C48CDE9006500
:10B44000F6F75EFB9948F6F786FB00BF02A997481E
:10B45000F6F7D2FB0028F9D146E0032C44D184480A
:10B46000C01CF6F72FFD8348401DF6F72BFD8148E1
:10B47000401DF6F727FD7F48401DF6F723FD7D4868
:10B48000401DF6F71FFD8A48F5F75AFF8948F5F782
:10B4900057FF8948F5F754FF8848F5F751FF082111
:10B4A0008748F5F7CFFE04218548F5F7CBFE02214A
:10B4B0008348F5F7C7FE01218148F5F7C3FEFDF784
:10B4C00067FF814643463A4649467E48CDE90065D6
:10B4D000F6F716FB7B48F6F73EFB00BF02A979485A
:10B4E000F6F78AFB0028F9D104EB44005F4901EB31
:10B4F000800080F8098004EB440001EB8000857235
:10B5000004EB440001EB8000466004EB440001EBD7
:10B5100080000772012004EB4401544A02F8210024
:10B520000020AEE6F8B504460E4615460020009011
:10B530000027042C00DA15B94FF0FF30F8BD04EBFA
:10B5400044004A4911F82000012802D04FF0FF3092
:10B55000F4E7012004EB4401444A02EB8101C87284
:10B56000F7F746FD0746ACB900BF69464248F6F713
:10B5700043FB0028F9D131463F48F6F722FB00BFD4
:10B580003D48F6F74CFB0028FAD169463A48F6F7F1
:10B590002AFB46E0012C15D100BF69463D48F6F76D
:10B5A0002BFB0028F9D131463A48F6F70AFB00BFD9
:10B5B0003848F6F734FB0028FAD169463548F6F7E3
:10B5C00012FB2EE0022C15D100BF69463748F6F772
:10B5D00013FB0028F9D131463448F6F7F2FA00BFE0
:10B5E0003248F6F71CFB0028FAD169462F48F6F7D7
:10B5F000FAFA16E0032C14D100BF69463148F6F779
:10B60000FBFA0028F9D131462E48F6F7DAFA00BFE6
:10B610002C48F6F704FB0028FAD169462948F6F7CA
:10B62000E2FA009828703846F7F7E6FC002004EBB1
:10B6300044010E4A02EB8101C87200BF7EE72DE98A
:10B64000FC4704460E46174698460A9D042C03DB29
:10B650004FF0FF30BDE8FC87B5B32878042802DB43
:10B660002878102831DD4FF0FF30F3E73C3300201D
:10B67000001C00F0000800F0008000400F140100E2
:10B680000F1001000F1004000F14040000500040C0
:10B6900000400240009000400F0C03000F08030020
:10B6A0000F0403000F0003000070004000A00040E2
:10B6B0000E0C05000E0805000E0405000E00050026
:10B6C0000050024000B00040FFE704EB4400A449F2
:10B6D00011F8200010B94FF0FF30BBE700BF04EBBA
:10B6E00044009F4901EB8000C07A0128F7D0002078
:10B6F00004EB44019A4A02F821002EB1307804EBA1
:10B70000440102EB8101087237B1387804EB44013F
:10B71000934A02EB81014872B8F1000F07D004EBA5
:10B7200044018F4A02EB8101D8F80000486035B12E
:10B73000287804EB44018A4A02EB8101887264BBD9
:10B7400000BF8848F6F76BFA0028FAD18548F6F76B
:10B7500007FAFDF71DFE814604EB4400804901EB2A
:10B760008000807A04EB44017D4A02EB8101496844
:10B77000CDE9001004EB4400114601EB8000437A50
:10B7800004EB440001EB8000027A49467548F6F765
:10B79000B7F97448F6F7DFF98BE0012C2CD100BF24
:10B7A0007148F6F73CFA0028FAD16F48F6F7D8F955
:10B7B000FDF7EEFD814604EB4400694901EB800092
:10B7C000807A04EB4401664A02EB81014968CDE9C5
:10B7D000001004EB4400114601EB8000437A04EBB7
:10B7E000440001EB8000027A49465F48F6F788F989
:10B7F0005D48F6F7B0F95CE0022C2CD100BF5B4845
:10B80000F6F70DFA0028FAD15848F6F7A9F9FDF72E
:10B81000BFFD814604EB4400514901EB8000807A72
:10B8200004EB44014E4A02EB81014968CDE9001066
:10B8300004EB4400114601EB8000437A04EB440022
:10B8400001EB8000027A49464848F6F759F9474823
:10B85000F6F781F92DE0032C2BD100BF4448F6F711
:10B86000DEF90028FAD14248F6F77AF9FDF790FDA3
:10B87000814604EB44003A4901EB8000807A04EBF6
:10B880004401374A02EB81014968CDE9001004EB1D
:10B890004400114601EB8000437A04EB440001EBC5
:10B8A0008000027A49463248F6F72AF93048F6F71E
:10B8B00052F9012004EB4401294A02F8210000203A
:10B8C000C8E670B504460D46042C02DB4FF0FF308D
:10B8D00070BD04EB4400224911F8200010B94FF06C
:10B8E000FF30F5E774B935B9F72208214FF0402051
:10B8F000F5F795FB32E0082211464FF04020F5F7AE
:10B900008EFB2BE0012C0CD12DB9EF221021194810
:10B91000F5F785FB22E0102211461648F5F77FFB6C
:10B920001CE0022C0CD12DB9FB2204211248F5F7A2
:10B9300076FB13E0042211460F48F5F770FB0DE08B
:10B94000032C0BD12DB9FB2204210C48F5F767FB22
:10B9500004E0042211460948F5F761FB0020B7E72F
:10B960003C330020008000400090004000A00040D8
:10B9700000B0004000500040007000400050024005
:10B9800010B52348F6F79EFA012211462148F5F733
:10B990001FF90823012211461E48F5F7A6F91C4895
:10B9A000F6F790FA012202211A48F5F711F9082357
:10B9B000012202211748F5F798F910BD704710B51C
:10B9C000FFF7FCFFFFF7DCFFF5F7E8FEFDF774FF7C
:10B9D00010BD10B504462CB9012211460D48F5F7EB
:10B9E0001EFB04E0FE2201210A48F5F718FB10BDFA
:10B9F00010B504462CB9022211460648F5F70FFB94
:10BA000004E0FD2202210348F5F709FB10BD000008
:10BA1000030800F00070004010B50024F8F730F97A
:10BA2000F7F7E6FA04460121FE48F7F79DF8FE48CD
:10BA3000C069401CFC49C8612046F7F7DDFAF8F7F9
:10BA400035F910BD10B50024F8F71AF9F7F7D0FA58
:10BA500004460121F548F7F787F8F3488069401C50
:10BA6000F14988612046F7F7C7FAF8F71FF910BDCA
:10BA700010B50024F8F704F9F7F7BAFA04460121E3
:10BA8000EB48F7F771F8E8484069401CE64948611F
:10BA90002046F7F7B1FAF8F709F910BD10B5002400
:10BAA000F8F7EEF8F7F7A4FA04460121E148F7F7B2
:10BAB0005BF8DD480069401CDB4908612046F7F768
:10BAC0009BFAF8F7F3F810BD10B50024F8F7D8F892
:10BAD000F7F78EFA04460121D748F7F745F8D24820
:10BAE000C068401CD049C8602046F7F785FAF8F7CF
:10BAF000DDF810BD10B50024F8F7C2F8F7F778FAB2
:10BB000004460121CD48F7F72FF8C7488068401C4C
:10BB1000C54988602046F7F76FFAF8F7C7F810BDF7
:10BB200010B50024F8F7ACF8F7F762FA04460121E3
:10BB3000C348F7F719F8BC484068401CBA49486048
:10BB40002046F7F759FAF8F7B1F810BD10B5002400
:10BB5000F8F796F8F7F74CFA04460121B948F7F7D9
:10BB600003F8B1480068401CAF4908602046F7F769
:10BB700043FAF8F79BF810BD70B504460D46082C43
:10BB800002DB4FF0FF3070BD34BBAF48F6F79AF9D7
:10BB90002221AC48F6F7B4FEFDF7FAFB4FF47A71B8
:10BBA000B0FBF1F000FB05F63246FF21A548F6F7A1
:10BBB00059FF2320F5F75EFEA4491320FDF7CDF8C9
:10BBC0001320FDF7C0F801219E48F6F7BFFFFF21C3
:10BBD0009C48F6F787FE4CE1012C27D19A48401C7F
:10BBE000F6F770F922219648F6F78AFEFDF7D0FBAA
:10BBF0004FF47A71B0FBF1F000FB05F63246FF21FD
:10BC00008F48F6F72FFF2520F5F734FE90491520D1
:10BC1000FDF7A3F81520FDF796F801218848F6F7FF
:10BC200095FFFF218648F6F75DFE22E1022C27D121
:10BC30008548801CF6F746F922218048F6F760FE19
:10BC4000FDF7A6FB4FF47A71B0FBF1F000FB05F6AF
:10BC50003246FF217948F6F705FF2720F5F70AFE5F
:10BC60007C491720FDF779F81720FDF76CF80121C2
:10BC70007248F6F76BFFFF217048F6F733FEF8E0E5
:10BC8000032C27D17048C01CF6F71CF922216A4802
:10BC9000F6F736FEFDF77CFB4FF47A71B0FBF1F05E
:10BCA00000FB05F63246FF216348F6F7DBFE332042
:10BCB000F5F7E0FD68492320FDF74FF82320FDF755
:10BCC00042F801215C48F6F741FFFF215A48F6F798
:10BCD00009FECEE0042C27D15B48001DF6F7F2F8F0
:10BCE00022215448F6F70CFEFDF752FB4FF47A710F
:10BCF000B0FBF1F000FB05F63246FF214D48F6F7A8
:10BD0000B1FE4F20F5F7B6FD54493F20FDF725F869
:10BD10003F20FDF718F801214648F6F717FFFF21ED
:10BD20004448F6F7DFFDA4E0052C27D14648401D26
:10BD3000F6F7C8F822213E48F6F7E2FDFDF728FBAA
:10BD40004FF47A71B0FBF1F000FB05F63246FF21AB
:10BD50003748F6F787FE5120F5F78CFD4049412022
:10BD6000FCF7FBFF4120FCF7EEFF01213048F6F71E
:10BD7000EDFEFF212E48F6F7B5FD7AE0062C27D11F
:10BD80003148801DF6F79EF822212848F6F7B8FDC5
:10BD9000FDF7FEFA4FF47A71B0FBF1F000FB05F607
:10BDA0003246FF212148F6F75DFE7220F5F762FD6D
:10BDB0002C496220FCF7D1FF6220FCF7C4FF01216F
:10BDC0001A48F6F7C3FEFF211848F6F78BFD50E03E
:10BDD000072C4BD11C48C01DF6F774F822211148DE
:10BDE000F6F78EFDFDF7D4FA4FF47A71B0FBF1F05F
:10BDF00000FB05F63246FF210A48F6F733FE7420B1
:10BE0000F5F738FD18496420FCF7A7FF6420FCF71C
:10BE10009AFF01210348F6F799FEFF210148F6F742
:10BE200061FD26E000100E406C33002000000E4043
:10BE30000050034000400340003003400020034016
:10BE40000010034000000340000400F04DBB000060
:10BE500021BB0000F5BA0000C9BA00009DBA00007D
:10BE600071BA000045BA000019BA00004FF0FF3067
:10BE700089E6002087E60246082A00DC11B94FF067
:10BE8000FF307047024850F8220008600020F8E7B1
:10BE90006C33002070B50024F7F7F2FEF7F7A8F82E
:10BEA00004460121F748F6F7D2FF05462946F54832
:10BEB000F6F7D3FF11E0F348F6F771FFF249087087
:10BEC000F24890F8BD00012807D1F148006820B180
:10BED00008460078EE4909688847EA48F6F753FFB4
:10BEE0000028E8D12046F7F787F8F7F7DFFE70BDA6
:10BEF00070B50024F7F7C4FEF7F77AF8044601217D
:10BF0000E448F6F7A4FF05462946E248F6F7A5FF00
:10BF100011E0E048F6F743FFDF490870DB4890F88E
:10BF2000A500012807D1DD48006820B10846007847
:10BF3000DA4909688847D748F6F725FF0028E8D18D
:10BF40002046F7F759F8F7F7B1FE70BD70B5002439
:10BF5000F7F796FEF7F74CF804460121D048F6F7BC
:10BF600076FF05462946CE48F6F777FF11E0CC4824
:10BF7000F6F715FFCB490870C44890F88D000128EA
:10BF800007D1C948006820B108460078C649096849
:10BF90008847C348F6F7F7FE0028E8D12046F7F7B0
:10BFA0002BF8F7F783FE70BD70B50024F7F768FE35
:10BFB000F7F71EF804460121BC48F6F748FF05468E
:10BFC0002946BA48F6F749FF11E0B848F6F7E7FE08
:10BFD000B7490870AD4890F87500012807D1B548F9
:10BFE000006820B108460078B24909688847AF4820
:10BFF000F6F7C9FE0028E8D12046F6F7FDFFF7F76F
:10C0000055FE70BD70B50024F7F73AFEF6F7F0FF65
:10C0100004460121A848F6F71AFF05462946A64816
:10C02000F6F71BFF11E0A448F6F7B9FEA349087024
:10C03000964890F85D00012807D1A148006820B11A
:10C04000084600789E49096888479B48F6F79BFE9A
:10C050000028E8D12046F6F7CFFFF7F727FE70BD9E
:10C0600070B50024F7F70CFEF6F7C2FF0446012175
:10C070009448F6F7ECFE054629469248F6F7EDFEA1
:10C0800011E09048F6F78BFE8F4908707F4890F8D2
:10C090004500012807D18D48006820B10846007886
:10C0A0008A49096888478748F6F76DFE0028E8D175
:10C0B0002046F6F7A1FFF7F7F9FD70BD70B5002433
:10C0C000F7F7DEFDF6F794FF044601218048F6F706
:10C0D000BEFE054629467E48F6F7BFFE11E07C48C5
:10C0E000F6F75DFE7B490870684890F82D0001283E
:10C0F00007D17948006820B1084600787649096878
:10C1000088477348F6F73FFE0028E8D12046F6F747
:10C1100073FFF7F7CBFD70BD70B50024F7F7B0FDE6
:10C12000F6F766FF044601216C48F6F790FE0546D7
:10C1300029466A48F6F791FE10E06848F6F72FFEA8
:10C14000674908705148407D012807D1654800685B
:10C1500020B1084600786349096888475F48F6F7C8
:10C1600012FE0028E9D12046F6F746FFF7F79EFDBC
:10C1700070BD2DE9F04704460D4616461F46DDF812
:10C180002080082C03DB4FF0FF30BDE8F087B5F5C9
:10C19000965F18D0B5F5165F15D0B5F5615F12D072
:10C1A000B5F5964F0FD0B5F5164F0CD04DF6C02013
:10C1B000854208D0B5F5614F05D0B5F5E13F02D015
:10C1C0004FF0FF30E1E704EB4400304901EBC000E1
:10C1D0004560052E06D0062E0CD0072E12D0082E54
:10C1E00020D117E0002004EB4401284A02EBC101F2
:10C1F00088601AE0202004EB4401244A02EBC101CC
:10C20000886012E0402004EB4401204A02EBC101A7
:10C2100088600AE0602004EB44011C4A02EBC10183
:10C22000886002E04FF0FF30AFE700BF012F02D07F
:10C23000022F10D107E0002004EB4401134A02EB67
:10C24000C101C8600AE0082004EB44010F4A02EB78
:10C25000C101C86002E04FF0FF3096E700BFB8F1BF
:10C26000000F06D0B8F1010F3ED0B8F1020F4BD14C
:10C2700042E0002004EB4401044A02EBC1010861E2
:10C2800045E0000000300140A3000020C400002071
:10C29000C000002000200140A2000020BC000020BF
:10C2A00000100140A1000020B80000200000014063
:10C2B000A0000020B400002000F000409F000020FB
:10C2C000B000002000E000409E000020AC000020F4
:10C2D00000D000409D000020A800002000C00040C9
:10C2E0009C000020A4000020062004EB4401FE4A2C
:10C2F00002EBC10108610AE0022004EB4401FA4AA2
:10C3000002EBC101086102E04FF0FF303DE700BFE2
:10C3100000BF04EB4400F44901EBC000007D01289C
:10C32000F7D004EB440001EBC000407D0128F0D0C1
:10C33000002004EB4401EC4A02F83100002C7DD1CE
:10C34000EA48F5F7BFFDEA48F5F7BCFDE848F5F720
:10C35000B9FD0120F4F7F4FF40F20140F4F7F0FFDB
:10C3600001214FF04020F4F79AFF02214FF04020C6
:10C37000F4F795FFFDF70CF8824604EB4400DA4928
:10C3800001EBC000806804EB4401DFF85CC30CEBF8
:10C39000C101C968084304EB44010CEBC101096900
:10C3A00040EA010304EB4400614601EBC000514642
:10C3B0004268D048F6F754FC04EB4400CA4901EB4C
:10C3C000C0004078022816D1C948F5F77BFD01224C
:10C3D00002214FF04020F4F7FBFB4FF4847301225D
:10C3E00002214FF04020F4F780FCFD2202214FF0A3
:10C3F0004020F4F714FEC0490520FCF7AEFC0520F0
:10C40000FCF7A1FC1520F5F735FA60211520F5F7AA
:10C410000FFA5021B748F6F712FD0121B548F6F79B
:10C4200016FD81464946B348F6F717FD00BFB148EF
:10C43000F6F7B5FC0028FADAE0E3FFE7012C7DD13E
:10C44000AA48401CF5F73EFDA948401CF5F73AFD07
:10C45000A748401CF5F736FD4FF00110F4F770FFC8
:10C46000A648F4F76DFF0121A548F4F718FF022153
:10C47000A348F4F714FFFCF78BFF824604EB44005B
:10C48000994901EBC000806804EB4401DFF858C211
:10C490000CEBC101C968084304EB44010CEBC1017A
:10C4A000096940EA010304EB4400614601EBC00066
:10C4B000514642689348F6F7D3FB8D480930F5F7AB
:10C4C00001FD012210219048F4F782FB0C23012288
:10C4D00010218D48F4F709FC04EB4400824901EB7C
:10C4E000C0004078022819D181480A30F5F7EAFCEB
:10C4F000EF2210218448F4F792FD0122114683486F
:10C50000F4F766FB0C23012211468048F4F7EDFB9B
:10C51000FE2201217D48F4F782FD04E0102211463D
:10C520007948F4F77CFD7A490620FCF716FC0620D2
:10C53000FCF709FC1620F5F79DF900E017E06021F3
:10C540001620F5F775F950216E48F6F778FC0121B1
:10C550006C48F6F77CFC814649466A48F6F77DFC54
:10C5600000BF6848F6F71BFC0028FADA46E3022C05
:10C570007CD15E48801CF5F7A5FC5D48F5F7A2FC70
:10C580005B48F5F79FFC41F60100F4F7D9FE41F650
:10C590000140F4F7D5FE40214FF04020F4F77FFE34
:10C5A00080214FF04020F4F77AFEFCF7F1FE82463E
:10C5B00004EB44004C4901EBC000806804EB4401EB
:10C5C000DFF824C10CEBC101C968084304EB440146
:10C5D0000CEBC101096940EA010304EB4400614628
:10C5E00001EBC000514642684A48F6F739FB04EBBC
:10C5F00044003D4901EBC0004078022813D13C487B
:10C60000401DF5F75FFC012210214348F4F7E0FAE2
:10C610000C23012210214048F4F767FBEF22102180
:10C620003D48F4F7FCFC3D492120FCF796FB212016
:10C63000FCF789FB3120F5F71DF960213120F5F772
:10C64000F7F850213348F6F7FAFB01213148F6F7A5
:10C65000FEFB814649462F48F6F7FFFB00BF2D48F9
:10C66000F6F79DFB0028FADAC8E2FFE7032C7CD13D
:10C670001E48C01CF5F726FC1D48F5F723FC1C4896
:10C68000F5F720FC41F20100F4F75AFE41F20140B7
:10C69000F4F756FE10214FF04020F4F700FE202161
:10C6A0004FF04020F4F7FBFDFCF772FE824604EBEE
:10C6B00044000D4901EBC000806804EB4401DFF841
:10C6C00028C00CEBC101C968084304EB44010CEB22
:10C6D000C101096940EA010304EB4400614601EB32
:10C6E000C000514642681BE0C4000020001800F062
:10C6F000000800F000C0004019C100000104010062
:10C700000050004000D000400010064000200640CD
:10C71000BDC0000000E000400050024061C00000C9
:10C72000FE48F6F79DFA04EB4400FD4901EBC0001A
:10C730004078022816D1FB48F5F7C4FB01220221FC
:10C740004FF04020F4F744FA4FF4847301220221A1
:10C750004FF04020F4F7C9FAFD2202214FF04020AB
:10C76000F4F75DFCF049382000E01FE0FCF7F5FA33
:10C770003820FCF7E8FA4820F5F77CF860214820DB
:10C78000F5F756F85021E548F6F759FB0121E34843
:10C79000F6F75DFB81464946E048F6F75EFB00BFD1
:10C7A000DE48F6F7FCFA0028FADA27E2042C7ED1FC
:10C7B000DE48F5F787FBDB48F5F784FBD948F5F74A
:10C7C00081FB40F60100F4F7BBFD40F60140F4F7B1
:10C7D000B7FD04214FF04020F4F761FD08214FF030
:10C7E0004020F4F75CFDFCF7D3FD824604EB4400E7
:10C7F000CB4901EBC000806804EB4401DFF820C3A3
:10C800000CEBC101C968084304EB44010CEBC10106
:10C81000096940EA010304EB4400614601EBC000F2
:10C8200051464268C248F6F71BFA04EB4400BC4983
:10C8300001EBC0004078022816D1BA48F5F742FB58
:10C84000012202214FF04020F4F7C2F94FF4847323
:10C85000012202214FF04020F4F747FAFD22022185
:10C860004FF04020F4F7DBFBB2493920FCF775FAB2
:10C870003920FCF768FA4920F4F7FCFF60214920D1
:10C88000F4F7D6FF5021AA48F6F7D9FA0121A848B3
:10C89000F6F7DDFA81464946A548F6F7DEFA00BF0D
:10C8A000A348F6F77CFA0028FADAA7E1FFE7052C9F
:10C8B0007DD19E48401CF5F705FB9A48801CF5F792
:10C8C00001FB9848801CF5F7FDFA9B48F4F738FD0A
:10C8D0009A48F4F735FD40219948F4F7E0FC8021AF
:10C8E0009748F4F7DCFCFCF753FD824604EB440068
:10C8F0008B4901EBC000806804EB4401DFF820C2E3
:10C900000CEBC101C968084304EB44010CEBC10105
:10C91000096940EA010304EB4400614601EBC000F1
:10C92000514642688748F6F79BF904EB44007C497E
:10C9300001EBC0004078022816D17A48F5F7C2FA18
:10C94000012202214FF04020F4F742F94FF48473A2
:10C95000012202214FF04020F4F7C7F9FD22022105
:10C960004FF04020F4F75BFB77493A20FCF7F5F9EC
:10C970003A20FCF7E8F94A20F4F77CFF60214A20CE
:10C98000F4F756FF50216F48F6F759FA01216D4828
:10C99000F6F75DFA814649466A48F6F75EFA00BF47
:10C9A0006848F6F7FCF90028FADA27E1FFE7062CD9
:10C9B0007DD15E48801CF5F785FA5A480D30F5F7B1
:10C9C00081FA58480D30F5F77DFA6048F4F7B8FC65
:10C9D0005F48F4F7B5FC01215E48F4F760FC0221E2
:10C9E0005C48F4F75CFCFCF7D3FC824604EB4400A3
:10C9F0004B4901EBC000806804EB4401DFF820C123
:10CA00000CEBC101C968084304EB44010CEBC10104
:10CA1000096940EA010304EB4400614601EBC000F0
:10CA2000514642684C48F6F71BF904EB44003C4978
:10CA300001EBC0004078022816D13A48F5F742FAD7
:10CA4000012202214FF04020F4F7C2F84FF4847322
:10CA5000012202214FF04020F4F747F9FD22022184
:10CA60004FF04020F4F7DBFA3C493B20FCF775F926
:10CA70003B20FCF768F94B20F4F7FCFE60214B20CB
:10CA8000F4F7D6FE50213448F6F7D9F9012132489F
:10CA9000F6F7DDF9814649462F48F6F7DEF900BF83
:10CAA0002D48F6F77CF90028FADAA7E0FFE7072C13
:10CAB0007ED11E48C01CF5F705FA1A48801CF5F710
:10CAC00001FA1848801CF5F7FDF92548F4F738FC01
:10CAD0002448F4F735FC10211948F4F7E0FB202135
:10CAE0001748F4F7DCFBFCF753FC824604EB4400E8
:10CAF0000B4901EBC000806804EB4401DFF820C063
:10CB00000CEBC101C968084304EB44010CEBC10103
:10CB1000096940EA010304EB440025E000F000400D
:10CB2000C4000020000800F005C00000041800F058
:10CB300000000140A9BF000001180200011C020012
:10CB400000600040001001404DBF000001000D00DA
:10CB500001040D000050064000200140F1BE00001D
:10CB60000110020001140200614601EBC0005146B1
:10CB70004268FB48F6F774F804EB4400F94901EB0E
:10CB8000C0004078022818D1F748F5F79BF9012238
:10CB900002214FF04020F4F71BF84FF48473012278
:10CBA00002214FF04020F4F7A0F8FD22022100E01E
:10CBB00024E04FF04020F4F732FAEC493C20FCF737
:10CBC000CCF83C20FCF7BFF84C20F4F753FE602172
:10CBD0004C20F4F72DFE5021E148F6F730F9012101
:10CBE000DF48F6F734F981464946DD48F6F735F96E
:10CBF00000BFDB48F6F7D3F80028FADA012004EB8F
:10CC00004401D84A02F831000020FFF7BEBA2DE9EE
:10CC1000F04104460E4617460025A846082C02DBC4
:10CC2000681EBDE8F08104EB4400CE4911F83000E5
:10CC3000012802D04FF0FF30F3E700BF04EB4400BF
:10CC4000C84901EBC000007D0128F7D0012004EBAA
:10CC50004401C44A02EBC1010875F6F7C9F98046E0
:10CC600054BB04EB4400BF4901EBC00040780228EC
:10CC700005D1022211464FF04020F4F7D0F904E02C
:10CC8000715DBB48F6F7A8F86D1CBD42F8D300BF34
:10CC9000B748F6F7B3F80028FAD104EB4400B149DD
:10CCA00001EBC0004078022805D1FD2202214FF09F
:10CCB0004020F4F7B4F935E1012C28D104EB44000D
:10CCC000A84901EBC0004078022804D10122114696
:10CCD000A848F4F7A4F904E0715DA748F6F77CF8DA
:10CCE0006D1CBD42F8D300BFA348F6F787F80028B3
:10CCF000FAD104EB44009B4901EBC00040780228C4
:10CD0000D9D1FE2201219B48F4F789F90AE1022CCE
:10CD100028D104EB4400934901EBC000407802287D
:10CD200004D1102211469548F4F779F904E0715DB9
:10CD30009348F6F751F86D1CBD42F8D300BF9048F8
:10CD4000F6F75CF80028FAD104EB4400854901EBC2
:10CD5000C00040780228AED1EF2210218748F4F7B6
:10CD60005EF9DFE0032C2AD104EB44007D4901EB9E
:10CD7000C0004078022805D1022211464FF0402021
:10CD8000F4F74DF904E0715D7E48F6F725F86D1C67
:10CD9000BD42F8D300BF7B48F6F730F80028FAD13F
:10CDA00004EB44006F4901EBC00040780228ADD18C
:10CDB000FD2202214FF04020F4F731F9B2E0042CBB
:10CDC0002AD104EB4400674901EBC00040780228F7
:10CDD00005D1022211464FF04020F4F720F904E07B
:10CDE000715D6948F5F7F8FF6D1CBD42F8D300BFCF
:10CDF0006548F6F703F80028FAD104EB44005949D6
:10CE000001EBC0004078022805D1FD2202214FF03D
:10CE10004020F4F704F985E0052C2AD104EB440006
:10CE2000504901EBC0004078022805D1022211468A
:10CE30004FF04020F4F7F3F804E0715D5348F5F744
:10CE4000CBFF6D1CBD42F8D300BF5048F5F7D6FFAD
:10CE50000028FAD104EB4400424901EBC0004078BD
:10CE600002285FD1FD2202214FF04020F4F7D7F8CD
:10CE700058E0062C2AD104EB44003A4901EBC000EB
:10CE80004078022805D1022211464FF04020F4F7E5
:10CE9000C6F804E0715D3E48F5F79EFF6D1CBD428B
:10CEA000F8D300BF3A48F5F7A9FF0028FAD104EB00
:10CEB00044002C4901EBC0004078022832D1FD2209
:10CEC00002214FF04020F4F7AAF82BE0072C29D1DB
:10CED00004EB4400234901EBC0004078022805D14F
:10CEE000022211464FF04020F4F799F804E0715DFA
:10CEF0001B48F5F771FF6D1CBD42F8D300BF184801
:10CF0000F5F77CFF0028FAD104EB4400154901EB4A
:10CF1000C0004078022805D1FD2202214FF04020B8
:10CF2000F4F77DF84046F6F767F8002004EB44017B
:10CF30000C4A02EBC101087500BF72E610B502464B
:10CF4000082A00DA11B94FF0FF3010BD02EB4200A1
:10CF5000044B13F8300001281CD04FF0FF30F4E7E9
:10CF600000300140C4000020000800F095BE000021
:10CF700000C000400020064000D0004000500240A9
:10CF800000E0004000F000400000014000100140BF
:10CF90000020014000BF02EB4200FE4B03EBC0004B
:10CFA000407D0128F7D0012002EB4203F94C04EB4D
:10CFB000C3035875082A1DD2DFE802F004070A0DE2
:10CFC00010131619F448016017E0F448016014E0EA
:10CFD000F348016011E0F34801600EE0F24801609F
:10CFE0000BE0F248016008E0F148016005E0F1481B
:10CFF000016002E04FF0FF30A7E700BF0020A4E788
:10D000000146082902DB4FF0FF30704701EB410079
:10D01000E04A12F83000012802D04FF0FF30F4E768
:10D02000082925D2DFE801F004080C1014181C2090
:10D030000020D94A10601EE00020D84A10601AE093
:10D040000020D74A106016E00020D64A106012E097
:10D050000020D54A10600EE00020D44A10600AE09B
:10D060000020D34A106006E00020D24A106002E09F
:10D070004FF0FF30C9E700BF002001EB4102C54B74
:10D0800003EBC202507500BFBFE72DE9F04704462D
:10D090000D4616461F46DDF82080082C03DB4FF0B6
:10D0A000FF30BDE8F087B5F5965F18D0B5F5165F8F
:10D0B00015D0B5F5615F12D0B5F5964F0FD0B5F527
:10D0C000164F0CD04DF6C020854208D0B5F5614F03
:10D0D00005D0B5F5E13F02D04FF0FF30E1E704EBBA
:10D0E0004400AC4901EBC0004560052E06D0062E79
:10D0F0000CD0072E12D0082E20D117E0002004EB10
:10D100004401A44A02EBC10188601AE0202004EB2C
:10D110004401A04A02EBC101886012E0402004EB08
:10D1200044019C4A02EBC10188600AE0602004EBE4
:10D130004401984A02EBC101886002E04FF0FF30E1
:10D14000AFE700BF012F02D0022F10D107E000206F
:10D1500004EB44018F4A02EBC101C8600AE00020E1
:10D1600004EB44018B4A02EBC101C86002E04FF0BE
:10D17000FF3096E700BFB8F1000F06D0B8F1010FFD
:10D180000BD0B8F1020F18D10FE0002004EB4401DE
:10D19000804A02EBC101086112E0062004EB440161
:10D1A0007C4A02EBC10108610AE0022004EB440161
:10D1B000784A02EBC101086102E04FF0FF3070E7EE
:10D1C00000BF00BF04EB4400724901EBC000407D8A
:10D1D0000128F7D004EB440001EBC000007D0128DA
:10D1E000F0D0002004EB44016A4A02F8310014BB7D
:10D1F000FCF7CEF8814604EB4400664901EBC00021
:10D20000806804EB4401DFF88CC10CEBC101C968F4
:10D21000084304EB44010CEBC101096940EA010336
:10D2200004EB4400614601EBC00049464268624895
:10D23000F5F716FD1EE1012C22D1FCF7A9F8814675
:10D2400004EB4400534901EBC000806804EB440147
:10D25000DFF840C10CEBC101C968084304EB44018D
:10D260000CEBC101096940EA010304EB440061468B
:10D2700001EBC000494642685048F5F7F1FCF9E07F
:10D28000022C22D1FCF784F8814604EB440041498A
:10D2900001EBC000806804EB4401DFF8F8C00CEB40
:10D2A000C101C968084304EB44010CEBC1010969E1
:10D2B00040EA010304EB4400614601EBC00049462B
:10D2C00042683F48F5F7CCFCD4E0032C22D1FCF7B0
:10D2D0005FF8814604EB44002E4901EBC0008068F2
:10D2E00004EB4401DFF8ACC00CEBC101C968084392
:10D2F00004EB44010CEBC101096940EA010304EBB2
:10D300004400614601EBC000494642682D48F5F7EC
:10D31000A7FCAFE0042C22D1FCF73AF8814604EBDD
:10D3200044001C4901EBC000806804EB4401DFF8B5
:10D3300064C00CEBC101C968084304EB44010CEB69
:10D34000C101096940EA010304EB4400614601EBB5
:10D35000C000494642681C48F5F782FC8AE0052C6B
:10D360003FD1FCF715F8814604EB4400094901EB75
:10D37000C000806804EB4401DFF818C00CEBC10169
:10D38000C968084304EB44010CEBC101096940EA98
:10D3900001031BE0C4000020A4000020A80000201E
:10D3A000AC000020B0000020B4000020B800002035
:10D3B000BC000020C000002000C0004000D00040A1
:10D3C00000E0004000F000400000014004EB440099
:10D3D000614601EBC000494642682A48F5F740FC27
:10D3E00048E0062C22D1FBF7D3FF814604EB440032
:10D3F000254901EBC000806804EB4401DFF888C0D8
:10D400000CEBC101C968084304EB44010CEBC101FA
:10D41000096940EA010304EB4400614601EBC000E6
:10D42000494642681948F5F71BFC23E0072C21D137
:10D43000FBF7AEFF814604EB4400134901EBC0004B
:10D44000806804EB4401DFF840C00CEBC101C968FF
:10D45000084304EB44010CEBC101096940EA0103F4
:10D4600004EB4400614601EBC000494642680848AD
:10D47000F5F7F6FB012004EB4401034A02F8310002
:10D4800000200EE600100140C400002000200140F2
:10D490000030014010B54FF08040F5F747FDFBF735
:10D4A00077FF044621464FF08040F5F74BFD4FF0E3
:10D4B0008040F5F737FD10BD10B5F6F7E1FB2448C5
:10D4C0000078401C22490870084600781E2802DDBA
:10D4D0000120204908701F48007828B94FF080408B
:10D4E000F5F757FDFFF7D6FFF6F7E0FB10BD10B5D7
:10D4F0004FF07040F4F7E6FC2220F4F7BBF94FF050
:10D500008040F5F713FDFBF743FF044621464FF03B
:10D510008040F5F717FD4FF08040F5F7F9FC4FF02C
:10D520008040F5F7FFFC0C491220FBF716FC122097
:10D53000FBF709FC4FF08040F5F7E5FC10BD00203B
:10D5400003490870704701200249087070470000C5
:10D550008401002085010020B9D40000F8B50446FC
:10D560000D4608208DF800008DF80150A07D0223A3
:10D570006A466F21E769B84746B2002E02DA4FF0DB
:10D58000FF30F8BD0020FCE7F8B504460D46072043
:10D590008DF800008DF80150A07D02236A466F21AE
:10D5A000E769B84746B2002E02DA4FF0FF30F8BD07
:10D5B0000020FCE710B5044614B94FF0FF3010BD51
:10D5C000A06908B1E06910B94FF0FF30F7E790218A
:10D5D0002046FFF7D9FF00212046FFF7BFFF0020BC
:10D5E000EDE77CB504460520019000200090A07D69
:10D5F000012301AA6F21E669B04745B2002D02DA86
:10D600004FF0FF307CBDA07D01236A466F21A669E3
:10D61000B04745B2002D02DA4FF0FF30F2E79DF837
:10D62000000000F00F009DF80010090901EB8101D6
:10D6300000EB4100FC49098801EBC10202EB01113A
:10D6400000EB810020810020DCE77CB5044604204B
:10D65000019000200090A07D012301AA6F21E669BE
:10D66000B04745B2002D02DA4FF0FF307CBDA07DFF
:10D6700001236A466F21A669B04745B2002D02DA40
:10D680004FF0FF30F2E79DF8000000F00F009DF82A
:10D690000010C1F3001101EB810100EB4101E171C8
:10D6A0000020E3E77CB504460320019000200090B1
:10D6B000A07D012301AA6F21E669B04745B2002D84
:10D6C00002DA4FF0FF307CBDA07D01236A466F2156
:10D6D000A669B04745B2002D02DA4FF0FF30F2E7FD
:10D6E0009DF8000000F00F009DF80010C1F301113B
:10D6F00001EB810100EB4101A1710020E3E77CB562
:10D7000004460220019000200090A07D012301AA80
:10D710006F21E669B04745B2002D02DA4FF0FF30C5
:10D720007CBDA07D01236A466F21A669B04745B242
:10D73000002D02DA4FF0FF30F2E79DF8000000F014
:10D740000F009DF80010C1F3011101EB810100EB06
:10D75000410161710020E3E77CB50446012001909E
:10D7600000200090A07D012301AA6F21E669B04747
:10D7700045B2002D02DA4FF0FF307CBDA07D0123C1
:10D780006A466F21A669B04745B2002D02DA4FF014
:10D79000FF30F2E79DF8000000F00F009DF8001048
:10D7A000C1F3021101EB810100EB41012171002065
:10D7B000E3E77CB50446002001900090A07D0123A2
:10D7C00001AA6F21E669B04745B2002D02DA4FF099
:10D7D000FF307CBDA07D01236A466F21A669B0475A
:10D7E00045B2002D02DA4FF0FF30F2E79DF800005D
:10D7F00000F00F009DF80010C1F3021101EB810150
:10D8000000EB4101E1700020E3E770B505462846D2
:10D81000FFF7CFFF44B2002C02DA4FF0FF3070BDAB
:10D820002846FFF799FF44B2002C02DA4FF0FF3090
:10D83000F5E72846FFF763FF44B2002C02DA4FF009
:10D84000FF30ECE72846FFF72DFF44B2002C02DA48
:10D850004FF0FF30E3E72846FFF7F7FE44B2002C15
:10D8600002DA4FF0FF30DAE72846FFF7BAFE44B29B
:10D87000002C02DA4FF0FF30D1E70020CFE7F8B5F7
:10D880000446608A642190FBF1F067490880608A51
:10D89000098801EBC10202EB0111A0EB810060825B
:10D8A00005208DF80000608A0A2190FBF1F201FB4F
:10D8B00012010A2290FBF2F041EA0010C0B28DF88A
:10D8C0000100A07D02236A466F21E669B04745B298
:10D8D000002D02DA4FF0FF30F8BD0020FCE7F8B56C
:10D8E000044604208DF80000607C0A2190FBF1F2D0
:10D8F00001FB12010A2290FBF2F041EA0010C0B2D3
:10D900008DF80100A07D02236A466F21E669B047C9
:10D9100045B2002D02DA4FF0FF30F8BD0020FCE7E1
:10D92000F8B5044603208DF80000207C0A2190FB06
:10D93000F1F201FB12010A2290FBF2F041EA001021
:10D94000C0B28DF80100A07D02236A466F21E6690E
:10D95000B04745B2002D02DA4FF0FF30F8BD00208D
:10D96000FCE7F8B5044602208DF80000E07B0A21B0
:10D9700090FBF1F201FB12010A2290FBF2F041EA66
:10D980000010C0B240F080008DF80100A07D02239D
:10D990006A466F21E669B04745B2002D02DA4FF0C2
:10D9A000FF30F8BD0020FCE7F8B5044601208DF8F3
:10D9B0000000A07B0A2190FBF1F201FB12010A2278
:10D9C00090FBF2F041EA0010C0B28DF80100A07D9A
:10D9D00002236A466F21E669B04745B2002D02DA9C
:10D9E0004FF0FF30F8BD0020FCE7F8B504460020FA
:10D9F0008DF80000607B0A2190FBF1F201FB12011F
:10DA00000A2290FBF2F041EA0010C0B28DF801004A
:10DA1000A07D02236A466F21E669B04745B2002D1A
:10DA200004DA4FF0FF30F8BD860100200020FAE74D
:10DA300070B505462846FFF7D8FF44B2002C02DA3D
:10DA40004FF0FF3070BD2846FFF7AEFF44B2002C08
:10DA500002DA4FF0FF30F5E72846FFF782FF44B2C5
:10DA6000002C02DA4FF0FF30ECE72846FFF758FFB2
:10DA700044B2002C02DA4FF0FF30E3E72846FFF70C
:10DA80002EFF44B2002C02DA4FF0FF30DAE72846CE
:10DA9000FFF7F5FE44B2002C02DA4FF0FF30D1E779
:10DAA0000020CFE730B589B0044600254FF6FF705F
:10DAB00005903EA103C9CDE903010020009001902B
:10DAC000029014B9401E09B030BD20788DF80C00CA
:10DAD00005AA062103A8A3699847BDF81400000A07
:10DAE0008DF81300BDF81400C0B28DF812000821A3
:10DAF00003A82269904709216846E26890470546D5
:10DB0000002D02DA4FF0FF30DDE79DF800002178AC
:10DB1000884207D19DF80100032803D19DF8020037
:10DB2000042802D04FF0FF30CDE74FF6FF7005908C
:10DB300005AA07216846A36998479DF807009DF844
:10DB4000081040EA0120BDF81410884202D04FF0BE
:10DB5000FF30B8E79DF804009DF8031040EA01206B
:10DB6000069006980790BDF91C0000EE100AB8EE6A
:10DB7000C00AF2EE040A80EE201A84ED021A9DF823
:10DB800006009DF8051040EA0120069006980890CE
:10DB9000BDF9200000EE100AB8EEC00AF2EE040A49
:10DBA00080EE201A84ED011A00208CE701030000AA
:10DBB0000002C40B1CB5044614B9F748019001E0FB
:10DBC000F6480190002001AB024601460090032078
:10DBD000FDF735FD1CBD38B50446002000906A46AF
:10DBE00021460320FDF79EFC9DF8000038BD10B5CE
:10DBF000044621460320FDF764FE10BD10B5012048
:10DC0000FFF7F5FFFF20FFF7E6FF10BD38B5002452
:10DC100000BFFF20FFF7DFFF0546FF2D01D10020E9
:10DC200038BD641C6FF07F40B4FBF0F100FB114085
:10DC300050B90820DA4B0022114600900320FDF76E
:10DC400011FB0020FFF7D3FF6FF070408442E0D358
:10DC50000120E5E710B50020FFF7C9FFFFF7D6FF69
:10DC600008B9002010BDFFF7C9FF0120FAE72DE930
:10DC7000F04105460C4617464FF00008FFF7BEFF7F
:10DC8000FFF7E8FF10B1FF20BDE8F08145F040004C
:10DC9000FFF7A1FF200EFFF79EFFC4F30740FFF739
:10DCA0009AFFC4F30720FFF796FFE0B2FFF793FF58
:10DCB0003846FFF790FF0C2D02D1FF20FFF78BFFB6
:10DCC0004FF01F0800BFFF20FFF785FF064606F054
:10DCD000800030B1B8F10000A8F1010101F0FF08A7
:10DCE000F1D13046D0E77CB50820AD4B002211467B
:10DCF00000900320FDF7B6FA0020FFF778FF002020
:10DD0000FFF758FF002505E0FF20FFF764FF0446FA
:10DD1000681C85B2642DF7DB4020FFF75CFF002014
:10DD2000FFF759FF0020FFF756FF0020FFF753FFD2
:10DD30000020FFF750FF9520FFF74DFF142600BF8E
:10DD4000952200210846FFF792FF0446012C04D0DB
:10DD5000301EA6F101018EB2F2D100209149087067
:10DD6000012C4AD187224FF4D5710820FFF77FFF9D
:10DD7000012847D1002506E0FF20FFF72CFF01A96D
:10DD80004855681C85B2042DF6DB9DF80600012875
:10DD900079D19DF80700AA2875D14FF6FE7600BF0D
:10DDA000012200213720FFF762FF0122910729207D
:10DDB000FFF75DFF044624B1301EA6F101018EB2CB
:10DDC000EED1002E5FD0012200213A20FFF74FFF55
:10DDD000002858D1002506E0FF20FFF7FCFE01A92E
:10DDE0004855681C85B2042DF6DB9DF8040000F050
:10DDF000400018B106206B49087044E004206949CE
:10DE0000087040E0012200213720FFF730FF012297
:10DE100000212920FFF72BFF0446012C17DC0220EC
:10DE2000604908704FF6FE7600BF012200213720BE
:10DE3000FFF71DFF012200212920FFF718FF0446EC
:10DE4000BCB1301EA6F101018EB2EED111E001206D
:10DE5000544908704FF6FE7600BF0122002110469B
:10DE6000FFF705FF044624B1301EA6F101018EB272
:10DE7000F3D12EB1012251021020FFF7F8FE10B1AC
:10DE8000002048490870FFF7B9FE0120FFF792FE15
:10DE90004448007808B100207CBD0CB12046FBE767
:10DEA000AA20F9E770B505464FF6FF7401E0601E41
:10DEB00084B2FF20FFF78FFEA84201D0002CF6D1DC
:10DEC0000CB9FF2070BD0020FCE770B504460D467C
:10DED000FE20FFF7E7FF08B1012070BD04E0FF203E
:10DEE000FFF779FE2070641C281EA5F101018DB298
:10DEF000F5D1FF20FFF76FFEFF20FFF76CFE00203B
:10DF0000EBE72DE9F04106460F4615462548007817
:10DF1000062800D07F02012D0CD1012239461120A4
:10DF2000FFF7A5FE0446FCB969023046FFF7CDFFB6
:10DF3000044619E0012239461220FFF798FE0446F4
:10DF400000BF4FF400713046FFF7BFFF044606F5EF
:10DF50000076681EC0B2051E01D0002CF1D001224F
:10DF600000210C20FFF783FEFFF748FE2046BDE8A6
:10DF7000F0812DE9F04106460D46FFF747FE0746C2
:10DF800017B10120BDE8F0812846FFF724FEFD2DE2
:10DF900022D000240DE00000400D0300003FAB0143
:10DFA00040420F0088010020305DFFF714FE601C26
:10DFB00084B2B4F5007FF7DBFF20FFF70CFEFF20F3
:10DFC000FFF709FEFF20FFF706FE074607F01F00D8
:10DFD000052801D00220D5E70020D3E72DE9F04144
:10DFE00006460F4615464A480078062800D07F02AC
:10DFF000012D0CD1012239461820FFF738FE0446C6
:10E000006CBBFE213046FFF7B4FF044627E04048D2
:10E010000078012809D0012200213720FFF727FED0
:10E02000012229461720FFF722FE01223946192036
:10E03000FFF71DFE044694B900BFFC213046FFF7F0
:10E0400098FF044606F50076681EC0B2051E01D092
:10E05000002CF2D0FD210020FFF78BFF0446FFF7D4
:10E06000CDFD2046BDE8F08170B5054601220021B6
:10E070000920FFF7FCFD044624B910212846FFF7CC
:10E0800024FF0446FFF7BAFD0CB1012070BD00204B
:10E09000FCE770B510211F4808F05FF91D48FFF735
:10E0A000E3FF08B1002070BD1A48007800F0C000FE
:10E0B000402809D11748407A1649097A00EB012017
:10E0C000401C84B2A50220E01248407900F00F0005
:10E0D0001049897A00EBD1100E49497A01F0030109
:10E0E00000EB4100861C0B48007A80110949C97970
:10E0F00000EB81000749897901F0030100EB8120E1
:10E10000441CA6F1090004FA00F52846CBE70000FC
:10E11000880100208C33002010B500231A46664980
:10E120000120FBF717FC0446002C02DA4FF0FF3009
:10E1300010BD012061498875614888616148C861E6
:10E140000846FFF737FA0446002C02DA4FF0FF309A
:10E15000EEE70020ECE770B50446E18857484182BD
:10E160006179417421790174E178C173A178817377
:10E1700061784173FFF75CFC0546002D02DA4FF031
:10E18000FF3070BD0020FCE770B504464B48FFF738
:10E190003CFB0546002D02DA4FF0FF3070BD4748CA
:10E1A0000089E0804548C0796071444880792071D9
:10E1B00042484079E07041480079A0703F48C078FB
:10E1C00060700020EAE770B504463C48FFF71DFB8D
:10E1D0000546002D02DA4FF0FF3070BDE188374868
:10E1E0000089814201DD0220F7E7E1883348008998
:10E1F000814201DA0120F0E761793048C07981423B
:10E2000001DD0220E9E761792C48C079814201DA19
:10E210000120E2E7217929488079814201DD02204D
:10E22000DBE7217925488079814201DA0120D4E7B2
:10E23000E17822484079814201DD0220CDE7E17892
:10E240001E484079814201DA0120C6E7A1781B48C7
:10E250000079814201DD0220BFE7A17817480079EB
:10E26000814201DA0120B8E761781448C078814220
:10E2700001DD0220B1E761781048C078814201DAFF
:10E280000120AAE70020A8E710B58CB00446E0887A
:10E29000A0F26C7006906079401E05902079049081
:10E2A000E0780390A07802906078019001A808F0CF
:10E2B000FCF80CB010BD0000801A06009C33002052
:10E2C00061A60000259D0000014609B900207047A5
:10E2D0000120FCE770B5054665B9FFF704FD04466B
:10E2E00034B10120FFF766FCFF20FFF774FC01E06A
:10E2F000002070BD00BF0120FBE72DE9F04106467C
:10E300000F4690461C4614B90420BDE8F0816EB952
:10E31000E2B241463846FFF7F4FD054625B1FF203D
:10E32000FFF759FC0120F0E70020EEE70420ECE7BE
:10E330002DE9F04105460E461746984665B908F0A6
:10E34000FF0239463046FFF749FE044614B9002063
:10E35000BDE8F0810120FBE70420F9E72DE9F04159
:10E3600006460F4615462EBB37B1012F1AD0022F95
:10E370000FD0032F1BD111E00020FFF738FCFFF76F
:10E3800045FC08B9002400E001240120FFF72FFC20
:10E390000FE04FF40070288000240AE00820288055
:10E3A000002406E0FFF775FE2860002401E0042445
:10E3B00000BF00E001242046BDE8F0810EB56846AC
:10E3C000FFF7E2FEC0B9BDF80600A0F2BC7040063F
:10E3D0009DF8051040EA41509DF8041040EA0140C4
:10E3E0009DF8031040EAC1209DF8021040EA411058
:10E3F0009DF8011008430EBD0048FCE72252A556C7
:10E40000014648780A7842EA002070470146C878F9
:10E410008A7842EA00204A7842EA00200A7842EAF2
:10E420000020704700F8011B091200F8011B70471B
:10E4300000F8011B090A00F8011B090A00F8011B7A
:10E44000090A00F8011B704730B503460C463AB183
:10E4500000BF14F8015B03F8015B551E2A1EF8D1BA
:10E4600030BD10B5034600BF03F8011B541E221E29
:10E47000FAD110BDF0B503461D460C46002000BF82
:10E4800015F8017B14F801CBA7EB0C00561E321EC9
:10E4900001D00028F4D0F0BD024600E0521C1078F4
:10E4A00010B110788842F9D110787047014609B14F
:10E4B000002070470020FCE7014609B100207047AA
:10E4C0000020FCE72DE9F0410646356815F8014BC0
:10E4D0002046FFF7EBFF60B115F8017B3846FFF7E8
:10E4E000EBFF18B94FF0FF30BDE8F08107EB0420D7
:10E4F00084B24CB140F2B511204603F056FA0446FE
:10E5000014B94FF0FF30EFE7A04635604046EBE727
:10E510002DE9F04107460C46164640F2B511384643
:10E5200003F026FA0546FF2D0BDD022E02D2002055
:10E53000BDE8F081281204F8010B04F8015B022009
:10E54000F6E705B10EB90020F2E704F8015B0120FF
:10E55000EEE770B504460025E078E8B16078012365
:10E5600004F13801626BFFF7E3FEA0B90020E07010
:10E57000A16A606B401A216A88420DD2A0780228F5
:10E580000AD1236A616BCA186078012304F138014B
:10E59000FFF7CEFE00E00125284670BD70B50446A9
:10E5A0000D460026606BA84210D02046FFF7D1FF31
:10E5B00006465EB9607801232A4604F13801FFF768
:10E5C0009CFE10B14FF0FF3501266563304670BDEB
:10E5D00070B504462046FFF7BCFF0546002D38D134
:10E5E000207803282ED1207901282BD14202002146
:10E5F00004F13800FFF735FF4AF6552104F23620C2
:10E60000FFF710FFF74904F13800FFF711FFF64953
:10E6100004F50770FFF70CFF04F508706169FFF758
:10E6200007FF04F509702169FFF702FF606A401CCB
:10E6300060636078012304F13801626BFFF778FEB4
:10E6400000202071607800221146FFF787FE00B19C
:10E650000125284670BD0246891ED069801E884269
:10E6600001D8002070475389106B03FB0100F9E7C4
:10E670002DE9F04781460C46D9F80050022C02D310
:10E68000E869A04202D84FF001085EE04FF0FF3881
:10E690002878012804D002282CD0032851D13CE04E
:10E6A000264606EB5606A86A00EB56212846FFF7D9
:10E6B00075FF00B148E03046761CC0F3080105F153
:10E6C0003800475CA86A00EB56212846FFF766FF32
:10E6D00000B139E0C6F3080105F13800405C47EAB3
:10E6E000002704F0010008B1380901E0C7F30B006E
:10E6F000804629E0A86A00EB14212846FFF74EFF68
:10E7000000B121E040F2FF1101EA440205F13801B5
:10E710005018FFF775FE804616E0A86A00EBD4118A
:10E720002846FFF73BFF00B10EE040F2FF1101EA7F
:10E73000840205F138015018FFF768FE20F0704898
:10E7400002E04FF0010800BF00BF4046BDE8F0877F
:10E750002DE9F04704460D4616464FF00209022DFA
:10E7600074D3E069A84271D92078012804D0022826
:10E7700049D003280DD15EE02F4607EB5707A06A6A
:10E7800000EB57212046FFF709FF8146B9F1000F42
:10E7900000D075E038467F1CC0F3080104F1380052
:10E7A00001EB000805F0010028B1F1B298F8000073
:10E7B00061F31F1000E0304688F800000120E0708F
:10E7C000A06A00EB57212046FFF7E8FE8146B9F129
:10E7D000000F00D054E0C7F3080104F1380001EB4A
:10E7E000000805F0010010B1C6F3071006E098F824
:10E7F000000000F0F000C6F30321084388F8000091
:10E800000120E0703CE0A06A00EB15212046FFF7F4
:10E81000C5FE8146B9F1000F00D031E0B1B240F23F
:10E82000FF1202EA450304F138029818FFF7FAFDD7
:10E830000120E07024E0A06A00EBD5112046FFF72C
:10E84000ADFE8146B9F1000F01D019E019E040F2A8
:10E85000FF1101EA850204F138015018FFF7D6FDD7
:10E8600066F31B00064640F2FF1101EA850204F13F
:10E87000380150183146FFF7DBFD0120E07000BF82
:10E8800000BF4846BDE8F0872DE9F04781460E46B7
:10E8900017464FF00008D9F80040022E02D3E06975
:10E8A000B04202D80220BDE8F08767B100BF4FF048
:10E8B000FF3239462046FFF74BFF8046B8F1000F84
:10E8C00001D04046EFE700BF31464846FFF7D0FE93
:10E8D000054605B922E0012D01D10220E3E7681CBD
:10E8E00008B90120DFE7002231462046FFF730FF5C
:10E8F0008046B8F1000F01D04046D4E7E069801EA1
:10E900006169814206D26069401C6061207940F0F3
:10E91000010020712E46E069B042D5D800BF00202A
:10E92000C1E72DE9F04782468846DAF80040B8F1A1
:10E93000000F06D1276917B1E069B84215D8012741
:10E9400013E041465046FFF793FE0546022D02D2E2
:10E950000120BDE8F087681C08B92846F9E7E0699E
:10E96000A84201D92846F4E74746606908B9002063
:10E97000EFE70026474518D17E1CE069B04200D879
:10E98000022631465046FFF773FE0546012D01D0A1
:10E99000681C08B92846DCE73DB12569022D03D380
:10E9A000E069A84200D92F46002606BB3E4600BFBC
:10E9B000761CE069B04204D80226BE4201D900208C
:10E9C000C7E731465046FFF753FE054605B90DE04F
:10E9D000012D01D0681C08B92846BAE7BE42E7D12C
:10E9E0000020B6E7525261417272416100BF4FF0A0
:10E9F000FF3231462046FFF7ABFE8146B9F1000FEA
:10EA000008D1B8F1000F05D0324641462046FFF745
:10EA10009FFE8146B9F1000F0DD12661E069801E8D
:10EA20006169814202D86069401E6061207940F0CE
:10EA30000100207107E0B9F1010F02D14FF0FF3062
:10EA400000E001200646304683E7F0B503460D4658
:10EA50001E68986A021D680A7789B0FBF7F400BF48
:10EA600002CA09B90020F0BD8C4200D202E0641A4B
:10EA7000121DF5E700BF10682044F4E72DE9F047C8
:10EA8000044689462046FFF764FD10B10120BDE829
:10EA9000F08749462046FFF7DEFD074667634FF4DF
:10EAA0000072002104F13800FFF7DBFC60894FF4AD
:10EAB0000041B1EB402F01D8084601E060894002D7
:10EAC00006464FF0000800E07608B6F5007F05D94D
:10EAD000304602F041FFB0F10008F5D0B6F5007FF6
:10EAE00017D9324600214046FFF7BBFC760A0025C5
:10EAF00000E035446089A84207D97A196078334626
:10EB00004146FFF715FC0028F3D0404602F02AFFEB
:10EB100010E004F138080126002500E03544608942
:10EB2000A84207D97A19607833464146FFF700FCBE
:10EB30000028F3D06089A84201D00120A7E7002077
:10EB4000A5E72DE9F04104460D462668B5F5001FFE
:10EB500002D205F01F0010B10220BDE8F08125614E
:10EB6000A7681FB93078032800DBF76A47B93089F6
:10EB7000B0EB551F01D80220EFE7F06AA0611CE05E
:10EB800070894FEA402811E039462046FFF770FDB2
:10EB90000746781C08B90120DFE7022F02D3F0698D
:10EBA000B84201D80220D8E7A5EB08054545EBD2CD
:10EBB00039463046FFF74FFDA0616761A06908B98B
:10EBC0000220CAE7A06900EB5520A061C5F3080147
:10EBD00006F138000844E0610020BEE72DE9F0416D
:10EBE000044688462768206900F12006B6F5001F14
:10EBF00001D30020A061A06910B90420BDE8F08114
:10EC0000C6F30800002845D1A069401CA0616069D6
:10EC100038B93889B0EB561F3CD80020A0610420D9
:10EC2000ECE77889401E00EA562098BB20466169CF
:10EC3000FFF71EFD0546012D01D80220DEE7681C06
:10EC400008B90120DAE7F869A8421DD8B8F1000F29
:10EC500003D10020A0610420D0E720466169FFF7BE
:10EC600060FE05460DB90720C8E7012D01D102203D
:10EC7000C4E7681C08B90120C0E729463846FFF7F9
:10EC8000FDFE08B10120B9E7656129463846FFF766
:10EC9000E2FCA0612661C6F3080107F138000844D0
:10ECA000E0610020AAE72DE9F04104460E46D4F8C1
:10ECB000008000212046FFF744FF0546EDB90027FC
:10ECC00000BF4046A169FFF769FC054605B113E0A6
:10ECD000E0690078E52802D0E069007820B9781C66
:10ECE0000746B04201D107E0002701212046FFF787
:10ECF00075FF0546002DE4D000BF042D00D1072587
:10ED00002846BDE8F08170B505460C4604F11A00AE
:10ED1000FFF776FB06462878032805D104F1140096
:10ED2000FFF76EFB46EA0046304670BD70B50646FA
:10ED30000C461546A9B204F11A00FFF773FB3078B0
:10ED4000032804D1290C04F11400FFF76BFB70BDFC
:10ED50002DE9F04780460C4604F11A00FFF750FBFE
:10ED600010B10020BDE8F087207800F03F00401E81
:10ED700000EB800101EBC0054FF00109002621E006
:10ED8000F849895D0819FFF73BFB0746B9F1000F09
:10ED900011D0FF2D0BD8384602F01AFE82462946C4
:10EDA0006D1C38F8110002F013FE824501D00020DE
:10EDB000D8E7B94605E04FF6FF70874201D0002042
:10EDC000D0E7761C0D2EDBD3207800F0400038B160
:10EDD000B9F1000F04D038F8150008B10020C1E7E0
:10EDE0000120BFE72DE9F04780460C4604F11A00E8
:10EDF000FFF706FB10B10020BDE8F087207820F077
:10EE00004000401E00EB800101EBC0054FF00109FE
:10EE1000002619E0D349895D0819FFF7F1FA074682
:10EE2000B9F1000F09D0FF2D01D90020E4E7B94660
:10EE300028466D1C28F8107005E04FF6FF708742D9
:10EE400001D00020D8E7761C0D2EE3D3207800F007
:10EE5000400048B1B9F1000F06D0FF2D01D90020C4
:10EE6000CAE7002028F815000120C5E72DE9F04782
:10EE700007460C461546984684F80D800F20E07230
:10EE800000202073002104F11A00FFF7CBFA681E5E
:10EE900000EB800101EBC00900200646824600BF5E
:10EEA0004FF6FF70864204D0484609F1010937F851
:10EEB0001060AC4911F80A1008193146FFF7B2FA90
:10EEC0000EB94FF6FF760AF1010082460D28E7D30E
:10EED0004FF6FF70864202D037F8190008B945F0A6
:10EEE00040052570BDE8F0872DE9FF4F83B08046CF
:10EEF00091461E460B2240460499FFF7A5FA052EBF
:10EF000018D9374611E039F802BB00250BE0584606
:10EF100067F35F0007464FEA6B0B07F4803008B1D8
:10EF2000914847406D1C102DF1D3B9F8000000281E
:10EF3000E9D13E46072500BF06F00F0000F1300A78
:10EF4000BAF1390F03DD0AF1070000F0FF0A284685
:10EF50006D1E01A901F800A03609002EECD17E201B
:10EF6000485500240AE018F80400FFF79FFA20B182
:10EF7000681EA04200D107E0641C641CAC4203D2AE
:10EF800018F804002028EED100BF00BF082D04D2DD
:10EF900028466D1C01A9085C00E020202146641C65
:10EFA00008F80100082CF1D307B0BDE8F08F30B5A8
:10EFB000014600200B2200BF431003EBC01411F8E0
:10EFC000015B6319D8B2531E1A1EF5D130BD2DE96D
:10EFD000F05F044689460426D4F800A04FF0FF08ED
:10EFE000C34653E05046A169FFF7D8FA064606B17A
:10EFF0004FE0E06905780DB904264AE0E069C07A7F
:10F0000000F03F07A771E52D0AD02E2D08D027F07C
:10F010002000082801D1012000E00020484502D04E
:10F020004FF0FF082BE00F2F1DD105F0400038B145
:10F03000E06990F80DB005F0BF05A8462069E062D0
:10F0400045450CD1E069407B584508D1E169DAF8C3
:10F050000C00FFF7C7FE10B1A8F1010000E0FF208F
:10F0600000F0FF080BE0B8F1000F04D1E069FFF7F2
:10F070009EFF584502D04FF0FF30E06209E00021CA
:10F080002046FFF7ABFD064606B102E0A069002866
:10F09000A8D100BF0EB10020A0613046BDE8F09FAE
:10F0A0002DE9F0470446D4F800A000212046FFF7E0
:10F0B00048FD064616B13046BDE8F0874FF0FF0820
:10F0C000C1464FF0FF30E06200BF5046A169FFF734
:10F0D00065FA064606B162E0E06905780DB90426D6
:10F0E0005DE0E069C07A00F03F07A771E52D04D02C
:10F0F00007F0080038B10F2F05D04FF0FF084FF090
:10F10000FF30E06244E00F2F22D12B20005D00F0A1
:10F11000400030BB05F0400038B1E06990F80D9038
:10F1200005F0BF05A8462069E06245450CD1E069BD
:10F13000407B484508D1E169DAF80C00FFF708FE8A
:10F1400010B1A8F1010000E0FF2000F0FF081FE06F
:10F15000B8F1000F0AD1E069FFF729FF484505D152
:10F160001DE015E0F0730100211001002B20005D6F
:10F1700000F0010038B90B2204F12001E069FFF72B
:10F1800079F900B90BE04FF0FF084FF0FF30E06273
:10F1900000212046FFF722FD0646002E95D000BF35
:10F1A000304689E72DE9FE4F044626682B20005D96
:10F1B00000F0A00010B10620BDE8FE8F4FF000095E
:10F1C00001E009F10109F06830F819000028F8D1D0
:10F1D0000C2204F120016846FFF736F99DF80B0078
:10F1E00000F0010028B340212B2001554FF0010809
:10F1F0000EE04346694604F12000F268FFF774FE12
:10F200002046FFF74DFF054605B104E008F101086F
:10F21000B8F1640FEDD300BFB8F1640F01D107203E
:10F22000CAE7042D01D02846C6E79DF80B102B2015
:10F2300001559DF80B0000F0020030B109F10C00FF
:10F240000D21B0FBF1F0401C00E0012007463946DB
:10F250002046FFF728FD05464DBB781E071E26D029
:10F260002069A0EB47112046FFF76BFC0546F5B976
:10F2700004F12000FFF79BFE824600BF3046A169E3
:10F28000FFF78CF9054605B110E0FAB2E169534683
:10F29000F068FFF7EBFD0120F07000212046FFF73A
:10F2A0009DFC054615B9781E071EE7D100BFC5B9FC
:10F2B0003046A169FFF772F9054695B92022002171
:10F2C000E069FFF7CEF80B2204F12001E069FFF7B7
:10F2D000BBF82B20005D00F01800E16908730120E5
:10F2E000F070284668E72DE9F04104462668276952
:10F2F000E06A401C08B9002003E02046E16AFFF7FD
:10F3000020FC0546E5B900BF3046A169FFF746F984
:10F31000054605B110E000BFE520E1690870012055
:10F32000F0702069B84200D306E000212046FFF7C4
:10F3300055FC0546002DE7D000BF042D00D1022565
:10F340002846BDE8F0812DE9F05F07460C46D7F866
:10F3500000B00020A075B86908B9BDE8F09FF86A50
:10F36000401CA8B30025A946A84622E0404608F163
:10F370000108DBF80C2032F81060B9F1000F07D15A
:10F38000B6F5584F04DBB6F5604F01DAB14610E030
:10F39000C5F1FF0204F11603591946EA0940FFF7C7
:10F3A000B7F806460EB9002509E035444FF00009CC
:10F3B00000BFDBF80C0030F818000028D6D100BFE1
:10F3C000B9F1000F00D00025002104F116004155CD
:10F3D0000020054680461BE0404608F10108FA6916
:10F3E000165C202E00D113E0052E00D1E526B8F1E1
:10F3F000090F07D10C2D05D22E2228466D1C04F1D1
:10F4000009010A5428466D1C04F109010E5400BF7D
:10F41000B8F10B0FE0D3002104F109004155A07DA4
:10F42000B0BB35B93F2228466D1C04F116010A54C1
:10F4300025E00020054680464FF0080A19E004F157
:10F44000090010F808602E2E01D14FF0100A412E4D
:10F4500009DB5A2E07DCF869007B00EA0A0010B1CC
:10F4600006F1200086B204F11600465508F10108A5
:10F470006D1C04F1090010F808000028DFD10021FC
:10F4800004F116004155F869007B08B9002060724C
:10F49000F869C07A2072F96901F11C00FEF7B6FF25
:10F4A0002060F96901F11600FEF7AAFFE080F96912
:10F4B00001F11800FEF7A4FFA08000BF4DE72DE981
:10F4C000F34F83B08146049800680090D9F800009B
:10F4D000C768002500BF6846FEF7F4FF0290029857
:10F4E000401C18B9062005B0BDE8F08F0298B0F5B1
:10F4F000803F05D30298020C28466D1C27F8102087
:10F50000029884B2202C03DB2F2C01D05C2C00D17C
:10F5100011E0802C06DA2146FEA0FEF7BDFF08B1FF
:10F520000620E0E7FF2D01D30620DCE728466D1C0E
:10F5300027F81040CFE700BF202C01DA04260CE0AA
:10F54000002602E00098401C0090009800782F28C8
:10F55000F8D0009800785C28F4D0009904980160F5
:10F56000012D04D1681E37F810002E280BD0022D73
:10F5700024D1681E37F810002E281FD1A81E37F896
:10F5800010002E281AD1002027F8150080460AE026
:10F59000A84501D22E2100E0202109F1200000F829
:10F5A000081008F10108B8F10B0FF1D346F0200163
:10F5B00009F1200000F80810002094E708E0681E18
:10F5C00037F81040202C02D02E2C00D002E06D1E07
:10F5D000002DF4D100BF002027F815000DB906203A
:10F5E00081E74FF0000A01E00AF1010A37F81A003A
:10F5F0002028F9D0BAF1000F03D137F81A002E28CD
:10F6000001D146F0030600E06D1E25B1681E37F8F3
:10F6100010002E28F8D10B22202109F12000FEF73E
:10F6200020FF4FF00008C3460820019000BF50465D
:10F630000AF1010A37F8104004B968E0202C03D021
:10F640002E2C04D1AA4502D046F00306EFE701981C
:10F65000804501D2AA4516D101980B2802D146F067
:10F66000030654E0AA4501D046F00306AA4500D996
:10F670004DE0AA464FF008080B2001904FEA8B603E
:10F680004FEA106BD3E7802C0EDB46F0020640F207
:10F69000B511204602F06CF9044604F0800018B160
:10F6A00004F07F009E490C5CFF2C10DD0198401E89
:10F6B000404504D846F00306DDF80480B7E722127F
:10F6C000404608F1010809F120010A5418E024B16C
:10F6D000214694A0FEF7E0FE18B15F2446F0030631
:10F6E0000EE0412C03DB5A2C01DC4BF0020B612CA9
:10F6F00006DB7A2C04DC4BF0010BA4F1200084B271
:10F70000404608F1010809F120010C548FE700BFC1
:10F7100099F82000E52802D1052089F820000198F9
:10F72000082803D14FEA8B604FEA106B0BF00C00F6
:10F730000C2803D00BF00300032801D146F0020689
:10F7400006F0020048B90BF0010008B146F01006BF
:10F750000BF0040008B146F008062B2000F8096001
:10F760000020C0E62DE9F34104462768019800789F
:10F770002F2806D0019800785C2802D0B869A060D4
:10F780000DE002E00198401C0190019800782F28BC
:10F79000F8D0019800785C28F4D00020A06001988F
:10F7A0000078202808D280212B20015500212046F6
:10F7B000FFF7C7F9054637E000BF01A92046FFF76C
:10F7C0007EFE054605B12EE02046FFF769FC0546A2
:10F7D0002B20065D95B1042D0FD106F0200040B11D
:10F7E00006F0040000B9E8E780212B200155002530
:10F7F00003E006F0040000B9052514E006F004005B
:10F8000000B110E0A07900F0100008B905250AE069
:10F81000208AC0F3080207F1380011183846FFF7B4
:10F8200072FAA060C9E700BF2846BDE8FC8170B548
:10F8300004464FF0FF3026683146324601B970BDAC
:10F8400000BF12F8013B202B01D33A2BF9D13A2B00
:10F8500011D101250E78302E08DB0E78392E05DC0B
:10F860008E1C964202D10E78A6F13005012D01DAE8
:10F8700028462260E3E72D4E307800BFDFE72DE910
:10F88000F041044688460020E070401E6063414617
:10F890002046FEF783FE10B10420BDE8F08104F29B
:10F8A0003620FEF7ADFD074694F83850EB2D03D017
:10F8B000E92D01D0E82D4AD14AF65520874208D1DA
:10F8C00008221BA104F18A00FEF7D4FD08B900202C
:10F8D000E3E704F14300FEF793FD0646701E304057
:10F8E00060BBB6F5007F32DBB6F5007F2FDC45202C
:10F8F000055D1DB3681E284000BB4820005D01283F
:10F9000003D04820005D022821D104F14900FEF710
:10F9100077FD14E0222A3A3C3E3F7C7F0000000045
:10F92000FD7301002B2C3B3D5B5D0000920100202C
:10F9300046415433322020200000000007E030B15F
:10F9400004F14E00FEF75CFD08B10020A5E74AF681
:10F950005520874201D102209FE703209DE72DE932
:10F96000FF4107460D4600213846FFF788FF06464F
:10F97000022E06D0032E00D21DB9304604B0BDE8D9
:10F98000F08100BF00240AE007F5FB7101EB0411D0
:10F9900001F10800FEF73AFD4DF82400641C042C28
:10F9A000F2D30DB1681E00E00020044600BF5DF8F0
:10F9B000240028B15DF824103846FFF760FF00E00E
:10F9C000032006462DB9022E03D3601C04460428EA
:10F9D000EDD33046D2E72DE9F74F84B000210598EA
:10F9E00001600498FFF723FF03900398002803DACF
:10F9F0000B2007B0BDE8F08FFE49039851F8204076
:10FA00000CB90C20F5E705980460069800F0FE009C
:10FA10000690207878B16078FEF756FC074607F02C
:10FA2000010040B9069820B107F0040008B10A208F
:10FA3000DFE70020DDE70020207003986070607829
:10FA4000FEF748FC074607F0010008B10320D0E7A5
:10FA5000069820B107F0040008B10A20C9E7002188
:10FA60002046FFF77CFF0546042D01D10120C0E7A9
:10FA7000022D01D30D20BCE7D4F8349004F14300EB
:10FA8000FEF7BEFCB0F5007F01D00D20B1E704F118
:10FA90004E00FEF7B5FC064626B904F15C00FEF701
:10FAA000B5FC064626624820005DA070A0780128BB
:10FAB00004D0A078022801D00D209AE7A078464310
:10FAC0004520005D6081608918B16089411E084051
:10FAD00008B10D208DE704F14900FEF791FC20816B
:10FAE000207A00F00F0008B10D2082E704F14B00EE
:10FAF000FEF786FC8246BAF1000F04D104F15800EB
:10FB0000FEF784FC824604F14600FEF779FC83464A
:10FB1000BBF1000F01D10D206BE70BEB0600218933
:10FB200000EB111002900298824501D20D2060E78F
:10FB30000298AAEB00006189B0FBF1F8B8F1000F60
:10FB400001D10D2055E70025AB48804500D803259D
:10FB50004FF6F570804500D8022540F6F5708045D7
:10FB600000D801250DB90D2043E708F10200E0613E
:10FB7000C4F8249009EB0B00A0620298484420636B
:10FB8000032D13D104F16200FEF73AFC08B10D20F9
:10FB90002FE7208908B10D202BE704F16400FEF760
:10FBA00035FCE062E0698000019014E0208908B92A
:10FBB0000D201EE7A06A3044E062022D02D1E06908
:10FBC000400007E0207F00F00100E16901EB410106
:10FBD00000EB51000190216A019800F2FF10B1EB97
:10FBE000502F01D20D2004E74FF0FF3060612061FB
:10FBF00080202071032D2DD104F16800FEF700FC58
:10FC0000012827D109F101012046FEF7C7FC08BBF6
:10FC10000020207104F23620FEF7F2FB4AF655214F
:10FC2000884217D104F13800FEF7F0FB734988428F
:10FC300010D104F50770FEF7E9FB7149884209D13C
:10FC400004F50870FEF7E2FB606104F50970FEF749
:10FC5000DDFB206125706B480088401C80B269493B
:10FC60000880E0800020A06100BFC2E670B50446B5
:10FC70000D4609268CB1206878B12068007860B103
:10FC8000A0882168C988884207D121684878FEF792
:10FC90001BFB00F0010000B900260EB9206800E04F
:10FCA00000202860304670BDF7B582B01646039834
:10FCB000019001A8FFF7BBFD0546002D02DA0B20DD
:10FCC00005B0F0BD4B4850F825400CB10020207025
:10FCD000029810B10020029908704649029841F834
:10FCE00025000EB90020EBE7002202A903A8FFF7C8
:10FCF00072FE07463846E3E72DE9F74F90B0044619
:10FD000016461CB9092013B0BDE8F08F06F03F0677
:10FD1000324603A911A8FFF75EFE0546002D68D103
:10FD2000039804904FF4007001F016FE8346BBF177
:10FD3000000F01D11120E6E70398C0F80CB004A829
:10FD40001199FFF70FFD05462DB99DF83B0000F016
:10FD5000800000B1062506F01C00002862D045B1E5
:10FD6000042D03D104A8FFF71DFA054646F0080646
:10FD70000AE09DF8160000F0110008B1072503E025
:10FD800006F0040000B10825002D5CD106F0080043
:10FD9000002858D0FEF712FB01900B9901F10E00DC
:10FDA0000199FEF745FB0B9901F116000199FEF749
:10FDB0003FFB0B990398FEF7A6FF814620200B9985
:10FDC000C87200220B990398FEF7B0FF0B9901F15E
:10FDD0001C000021FEF72CFB01200399C870B9F12B
:10FDE000000F30D00398D0F834A00022494604A870
:10FDF0000AE093E08C010020F5FFFF0F52526141B1
:10FE00007272416190010020FEF73EFD054645B942
:10FE100051460398FEF7C2FB0546A9F1010003997C
:10FE2000086110E07DB99DF8160000F0100008B1DF
:10FE3000042508E006F0020028B19DF8160000F045
:10FE4000010000B107254DB906F0080008B146F0E1
:10FE500040060398406B20620B986062002D5AD1D7
:10FE60000B990398FEF74FFFA0600B9901F11C005E
:10FE7000FEF7CCFAE0600020A062039820600398AF
:10FE8000C088A080267400206074E06160614FF437
:10FE90000072002104F12C00FEF7E3FA06F02000C6
:10FEA00058B3E06848B3E068606103984089400255
:10FEB0000290A768D4F80C800DE039462046FEF782
:10FEC000D7FB0746012F00D80225781C00B9012571
:10FED0000298A8EB000815B902988045EDD8A761F3
:10FEE0005DB9C8F3080040B139460398FEF7B3FB8B
:10FEF0008246BAF1000F01D102250CE00AEB58202E
:10FF0000E061E26903994878012304F12C01FEF7CE
:10FF1000F4F900B10125584601F024FD0DB100208F
:10FF200020602846EFE62DE9FF4F85B004461546D0
:10FF30009A46DDF818B00020CAF8000003A9204650
:10FF4000FFF794FE0490049810B9607C049018B1F7
:10FF5000049809B0BDE8F08F207C00F0010008B9DA
:10FF60000720F6E76169E068401A01900198854230
:10FF700000D9019DA8E0A08AC0F30800002874D130
:10FF800003984089401E616900EA5129B9F1000FC8
:10FF90001FD1606910B9A06802900CE0A06A28B176
:10FFA00020466169FEF751FD029004E02046A169F8
:10FFB000FEF75EFB02900298022802D202206074D3
:10FFC000C7E70298401C10B901206074C1E702988D
:10FFD000A061A1690398FEF73EFB064616B9022010
:10FFE0006074B6E74E444FEA5528B8F1000F29D0A7
:10FFF00009EB080003994989884203D9039840898D
:020000040001F9
:10000000A0EB090803994878434632465946FEF763
:1000100074F910B1012060749BE7207C00F080002F
:1000200068B1E069801B404509D2E169891B0BEB8F
:1000300041204FF4007204F12C01FEF705FA4FEA5B
:10004000482737E0E069B04220D0207C00F08000F3
:1000500080B1E26903994878012304F12C01FEF78D
:1000600067F918B10120607473E710E0207C00F09C
:100070007F002074039948780123324604F12C0153
:10008000FEF73BF910B10120607462E7E661A08AD7
:10009000C0F30800C0F50077AF4200D92F46A08A10
:1000A000C0F3080204F12C0011183A465846FEF736
:1000B000CBF900BFED1BDAF800003844CAF80000A5
:1000C000BB44606938446061002D7FF454AF002068
:1000D0003FE72DE9FF4F83B0044615469B46049841
:1000E00000900020CBF8000001A92046FFF7BEFDDC
:1000F0000290029810B9607C029018B1029807B083
:10010000BDE8F08F207C00F0020008B90720F6E778
:1001100000BF606928446169884202D26069C0F109
:10012000FF35C3E0A08AC0F3080000287DD1019804
:100130004089401E616900EA512ABAF1000F26D1B8
:10014000606938B9A76897B900212046FEF7E9FB36
:1001500007460CE0A06A28B120466169FEF775FCED
:10016000074604E02046A169FEF7DBFB074607B916
:100170009FE0012F02D102206074C0E7781C10B903
:1001800001206074BBE7A761A06800B9A760207C6C
:1001900000F0800078B1E26901994878012304F108
:1001A0002C01FEF7C5F810B101206074A7E7207C90
:1001B00000F07F002074A1690198FEF74CFA064612
:1001C00016B9022060749AE756444FEA5529B9F1EE
:1001D000000F2BD00AEB090001994989884203D905
:1001E00001984089A0EB0A09019948784B463246AC
:1001F0000099FEF79DF810B1012060747FE7E06977
:10020000801B48450ED2E069801B009A02EB40211A
:100210004FF4007204F12C00FEF716F9207C00F078
:100220007F0020744FEA49282BE013E0E069B042D8
:100230000FD0E168606988420BD2019948780123A8
:10024000324604F12C01FEF758F810B10120607419
:1002500055E7E661A08AC0F30800C0F50078A8451C
:1002600000D9A846A18AC1F3080204F12C01501854
:1002700042460099FEF7E8F8207C40F080002074A8
:1002800000BFA5EB0805DBF800004044CBF80000F8
:10029000009840440090606940446061E168606992
:1002A000884201D9606900E0E068E060002D7FF4D9
:1002B00039AF00BF207C40F04000207400201EE7D2
:1002C000F8B5044669462046FFF7D0FC0646002EE6
:1002D00044D1207C00F0400000283FD0207C00F07A
:1002E000800070B1E26900994878012304F12C0183
:1002F000FEF71EF808B10120F8BD207C00F07F0059
:100300002074FEF75BF80746216A0098FEF746F96D
:1003100006461EBB656AE87A40F02000E87229466E
:10032000A2682068FEF702FD05F11C00E168FEF7F7
:100330007FF8394605F11600FEF77AF8002105F13D
:100340001200FEF76FF801200099C8700098FEF7C0
:100350003FF90646207C00F0BF0020743046CBE712
:1003600038B505462846FFF7ABFF04463CB9694659
:100370002846FFF77BFC04460CB900202860204685
:1003800038BD31B56846FFF752FA0446002C01DA51
:100390000B2038BDFB490C700020FAE731B58EB058
:1003A000002201A90EA8FFF716FB044674BB0198B2
:1003B00002904FF4007001F0CFFA054615B91120F4
:1003C0000FB030BD0198C56002A80E99FFF7CAF9B9
:1003D0000446ACB99DF8330000F0800018B10199D3
:1003E000049888610CE09DF80E0000F0100030B118
:1003F00009990198FEF787FC0199886100E00524BE
:10040000284601F0AFFA042C00D105242046D7E796
:100410002DE9F04F89B004460D4607A92046FFF7A5
:1004200025FC0890089808B9607C0890089818B1D5
:10043000089809B0BDE8F08FA06A00287CD0681C3D
:10044000002843D1D4F8289059F8040B02900220D8
:100450000190A76867B300BF03970020049001983C
:10046000801C019000BF05970498401C04903946F9
:100470002046FEF7FDF80746012F02D802206074DF
:10048000D7E7781C10B901206074D2E70598401CAA
:100490008742E8D0DDE90101884205D8049849F88F
:1004A000040B039849F8040B0798C069B842D3D8E5
:1004B0000198A16A0860DDE90101884203D80020A3
:1004C000C9F80000FAE011200890F7E0E068A842BF
:1004D00000D2E5686561002DF4D0691E2046FEF764
:1004E000B4FAA061A1690798FEF7B5F88246BAF19F
:1004F000000F02D1022060749BE707984089401EDC
:10050000691E00EA51208244A08AC0F30800002836
:10051000D8D0E0695045D5D0207C00F0800080B173
:10052000E26907994878012304F12C01FDF700FFE7
:1005300018B1012060747CE712E0207C00F07F009D
:100540002074079948780123524604F12C01FDF7E5
:10055000D4FE10B1012060746BE7C4F81CA0ADE0BC
:10056000E068A84204D2207C00F0020000B9E568EF
:10057000606906904FF0000BC4F814B0002D6AD0EB
:10058000079840894FEA4028069890B1681EB0FB52
:10059000F8F10698401EB0FBF8F0814209D30698A6
:1005A000401EA8F101018843606160692D1AA669A7
:1005B00012E0A6687EB900212046FEF7B2F9064691
:1005C000012E02D10220607433E7701C10B90120A3
:1005D00060742EE7A660A661D6B325E0A5EB0805FA
:1005E000606940446061207C00F0020040B100BFBF
:1005F00031462046FEF795F9064636B9002515E046
:1006000031462046FEF734F80646701C10B901202A
:1006100060740EE7012E03D90798C069B04202D872
:100620000220607405E7A6614545D7D800BF606920
:1006300028446061C5F3080050B131460798FEF7C1
:100640000AF88346BBF1000F03D102206074F0E684
:1006500001E00BEB552BE1686069884205D96069C0
:10066000E060207C40F040002074A08AC0F30800C5
:1006700020B3E069584521D0207C00F0800078B19B
:10068000E26907994878012304F12C01FDF750FE37
:1006900010B101206074CCE6207C00F07F00207453
:1006A0000799487801235A4604F12C01FDF725FEED
:1006B00010B101206074BCE6C4F81CB00898B8E61C
:1006C00073B582B0044614B9092004B070BD00228D
:1006D00001A903A8FFF77FF90546002D30D1019845
:1006E00020604FF4007001F037F906460EB9112072
:1006F000EBE70198C66020460399FFF733F80546FB
:10070000C5B92B20005D00F0800050B9A07900F041
:10071000100028B1E1690198FEF7F5FAA06000E049
:1007200005253DB90198C088A08000212046FEF72C
:1007300008FA0546304601F015F9042D00D10525CB
:100740000DB1002020602846BFE738B50446694651
:100750002046FFF78BFA05460DB900202060284699
:1007600038BDF8B507460E4669463846FFF77EFAAB
:1007700004465CBB46B900213846FEF7E2F9044660
:1007800024E00000920100204FF4007001F0E4F832
:1007900005460DB91120F8BD0098C5600021384606
:1007A000FEF715FC0446042C00D100245CB9314648
:1007B0003846FEF7C8FD00213846FEF70FFA04461A
:1007C000042C00D10024284601F0CCF82046E2E7B2
:1007D00073B58CB00E46002269460CA8FFF7FBF8F3
:1007E0000546FDB94FF4007001F0B6F8044614B99F
:1007F00011200EB070BD0098C46068460C99FEF7D9
:10080000B1FF05465DB99DF82B0000F0800008B1EE
:10081000062504E01EB131466846FEF794FD2046E9
:1008200001F0A0F82846E4E72DE9F74F86B08846A6
:100830009246002205A906A8FFF7CDF88146B9F136
:10084000000F68D10598CAF8000005984169C06991
:10085000801E814204D805984069C8F800005AE01B
:1008600000250598007801281BD1022605980190E3
:1008700000BF314601A8FDF7FBFE0746781C10B902
:100880004FF001090CE0012F02D14FF0020907E0FF
:1008900007B96D1C701C06460599C9698842E8D3E2
:1008A0002FE00598C6690598D0F828B0002400BF4D
:1008B00054B959460BF1010B0598FDF76FFE8146BF
:1008C000B9F1000F00D01BE005980078022808D18C
:1008D000059938310819FDF793FD00B96D1CA41C6A
:1008E00009E0059938310819FDF790FD20F07040B6
:1008F00000B96D1C241DC4F30804701E061ED7D158
:1009000000BFC8F80050059845610598007940F08F
:10091000010005990871484609B0BDE8F08FF8B5A7
:10092000044669462046FFF7A1F9054615B9607CE3
:10093000051E01D02846F8BD207C00F0020008B951
:100940000720F8E7E168606988423FD2606940B9F2
:1009500000222046A168FDF797FF05460020A06011
:1009600016E02046A169FDF783FE06460025701CAF
:1009700000B90125012E00D102254DB90098C069AA
:10098000B04205D931462046A269FDF77DFF0546F4
:100990006069E060207C40F04000207495B9207CC4
:1009A00000F0800070B1E26900994878012304F1F9
:1009B0002C01FDF7BDFC08B1012503E0207C00F00F
:1009C0007F00207415B165742846B4E72846B2E765
:1009D00071B599B000250222694619A8FEF7FBFF00
:1009E0000446002C60D100980D904FF4007000F088
:1009F000B3FF064616B911201AB070BD0098C66044
:100A00000DA81999FEF7AEFE04462CB99DF85F00BB
:100A100000F0200000B10624002C42D19DF85F00B8
:100A200000F0800008B1062405E09DF83A0000F0CF
:100A3000010000B1072414BB14990098FEF763F974
:100A400005469DF83A0000F01000C0B1009880699A
:100A5000A84201D1072412E00098019003950021DB
:100A600001A8FEF76EF804464CB9002101A8FEF774
:100A7000AEFA044604B90724042C00D1002484B93A
:100A80000DA8FEF730FC044634B92DB100222946EA
:100A90000DA8FDF7F9FE04461CB90098FDF798FD76
:100AA0000446304600F05EFF2046A5E72DE9F141FF
:100AB00091B00222694611A8FEF78DFF0446002C72
:100AC0007ED1009805904FF4007000F045FF064677
:100AD0001EB9112012B0BDE8F0810098C66005A8CB
:100AE0001199FEF73FFE044604B90824042C05D1F1
:100AF0009DF83F0000F0200000B10624042C6AD1CC
:100B000000980190002101A8FDF70BFF0546002485
:100B100005B90724012D00D10224681C00B9012465
:100B2000FDF74CFC8046BCBB29460098FDF7A6FFAC
:100B300004468CBB0B22202100983830FDF791FC35
:100B40002E20009981F838001021009880F8431079
:100B5000414600984E30FDF76BFC2A46009938312B
:100B60000098FEF7E3F820220099383100985830B9
:100B7000FDF76AFC2E21009880F85910079F3A462D
:100B8000009958310098FEF7D1F801200099C870FB
:100B900005A8FEF707FB0446C4B90C9901F116003D
:100BA0004146FDF745FC2A460C990098FEF7BEF831
:100BB00010200C99C87201200099C8702CB900E06F
:100BC0000CE00098FDF704FD044604E000222946ED
:100BD00001A8FDF759FE304600F0C4FE204679E733
:100BE0002DE9F341A2B023A8FEF721FE022209A9B4
:100BF00022A8FEF7F0FE0446002C7DD1099816903D
:100C00004FF4007000F0A8FE07461FB9112024B071
:100C1000BDE8F0810998C76016A82299FEF7A2FDE9
:100C200004462CB99DF8830000F0A00000B1062412
:100C3000002C6ED1202201A81D99FDF705FC302261
:100C400016A90AA8FDF700FC0AA82399FEF78AFD59
:100C500004465CB918990C98884205D11A990E98E7
:100C6000884201D1042000E008200446042C46D12B
:100C70000AA8FEF797FA0446002C40D1119D1322D2
:100C80000DF1110105F10D00FDF7DEFB9DF80F00E0
:100C9000E872E87A00F0100018B9E87A40F0200015
:100CA000E87201200999C870E87A00F0100030B3AA
:100CB0000C991898884222D029460998FEF723F803
:100CC000804641460998FDF7C6FC06460EB9022447
:100CD00015E031460998FDF761FC0446099800F1DA
:100CE000580564B968782E2809D129460C9A0998C4
:100CF000FEF71CF8012000E00EE00999C87044B925
:100D000016A8FEF7F0FA04461CB90998FDF760FC36
:100D10000446384600F026FE204678E72DE9FF4FCE
:100D200085B09A4603AA01210598FDF717FB18B173
:100D3000012009B0BDE8F08FDDF80C904FF03F08BE
:100D4000082701E07806070E37B1B9FBF7F0B0FBD2
:100D5000F8F0B0F5806FF5D807B9FF274FF40072AF
:100D600000215046FDF77DFB0AF5DF764FF0000BC2
:100D7000444669E0069850F82B50642D07D801D1FD
:100D8000484603E06420B9FBF0F06843054660196B
:100D9000484501D8601901D3A9EB040505B959E00C
:100DA000214606F10800FDF743FB294606F10C0039
:100DB000FDF73EFB07983071B4FBF8F0B0FBF7F09D
:100DC0000490B4FBF8F0B0FBF7F107FB1100C0B2E0
:100DD0000290B4FBF8F008FB1040401CC0B2019038
:100DE00002987070C021049801EA900001990843AC
:100DF000B0700498F0706019401EB0FBF8F0B0FBC2
:100E0000F7F004906019401EB0FBF8F0B0FBF7F16A
:100E100007FB1100C0B202906019401EB0FBF8F150
:100E200008FB1100401CC0B2019002987071C021F3
:100E3000049801EA900001990843B0710498F07198
:100E400010360BF1010B2C44BBF1040F02D20CB194
:100E50004C458FD300BF4AF655210AF5FF70FDF7C8
:100E6000E1FA0123002251460598FDF761FA08B125
:100E700001205EE700205CE72DE9FF4F99B00F46A7
:100E8000154619A8FEF7D3FC03900398002803DA4F
:100E90000B201DB0BDE8F08FFC49039851F82000ED
:100EA00028B10021F94A039852F8200001700398F4
:100EB000C0B216900020159007B9F54F1698FDF7AF
:100EC00009FA0290029800F0010008B10320E0E75F
:100ED000029800F0040008B10A20DAE7786813905D
:100EE000139838B913AA03211698FDF737FA08B1F9
:100EF00001201390139840B11398B0F5004F04D817
:100F00001398401E1399084008B1012013904FF424
:100F10000079387800F00F0018907878012804DB09
:100F20007878022801DC787800E001200690B96822
:100F300089B1B968B1F5004F0DD848464FEAE9715B
:100F400009EBD1614911BA68B2FBF1F301FB13213E
:100F500009B9B96801E04FF400710591F868B0F182
:100F6000807F05D8F868411E084008B9F86800E09D
:100F7000002007900798B0FBF9F007901C98B0FB91
:100F8000F9F01490149808B9112082E72C462CB976
:100F9000149901FB09F000F0DFFC04460CB91120A4
:100FA00077E700201190109000BF11AA0121169838
:100FB000FDF7D4F928B115B9204600F0D3FC012083
:100FC00067E7189800F0080040B911983F2805D944
:100FD0003F201090DDE91001081A11901198802827
:100FE00005D215B9204600F0BDFC0E2051E700BF28
:100FF00000BF0798802801D980200790189800F03A
:10100000020030B1189800F0010010B94FF0030849
:101010000CE0189800F0010028B915B9204600F03E
:10102000A1FC132035E74FF0020800BF00BF00BF4E
:10103000079EB8F1030F31D1A6B911984FEA504B72
:1010400000200490012603E00498401C04907600E0
:101050009049049831F8100020B1049831F810003C
:101060005845F1D91198B0FBF6FA082000EB8A0038
:101070004844401EB0FBF9F0099020200A9000205F
:1010800008904FF6F570824502D9834882453BD9D6
:1010900015B9204600F066FC0E20FAE6A6B91198B4
:1010A0004FEA103B00200490012603E00498401C06
:1010B000049076007949049831F8100020B1049822
:1010C00031F810005845F1D91198B0FBF6FA40F606
:1010D000F570824503D9042000EB4A0B07E04FF07E
:1010E00001080AEB4A00401C032101EB500B0BEBFB
:1010F0000900401EB0FBF9F0099001200A90059804
:101100004001B0FBF9F008900A99109808440F903C
:10111000069A09990F9801FB0201089808440E905D
:1011200013990E980844401E491E20EA01010E98AA
:10113000A1EB000BB8F1030F06D10A9858440A90AE
:101140000F9858440F9013E00698BBFBF0F100FB9A
:1011500011B038B1ABF1010B0A98401C0A900F98FE
:10116000401C0F900698BBFBF0F1099808440990C9
:101170000E9800EB06111098081A1199884205D9AB
:1011800015B9204600F0EEFB0E2082E611990A9870
:101190000A1A0699099800FB11210898081AB0FB51
:1011A000F6FAB8F1030F0FD14FF6F57082450BD860
:1011B000079818B97008079000B148E015B92046A3
:1011C00000F0D0FB0E2064E6B8F1020F31D14FF6EB
:1011D000F57082451CD9079830B94020B0EB460F16
:1011E00002D37000079032E0189800F0020010B1AE
:1011F0004FF003082BE0079820B970000790802873
:1012000000D824E015B9204600F0ACFB0E2040E6E3
:1012100040F6F57082450CD8079820B97000079009
:10122000802800D813E015B9204600F09BFB0E2063
:101230002FE6B8F1010F09D140F6F570824505D9C6
:1012400015B9204600F08EFB0E2022E600E0EFE606
:1012500000BF4A4600212046FDF703F90B2210A1EA
:101260002046FDF7F1F8494604F10B00FDF7DAF8E6
:1012700066730A9881B204F10E00FDF7D3F8069860
:101280002074B8F1030F11D1002010E08C01002070
:101290009C7401008C740100F5FFFF0F7E74010047
:1012A000EBFE904D53444F53352E3000059881B2DC
:1012B00004F11100FDF7B6F81198B0F5803F06D2A1
:1012C000119881B204F11300FDF7ACF804E004F1C9
:1012D00020001199FDF7ACF8F82060753F2104F16A
:1012E0001800FDF79FF8FF2104F11A00FDF79AF8A6
:1012F00004F11C001099FDF79BF8B8F1030F28D1F9
:10130000FDF75CF80146009004F14300FDF790F80A
:1013100004F124000999FDF78BF8022104F12C0057
:10132000FDF786F8012104F13000FDF77BF8062176
:1013300004F13200FDF776F8802084F8400029207F
:1013400084F842001322F9A104F14700FDF77CF86C
:1013500019E0FDF733F80146009004F12700FDF78E
:1013600067F8099881B204F11600FDF75BF8802058
:1013700084F82400292084F826001322F0A104F127
:101380002B00FDF761F84AF6552104F5FF70FDF7D3
:1013900049F801232146109A1698FCF7C9FF28B195
:1013A00015B9204600F0DEFA012072E5B8F1030F0E
:1013B00033D10123109A921D21461698FCF7B8FFED
:1013C0004A4600212046FDF74CF8E2492046FDF749
:1013D0002FF8E14904F5F270FDF72AF8AAF10101AE
:1013E00004F5F470FDF724F8022104F5F670FDF71A
:1013F0001FF84AF6552104F5FF70FDF713F8012395
:10140000109AD21D21461698FCF792FF0123109ADC
:10141000521C21461698FCF78BFF149800FB09F22A
:1014200000212046FDF71DF80F980D900020049034
:1014300048E0B8F1030F10D16FF007012046FCF728
:10144000F7FF4FF0FF31201DFCF7F2FF6FF0704106
:1014500004F10800FCF7ECFF0AE0B8F1010F01D13C
:10146000BE4801E06FF0070001462046FCF7E0FFB0
:101470000998129000BF14991298884201D91498C3
:1014800000E0129883465B4621460D9A1698FCF7B9
:101490004FFF28B115B9204600F064FA0120F8E4A6
:1014A0004A4600212046FCF7DCFF0D9858440D9079
:1014B0001298A0EB0B00129012980028DBD1049830
:1014C000401C0490069904988842B2D3B8F1030FE7
:1014D00001D1304600E00898129000BF149912988C
:1014E000884201D9149800E0129883465B46214651
:1014F0000D9A1698FCF71CFF28B115B9204600F08C
:1015000031FA0120C5E40D9858440D901298A0EBD3
:101510000B00129012980028E0D100BFB8F1030F21
:1015200002D10C2017900DE01198B0F5803F02D346
:101530000620179006E0B8F1020F01D1042000E068
:101540000120179000BF189800F0080090B911987A
:101550000B9000200C9023460BA9DDE91602FFF743
:10156000DDFB0190019828B115B9204600F0FAF989
:1015700001988EE4002211461698FCF7EFFE28B180
:1015800015B9204600F0EEF9012082E415B9204695
:1015900000F0E8F900207CE42DE9FC4780460C4689
:1015A000914600254646641E13E06B46012201A9C0
:1015B0004846FEF7B8FC0098012800D00BE09DF8E3
:1015C000047000BF06F8017B6D1C0A2F00D102E0F9
:1015D00000BFA542E9DB00BF0020307015B14046D6
:1015E000BDE8FC870020FBE7F8B504460E4600BFC7
:1015F0006568002D00DAF8BDA76828466D1C04F167
:101600000C010E543C2D0CDB6B462A462068FEF77D
:1016100060FD0098A84201D1002001E04FF0FF30AA
:1016200005466560781CA06000BFE4E738B5044655
:10163000606800280DDB6B4604F10C01D4E9000260
:10164000FEF747FD28B960680099884201D1A0687B
:1016500038BD4FF0FF30FBE770B504460D464C2215
:1016600000212046FCF7FDFE256070BD30B593B02B
:1016700004460D4629466846FFF7EEFF21466846B8
:10168000FFF7B2FF6846FFF7D1FF13B030BD30B5AA
:1016900093B004460D4629466846FFF7DDFF04E097
:1016A00014F8011B6846FFF79FFF20780028F7D148
:1016B0006846FFF7BBFF13B030BD0FB42DE9F04F04
:1016C0009DB009A82699FFF7C7FF28A81C9000BF66
:1016D000279810F8014B279004B932E1252C04D04B
:1016E000214609A8FFF780FFF2E700200646814661
:1016F000279810F8014B2790302C05D10126279808
:1017000010F8014B279006E02D2C04D102262798D3
:1017100010F8014B27902A2C22D11C9850F8049BDA
:101720001C90279810F8014B279028E04E4F204E30
:10173000414D4520202020464154333220202000B6
:101740004E4F204E414D4520202020464154202020
:10175000202020005252614172724161F8FFFF0067
:1017600009E009EB890004EB4000A0F1300927985B
:1017700010F8014B2790302C01DB392CF1DD6C2C5B
:1017800001D04C2C05D146F00406279810F8014BE7
:10179000279004B9D5E02546612D04DB7A2D02DCC3
:1017A000A5F12000C5B24F2D49D006DC422D43D013
:1017B000432D38D0442D4CD144E0532D04D0552D29
:1017C00041D0582D45D141E01C9850F804BB1C90E5
:1017D0004FF0000801E008F101081BF8080000289C
:1017E000F9D106F0020048B903E0202109A8FFF76B
:1017F000FBFE404608F101084845F6D304E01BF81B
:10180000011B09A8FFF7F0FE9BF800000028F6D1A5
:1018100003E0202109A8FFF7E7FE404608F1010890
:101820004845F6D354E71C9810F8042BD1B21C900D
:1018300009A8FFF7D9FE4BE7022008900EE0082028
:1018400008900BE000BF0A20089007E010200890E5
:1018500004E0214609A8FFF7C7FE39E700BF06F0FC
:10186000040028B11C9800681C99091D1C910CE00B
:10187000442D05D11C9800681C99091D1C9104E099
:101880001C9800681C99091D1C918246442D06D1A4
:101890000AF0004018B1CAF1000A46F00806002715
:1018A00000BF0898BAFBF0F100FB11A0C5B2089880
:1018B000BAFBF0FA092D06DD782C01D1272000E0D3
:1018C00007202844C5B205F13000C2B238467F1C5B
:1018D0000DF80020BAF1000F01D0202FE1D306F05F
:1018E000080020B12D2238467F1C0DF80020B84694
:1018F00006F0010008B1302000E02020054606F087
:10190000020048B903E0294609A8FFF76DFE4046EA
:1019100008F101084845F6D300BF781E07461DF8B8
:10192000001009A8FFF760FE002FF6D103E029465A
:1019300009A8FFF759FE404608F101084845F6D3CB
:10194000C6E600BF00201C9009A8FFF76FFE1DB07F
:10195000BDE8F00F5DF814FB10B50446204604F016
:10196000CFF910BD10B50446204604F0F8F910BDBB
:1019700010B502460020404B802A01D290B213E0FD
:10198000B2F5803F10D240F2B514A1420CD1002034
:1019900001E0441CA0B2802803DA33F810409442DE
:1019A000F7D100F18004E0B210BD10B5024600206E
:1019B000314B802A01DA104609E040F2B514A14209
:1019C00005D1FF2A03DCA2F1800433F8140010BD16
:1019D00070B5B0F5803F4DD281B2B1F5805F01DACC
:1019E000264E00E0264E324600BF32F8023B0BB1D5
:1019F000994200DA3CE032F8024B2512E4B21E199B
:101A00008E4230DD092D2CD2DFE805F005090F13D9
:101A1000171B1F232700CE1A32F8161021E0CE1A0A
:101A200006F001068E1BB1B21BE0A1F11006B1B2A7
:101A300017E0A1F12006B1B213E0A1F13006B1B276
:101A40000FE0A1F11A06B1B20BE001F10806B1B244
:101A500007E0A1F15006B1B203E0A1F5E356B1B23F
:101A600000BF00BF04E0002DBFD102EB4402BCE781
:101A700000BF084670BD0000AC740100AC750100E9
:101A80009E7701002DE9FF4FADF50F7D8946164683
:101A9000DDF8708200250027002001904FF480714E
:101AA000F74804F05AFC8F9860B18F9804F074FBEB
:101AB00040B1B9F1000F05D0B8F1000F02D00EB15E
:101AC000929828B94FF0FF300DF5137DBDE8F08FE7
:101AD00000240FE056F8240040B156F8240004F02A
:101AE0005BFB18B1929850F8240010B94FF0FF300A
:101AF000EAE7641C9D988442ECDB012203A88F99DD
:101B0000FEF7FAF88E908E9810B16FF00100DBE7C7
:101B10000024FDE0ECE003AA4FF48071D848FFF701
:101B20003BFD0290029888B906990898884201D135
:101B3000012000E0002018B1002048F82400E1E076
:101B400003A8FEF70DFC6FF00200BDE7002700259B
:101B50000EE004F0CDF80068C949495D405C00F032
:101B6000010020B9C648405DC549C8557F1C6D1CA1
:101B7000C34804F011FBA842EBD80020C049C85567
:101B800008460078232800D1B2E059F82410BC4858
:101B900004F0F0FAB0B1BA4800785B2812D1B84826
:101BA00004F0FAFA401EB649085C5D280AD10846DE
:101BB00004F0F2FAA0F1020A59F8240004F0ECFA59
:101BC000824500D094E087E003AA4FF48071AC48CE
:101BD000FFF7E2FC0290029888B9069908988842BB
:101BE00001D1012000E0002018B1002048F82400B5
:101BF0007CE003A8FEF7B4FB6FF0020064E7002767
